:020000020000FC
:060000000C946B0C0C9443
:1000060000000C9400000C9400000C9400000C946A
:100016005D0D0C948B0D0C94B90D0C94E70D0C949E
:10002600F90D0C94000E0C9400000C9400000C9436
:1000360000000C9400000C9400000C9400000C943A
:100046007D100C9400000C9400000C9400000C949D
:1000560089100C9400000C9400000C9400000C9481
:1000660003140C9400000C9400000C9400000C94F3
:1000760000000C9400000C9400000C94A30F0C9448
:1000860000000C9400000C9400000C94A1150C9434
:1000960000000C9400000C9400000C9400000C94DA
:1000A60000000C94DC0F0C9400000C9400000C94DF
:1000B60000000C9400000C9400000C9400000C94BA
:1000C60000000C9400000C948E170C9400000C9405
:1000D60000000C9402190C9400000C9400001027E8
:1000E600E80364000A00010000100001100001008E
:1000F6004D6F6E746167004D6F6E6461790044697F
:10010600656E737461670054756573646179004D3B
:10011600697474776F6368005765646E65736461AC
:100126007900446F6E6E657273746167005468750A
:10013600727364617900467265697461670046721C
:10014600696461790053616D73746167005361740A
:10015600757264617900536F6E6E746167005375D2
:100166006E64617900002042726964676520626F7F
:1001760061726420666F756E64002072756E6E69BA
:100186006E6720626F617264206861726477617263
:100196006520746573742E2E2E2E00444332632E12
:1001A60030342E31312032302E30332E323032334D
:1001B600004443322053577665723A200044433256
:1001C600635F6F63743230323200444332204857E3
:1001D6007665723A2000504F32655F6E6F76323028
:1001E600323200504F322048577665723A2000521C
:1001F600616D204572726F720052616D204F4B0027
:1002060020204443322074696D653A200020204442
:10021600433220646174653A20005254432F545788
:1002260049206572726F72002020696E742E2065F7
:100236006570726F6D206572726F72002020696E34
:10024600742E20656570726F6D204F4B00444332EB
:100256002055494420696E206865783A2000444359
:10026600322055494420696E206465633A20007641
:100276006F6C74616765206572726F720020496EDB
:1002860070757420766F6C74616765205B6D565D62
:100296003A200054656D70657261747572652065EB
:1002A60072726F72002054656D706572617475723A
:1002B60065205BB0435D3A2000202064696769745D
:1002C600616C2074657374206572726F723A2000D7
:1002D60020206469676974616C2074657374204FAB
:1002E6004B005254432D436C6F636B206572726FE3
:1002F60072005254432D545749206572726F720032
:1003060052544320697320776F726B696E67006F72
:10031600766572616C6C2073756363657373006FC9
:10032600766572616C6C206661696C7572650065D4
:1003360078742E20656570726F6D206572726F72AB
:10034600006578742E20656570726F6D20333220DB
:100356006B42204F4B006578742E20656570726F76
:100366006D203634206B42204F4B006578742E206A
:10037600656570726F6D2039366B42204F4B203F9A
:100386003F3F006578742E20656570726F6D203171
:100396003230206B42204F4B0000676F74206D6433
:1003A60062204E414B006D64622072657370206559
:1003B60072726F72007265706561742073746F700B
:1003C600006D6462206F6666006D6462206F6E0069
:1003D6006D646220737461727420706F6C6C696EE8
:1003E60067006D64622073746F7020706F6C6C6947
:1003F6006E67006D64622072657065617400656D7C
:1004060070206F666600454D5020636F756E74727E
:10041600793A2000454D50207363616C653A20009F
:10042600454D5020646563696D616C733A200065C3
:100436006D70207061792073746172742000656D2F
:1004460070207061792073746F702000656D702064
:10045600676F742068436F696E2000656D70206752
:100466006F7420636F696E2000656D702072642062
:10047600657272002D64796E5072302D002D64798C
:100486006E5072312D002D64796E5072322D002D12
:1004960064796E5072332D002D64796E5072342D4E
:1004A600002D64796E5072352D002D64796E507270
:1004B600362D002D64796E5072372D002D2D2D208E
:1004C60041544220476D6248202D2D2D002D2D2DA3
:1004D600205053412031323536202D2D2D002D2D23
:1004E6002054657374205072696E74202D2D004C53
:1004F6004F474F3A0073697A6520322F32004261C6
:1005060072436F646520322F353A00313233343509
:1005160036373839303132333435363738393000BA
:100526002D2D2D2D2D2D2D2D2D2D2D2D2D2D2D2DF5
:100536002D2D2D2D2D2D002020202020746869734F
:1005460020697320612074696E792074657874005F
:100556006E6F726D616C207465787400746869736F
:100566002069732061206869676820746578740063
:100576002020426F6C6420546578742000756E6488
:1005860065726C696E656420746578740020696EA6
:10059600766572732074657874005072696E74653E
:1005A60072206572726F7220002020204163636F93
:1005B600756E74696E672072656365697074004351
:1005C60061736820626F78206368616E6765206E6C
:1005D600723A200061743A00446174652028797982
:1005E6002F6D6D2F6464293A20002F0054696D65C4
:1005F600202868683A6D6D3A7373293A20004C6F6B
:1006060063616C20636F696E7320696E206361732A
:100616006820626F783A00546F6B656E203A20004E
:10062600466F726569676E20636F696E7320696EC7
:10063600206361736820626F783A00546F6B656E51
:1006460000318000328000302C358000302C328022
:1006560000302C318000437573746F6D65722D4EBA
:10066600722E3A20004D616368696E652D4E722EBA
:100676003A20004162732E566F6C756D653A200004
:100686004162732E4E72206F6620637574733A2032
:10069600006578636867616E676520726174653AA4
:1006A600200041544220476D6248204C7568652001
:1006B6004765726D616E79007072696E746572203D
:1006C60074656D706C61746520002D2D2D20656E2E
:1006D60064206F662066696C65202D2D2D00444FC1
:1006E60057206E6F7420736574007468697320698F
:1006F60073206120322F35626172636F646500007A
:100706003C20536C61766520526573706F6E73651D
:1007160000444332635F6F63743230323200504FAD
:1007260032655F6E6F763230323200444332632E6A
:1007360030342E31312032302E30332E32303233B7
:1007460000007468697320697320616E2041544209
:1007560020616363657373206361726400004443C0
:100766006D616B655265736574002D00776F6B65FF
:100776006E206279206D646200776F6B656E206211
:100786007920636F696E00776F6B656E20627920E2
:100796007074750074726967676572696E67206840
:1007A60065617274626561742E2E2E00706F7765B6
:1007B6007220646F776E006C696768742077616B6E
:1007C600650066756C6C2077616B65007374617289
:1007D60074696E6720626F6F746C6F616465722EE8
:1007E6002E2E0000746573742063616E63656C6CF5
:1007F6006564007374617274696E6720436F696E15
:10080600436865636B657220746573742E2E2E00C3
:1008160077696C6C2062652073746F7070656420F4
:1008260061667465722032307320776974686F75FB
:100836007420636F696E00496E7365727420636F0E
:10084600696E7320706C656173653A00656D702022
:10085600696E2069646C6520737461746500656DEA
:10086600702073746F7000656D70207761697469AC
:100876006E6720666F7220636F696E7300207E3E1E
:100886002076616C75653D00636F696E20746573D3
:100896007420656E640072756E6E696E672073747F
:1008A60061727475702074657374732E2E2E0052E7
:1008B600616D204F4B0052616D206572726F722020
:1008C600666F756E6400426F617264206877204FB0
:1008D6004B00426F617264206877206572726F7296
:1008E6002000527463206572726F72200052746326
:1008F600206F6B00556964206572726F7220005517
:100906006964206F6B00557070657220646F6F723A
:10091600206973206F70656E005661756C74206473
:100926006F6F72206973206F70656E004261747418
:1009360065727920646F6F72206973206F70656EBF
:1009460000446F6F7273206F6B0054656D70657233
:100956006174757265206572726F72200054656DE0
:100966007065726174757265206F6B00566F6C747A
:10097600616765206572726F722000566F6C7461D4
:100986006765206F6B00496E746565206572726FCE
:10099600722000496E746565206F6B00457874653A
:1009A60065206572726F7220004578746565206FE8
:1009B6006B00436F696E20657363726F7720657293
:1009C600726F722000436F696E20657363726F7772
:1009D600206F6B005072696E746572206572726F5B
:1009E6007220002020206E6F2070617065720020DA
:1009F60020206E6F74207265616479002020206E5D
:100A06006F20726573706F6E736500202020696EAB
:100A16007465726E616C206572726F7200202020A0
:100A260068656164206F70656E005072696E7465EA
:100A360072206F6B002020206C6F772070617065CC
:100A460072004E6F20636F696E20736166650043A6
:100A56006F696E2073616665206F6B004E6F206252
:100A6600696C6C20626F780042696C6C20626F78EA
:100A7600206F6B004D6462206572726F72004D6468
:100A860062206F6B004D6966526561646572206F06
:100A96006B004D6966526561646572206572726F9E
:100AA600722000436865636B696E67206D6F6465CD
:100AB6006D2C20706C7320776169742E2E2E004386
:100AC6006F696E20636865636B6572206F6B0043A8
:100AD6006F696E2063686B206572726F72200046C4
:100AE6006F756E64204552524F5228732900537910
:100AF6007374656D206F6B00444332632E30342E61
:100B060031312032302E30332E32303233004443EE
:100B1600322053577665723A2000444332635F6F42
:100B2600637432303232004443322048577665725D
:100B36003A2000504F32655F6E6F763230323200A7
:100B4600504F322048577665723A20004D6F6465E3
:100B56006D206F6B007265676973746572656400FA
:100B66005369676E616C20004D6F64656D20657218
:100B7600726F72200077726F6E67207479706500ED
:100B860053494D206E6F74207265616479007465F7
:100B96007374696E67207072696E7465722E2E2E7C
:100BA600000041542B4353510041542B43524547B7
:100BB6003F0041542B434C54533D3F002B4353516C
:100BC6003A20002B435245473A20004154004F4BF0
:100BD6000061742B6970723D31313532303000411D
:100BE6005445300041542B434C54533D310041543D
:100BF600490053494D37303030470041542B435359
:100C0600494D3D3F000006046F04DF045705D70534
:100C16005E06EC0682072008C5087109250AE10A66
:100C2600A40B6E0C400D170EE90EA80F4610B81057
:100C3600301106046F04DF045705D7055E06EC067F
:100C460082072008C5087109250AE10AA40B6E0C63
:100C5600400D170EE90EA80F4610B810301100010E
:100C660002030405060708090A0B0C0D0E0F0010F7
:100C760000006410B71DC8206E3BAC30D9269041E9
:100C8600DC76F4516B6B5861B24D3C710550208394
:100C9600B8ED44930FF0E8A3D6D68CB361CBB0C2BF
:100CA600649BD4D2D38678E20AA01CF2BDBD4174FF
:100CB6006250736131323536507475355F210037B5
:100CC60078A730203F3F660041544256414C554577
:100CD6004341524456303032000076616C696420DC
:100CE6004D696661726563617264205365727669E7
:100CF600636520646F6F720076616C6964204D696C
:100D06006661726563617264205661756C742064F5
:100D16006F6F720066696C6520697320746F6F204F
:100D26006269672C206D617820383030627974658D
:100D360000616C6C20636F756E74657273206465F8
:100D46006C6574656400736C656570206D6F6465B1
:100D5600206F666600736C656570204F4B00706C83
:100D66006561736520776169742E2E2E002D2D2DF9
:100D76002D2D2D2D2D2D2D2D2D2D2D2D2D2D2D2D9D
:100D86002D2D2D2D2D2D2D2D2D2D2D2D2D2D2D2D8D
:100D96002D2D2D2D2D2D2D2D2D2D2D2D2D2D2D00AA
:100DA6002D2D2D2D2D2D2D2D2D202044657669637D
:100DB6006520436F6E74726F6C6C65722048656C4B
:100DC600702053637265656E202D2D2D2D2D2D2DD2
:100DD6002D2D007C2D2D2D2D2D2D2D2D2D2D2D2D1B
:100DE6002D2D2D2D2D2D2D2D2D2D2D2D2D2D2D2D2D
:100DF6002D2D2D2D2D2D2D2D2D2D2D2D2D2D2D2D1D
:100E06002D2D2D2D2D007C007C20202027502720E5
:100E16003D20446973706C6179204D616368696E29
:100E2600652053657474696E6773007C20202027E3
:100E36005327203D20446973706C617920446576A0
:100E4600696365205374617465007C2020202757F0
:100E560027203D20446973706C61792057616B656A
:100E660020536F75726365007C202020277427202D
:100E76003D2052756E20636F6D706C6574652073CE
:100E8600797374656D20636865636B2028313773E9
:100E960029007C202020277027203D205072696E73
:100EA6007420546573747469636B6574007C2020C8
:100EB60020276327203D2052756E20636F696E20C0
:100EC6007465737409090909276227203D206F702C
:100ED600656E20636F696E20626C6F636B6572006E
:100EE6007C202020277527203D206F70656E207599
:100EF6007070657220636F76657209090927762717
:100F0600203D206F70656E207661756C7420646F6D
:100F16006F7220636F766572007C202020276C2715
:100F2600203D206C6564206F6E2033730909090922
:100F360009276F27203D206C6564206F6666007C5C
:100F4600202020273027203D20736C656570206F98
:100F56006666202873746179206177616B65292044
:100F6600202020273127203D20736C656570206F77
:100F76006E202864656661756C7429007C202020CB
:100F8600277327203D20736972656E206F6E206679
:100F96006F7220313073007C2020202764787827F8
:100FA600203D205072696E74205469636B6574200D
:100FB6006E72207878203D2030312E2E3332007C20
:100FC600202020276B636363636327203D20636FC4
:100FD6006C6C65637420616D6F756E742028356462
:100FE60069676974732920696E2063656E74007C75
:100FF600202020276527203D656E636173682020C9
:10100600202020277227203D2072657475726E207D
:10101600636F6C6C656374656420616D6F756E7467
:10102600007C20202073656E64206A736F6E2D66C7
:10103600696C652077697468202253454E442046C2
:10104600494C452D427574746F6E004D6163686935
:101056006E652053657474696E67733A00437573E1
:10106600746F6D65724E723A20004D616368696EE9
:10107600654E723A202000426F726F7567683A209B
:10108600202020005A6F6E653A2020202020202044
:1010960000416C6961734E723A20202020004D7920
:1010A600506C6163653A20004D6173746572204926
:1010B6006E746572666163653A0043757272656E39
:1010C600742042617564726174653A2000202020A4
:1010D60020303D393630302020313D31346B3420DC
:1010E60020323D31396B322020333D33386B34208A
:1010F60020343D35372C362020353D3131356B32A5
:101106002020363D3233306B3400437263206368EF
:1011160065636B3A20005061726974793A20002049
:1011260020202020202F2F207061726974793A20A8
:10113600303D6E6F2020313D6576656E2020323D54
:101146006F64640044617461626974733A200020BC
:1011560020202020202F2F20646174612062697472
:10116600733A20303D356269742020313D3662691C
:1011760074202020323D37626974202020333D38A8
:10118600626974202020343D396269740053746F9B
:1011960070626974733A20002020202020202F2FAF
:1011A60020303D3173746F706269742020202031C5
:1011B6003D3273746F706269747300446576696357
:1011C60065733A005072696E746572202020202083
:1011D6003A2000436F696E43686B20202020203A36
:1011E60020004D69666172652020202020203A206B
:1011F600004D61696E73537570706C79203A2000EA
:101206004D6F64656D202020202020203A20004369
:1012160072656469744361726420203A20004573E4
:1012260063726F772020202020203A200052656AC2
:101236004D6F746F72202020203A20005368757419
:1012460074657220202020203A200042696C6C20B0
:10125600202020202020203A20005661756C744CF6
:101266006F636B2020203A20004175746F416C61DA
:10127600726D2020203A20004175746F4F70656EA4
:10128600202020203A20004163635265636569701F
:101296007420203A2000446F6F725265636569704E
:1012A60074203A2000546F6B656E526563656970F1
:1012B600743A20005374617465206F6620616C6C0B
:1012C60020446576696365732028313D4F4B2020A5
:1012D6003178783D7761726E696E67202032787852
:1012E6003D6572726F72290052616D3A2000496E37
:1012F6007445653A200045787445653A2000527475
:10130600633A20004272642048573A200050726EB9
:101316003A20004D6F64656D3A20005369676E612F
:101326006C3A20005265676973743A20004D646216
:101336004275733A2000436F696E43686B3A20002A
:10134600457363726F773A20004D69665265616432
:101356003A200043437465726D3A200052656A650F
:1013660063743A20005661756C743A200042696CC9
:101376006C626F783A2000566F6C743A20005465A0
:101386006D703A20005077724F6E5473743A200095
:10139600446F6F7253746174653A2000446F6F72C4
:1013A6005761734F70656E3A20004368616E6765DA
:1013B600723A2000436F696E536C6F743A20004294
:1013C600696C6C3A20004C617374205265736574C5
:1013D6002062793A2000416C6C20436865636B6536
:1013E600643A2000416C61726D3A200044433263D6
:1013F6002E30342E31312032302E30332E323032F0
:1014060033004443322053577665723A20004443F2
:1014160032635F6F637432303232004443322048A5
:10142600577665723A2000504F32655F6E6F76329E
:1014360030323200504F322048577665723A2000DB
:10144600616C6C2064796E616D69632076616C7580
:1014560065733A006B657074206177616B65206215
:10146600793A2000646F6F725F6F70656E3A200084
:10147600757020006D6964646C652000646F776E1A
:10148600200020616C6C20646F6F727320636C6F38
:10149600736564206E6F77200020202F6F6E416C7D
:1014A60061726D0020202F43426368616E6765009C
:1014B60020202F4E6F436F696E626F780020202FB9
:1014C60055626174745B565D3D0020202F54656D36
:1014D600705BB0435D3A20006572726F7220696E70
:1014E60020636F6E6669672066696C6500636F6E60
:1014F60066696720757064617465207375636365DA
:101506007373006572726F7220696E2073657269FB
:10151600616C2066696C650073657269616C207523
:1015260070646174652073756363657373006572B7
:10153600726F7220696E20646576696365206669DC
:101546006C650064657669636520757064617465B1
:101556002073756363657373006572726F722069B9
:101566006E20636173682066696C650063617368E9
:1015760020757064617465207375636365737300A9
:101586006572726F7220696E207072696E747878F7
:101596002066696C65007072696E74787820757063
:1015A6006461746520737563636573730065727235
:1015B6006F7220696E2074696D652066696C6500BE
:1015C60074696D65207570646174652073756363F5
:1015D6006573730077726F6E672066696C65007459
:1015E60069746C65003F3F3F444332435F636F6EEF
:1015F600666967003F3F3F444332435F73657269E4
:10160600616C003F3F3F444332435F6465766963E4
:1016160065003F3F3F444332435F63617368202068
:10162600003F3F3F444332435F707269003F3F3F94
:10163600444332435F74696D6500637573744E7518
:101646006D006D6163684E756D00626F726F7567D0
:1016560068007A6F6E6500616C696173006C6F6318
:101666006174696F6E0063726343686B00626175D3
:1016760064526174650064617461007061726974BA
:10168600790073746F70007072696E7465720063AE
:101696006F696E43686B006D6966526400736F6CA8
:1016A6006172507772006D6F64656D006372656478
:1016B60069744361726400657363726F7700526583
:1016C6006A4D6F746F720073687574746572006228
:1016D600696C6C5264007661756C744C6F636B0058
:1016E6006175746F416C61726D006175746F4F70D6
:1016F600656E004163635072696E7400446F725088
:1017060072696E7400546F6B5072696E7400434256
:101716007761726E4C65760043426572724C6576EF
:1017260000436F696E44656E6F6D00436F696E5658
:10173600616C756500436F696E4163636570740023
:1017460045786368616E67655261746500546F6BB6
:10175600656E4368616E6E656C0042696C6C5661BD
:101766006C75657300637572722E796561720063BC
:101776007572722E6D6F6E746800637572722E6468
:101786006F6D00637572722E686F75720063757285
:10179600722E6D696E00637572722E7365630063D7
:1017A6007572722E646F770070726F6A656374006B
:1017B6007465787400697373756564007374796C05
:1017C600006665656400766172690067726166002D
:1017D60063617368207374617274207061796D65DA
:1017E6006E7400636173682073746F700063617355
:1017F600682072656164790063617368206C617347
:101806007420636F696E00656D702073746F7070FD
:10181600656420756E65787065637465646C79209F
:1018260000206361736820676F7420636F696E3A86
:10183600200020746F74616C3A2000636173682025
:101846007374617274436F6C6C20776974682000DE
:1018560063617368207365747570200073746F70AC
:10186600207061796D656E74206174200063616E0D
:1018760063656C207061796D656E742061742000FB
:101886005073613E0054696D3E004162733E004DE7
:1018960077203E00426F783E0056616C3E00456EF2
:1018A600643E00000A000000000000000000000086
:1018B6000000000000000000000000000000000022
:1018C6000000000000000100C71BAA18000000006D
:1018D600F894EE27EFBBF1E0F5BFE5BFE0937400A7
:1018E600E09375008DE0A2E0BB27ED938A95E9F7BA
:1018F60080E090E2A0E0B2E0ED930197E9F7ECEC2E
:10190600F8E1D0E0DBBF87919791009781F0A7912E
:10191600B79107901790C791D791BF01DBB7F00138
:10192600CBBF07900D920197E1F7FB01EBCFE0E00B
:10193600EEBBEFEFEDBFE1E2EEBFC0E0DAE00C9404
:101946003B6F0E9406C21A2F2B2F3C81343010F4B5
:101956000C94AE0C30E03295307F330F330F307C71
:1019660030937C00E7E9E0937A00012FAEE7B0E020
:10197600EC91E02BEC93EFEF0E27E0B3E023E0BB16
:10198600122F2227012FADE7B0E0EC91E02BEC936C
:10199600EFEF0E27A7E0B1E0EC91E023EC930E9475
:1019A6000DC225960895E0E0E0937A0008950A9323
:1019B6000A2F003110F40C94E30CE0E0099108952D
:1019C600083010F40C94EE0CE0917B00E860E09394
:1019D6007B00077005C0E0917B00E77FE0937B000A
:1019E600083010F00C94060DE0917C00E87FE0933F
:1019F6007C00ACE7B0E0EC91E02BEC93E0917A0050
:101A0600E064E0937A00E1E0099108950E9407C23C
:101A160000E010E0E0917A00E0712E2F81E791E07E
:101A26000197F1F7203011F00C94230DF80131964F
:101A36008F01E436A0E0FA0710F00C94230D01C0E4
:101A460001C0E8CFE0917A00E061E0937A0000916E
:101A56007800109179000E94FAAC0895E0E0EDBBA1
:101A6600E093680008950A930A2F003011F00C9451
:101A7600450DE0916A00E2600E94FFACEE7FE093C4
:101A86006A00EC9A013011F00C944F0DE0916A0057
:101A9600E360E0936A00EC9A023011F00C94590D61
:101AA600E0916A00EC7FE0936A00EC9A0991089550
:101AB600EC9808950E9404AD0E94FF730E9416AD33
:101AC60018950A930A2F003011F00C94730DE091CB
:101AD6006A00E8600E94FFACEB7FE0936A00ED9A33
:101AE600013011F00C947D0DE0916A00EC60E093FA
:101AF6006A00ED9A023011F00C94870DE0916A00AD
:101B0600E37FE0936A00ED9A09910895ED980895B0
:101B16000E9404AD0E9415740E9416AD18950A9392
:101B26000A2F003011F00C94A10DE0916A00E062DA
:101B36000E94FFACEF7EE0936A00EE9A013011F04E
:101B46000C94AB0DE0916A00E063E0936A00EE9AB4
:101B5600023011F00C94B50DE0916A00EF7CE09331
:101B66006A00EE9A09910895EE9808950E9404ADD0
:101B76000E942A740E9416AD18950A930A2F003007
:101B860011F00C94CF0DE0916A00E0680E94FFAC62
:101B9600EF7BE0936A00EF9A013011F00C94D90DB7
:101BA600E0916A00E06CE0936A00EF9A023011F06F
:101BB6000C94E30DE0916A00EF73E0936A00EF9AEC
:101BC60009910895EF9808950E9404AD0E943D740E
:101BD6000E9416AD18950E9428AD0E9428AD0E945D
:101BE60028ADA8E6B0E0EC91EC9308950E9404AD10
:101BF6000E948C740E9416AD18950E9404AD0E9436
:101C06008F740E9416AD18950D9400F008950E94E9
:101C16002EADF99B01C0FDCF22BD11BDF89A00B5CE
:101C26000E9433AD08950E9438ADF99B01C0FDCFE7
:101C360009851A852F81388540E0F901A42FB0E087
:101C4600AE17BF0710F00C94330E0E943DADAD8168
:101C5600BE81EE27A40FBE1FE0B5EC934F5FEDCF1C
:101C66000E940CC22B9608950E9405C22A2F3D8120
:101C76004E81F99B01C0FDCF1FB742BD31BDF89A19
:101C860000B5201711F40C944D0E20BDE4E0EFBB17
:101C9600E2E0EFBB17FF01C078940E940CC22796C2
:101CA60008950E9444ADF99B01C0FDCF0C851D85AA
:101CB6002A853B85EFB7EE8340E0F901A42FB0E01B
:101CC600AE17BF0710F00C94810EA885B985EE27D4
:101CD600A40FBE1F5C910E943DADE0B5EF83AF81BE
:101CE6005A1711F40C947F0E50BDE4E0EFBBE2E00E
:101CF600EFBBF99B01C0FDCF4F5FDFCFEE81E078F0
:101D060011F40C94870E78940E940BC22E960895B7
:101D16000A932B9823982A98229A2998219A289AE6
:101D2600209A02E0E02FE03011F00C949F0EE1E0E3
:101D3600EDBDE0E5ECBD35C0E13011F00C94A80E28
:101D4600E0E0EDBDE0E5ECBD2CC0E23011F00C9416
:101D5600B10EE1E0EDBDE1E5ECBD23C0E33011F0ED
:101D66000C94BA0EE0E0EDBDE1E5ECBD1AC0E4303E
:101D760011F00C94C30EE1E0EDBDE2E5ECBD11C03F
:101D8600E53011F00C94CC0EE0E0EDBDE2E5ECBDE3
:101D960008C0E63011F00C94D40EE0E0EDBDE3E5AA
:101DA600ECBD09910895E0E0ECBD0895E0E0E4BDE6
:101DB600E5BDE0936E00E093B000E093B100E093E0
:101DC6007000E093B600E3BDE0938000E0939000DE
:101DD600E093A000E0932001E0938100E09391005E
:101DE600E093A100E0932101E0938200E09392004A
:101DF600E093A200E0932201E0936F00E09371006C
:101E0600E0937200E093730008951A930A931CE01E
:101E1600E3B70E2FAE2FE5E0EA23AE2FE5E00E94F2
:101E2600A3C2E03011F40C94290FE12FE1501E2FCC
:101E3600EF5FAE2FEAE00E94ADC2E03011F40C94E1
:101E4600250FF3CFE0E0099119910895E0E0E4BD94
:101E5600E1E0E5BDE0E0E7BDE6EBF0E0DF01E0E074
:101E6600EC93E6BDE6B5AE2FE7E30E94A8C2E030EC
:101E760011F40C943F0FF6CFE0E009911991089503
:101E86000E9406C29D017894E0E0F0E08F010E9476
:101E9600080FF80131968F013197F801FF93EF9300
:101EA600F901AF91BF910E94B8C2E03011F40C94D1
:101EB6005D0FEDCFE7E0F0E08F018F010E940DC2CC
:101EC600249608950E9404C2AD01FA019F01E0E044
:101ED600F0E08F01E4E6F0E0DF010E94430FF80135
:101EE60031968F013197F801FF93EF93F901AF9186
:101EF600BF910E94B8C2E03011F40C94830FEACF70
:101F0600E8E0F0E08F018F010E940BC2269608954B
:101F1600E0E0E0939000E09392000E944AADE091E9
:101F26007100E260E0937100E2E0E0939100E8E482
:101F3600E0939900E0E0E0939800EFEFE8BB0895A6
:101F46000E9404AD0E944AADA0E0BAE00E9450ADE6
:101F56000E948774A4E0BAE00E9450ADA091040AE2
:101F6600B091050AA436E0E0BE0710F40C94C60F43
:101F7600E0E0E093040AE093050AA2E0BAE00E94DA
:101F860050AD0E948674EFEFE8BB0E9416AD18951F
:101F9600A0919100A03011F40C94D80FA09171007B
:101FA600A03011F40C94D80F02C0E0E00895E1E0EF
:101FB600089518950A930A2F083210F40C94E60F28
:101FC600E1E009910895E02F0E9456ADEA0FFB1F4C
:101FD600A091000AB091010AA083B183E0E00991C3
:101FE60008950E9404C25A2F583210F40C94FF0F21
:101FF6000E945CAD26960895452F2091000A3091E7
:10200600010AE42F0E9456AD0E9461AD10F40C94B3
:102016001710E42F0E9456AD0E9468ADDF01F9014A
:10202600EA1BFB0B8F0107C0E42F0E9456AD0E94EE
:1020360068AD0E946DADF8010E940BC22696089508
:102046000A930A2F043110F40C942C10E1E0099144
:102056000895E02F0E9477ADEA0FFB1FA091020AB8
:10206600B091030AA083B183E02FF0E0E258F54F68
:10207600A1E0A08309910895AA930E9405C24D810B
:10208600443110F40C944D10E0E0F0E00E940CC2D4
:1020960026960895E42FF0E0E258F54FE081E0300F
:1020A60011F00C945A100E947DAD26960895209149
:1020B600020A3091030AE42F0E9477AD0E9461ADB7
:1020C60010F40C947110E42F0E9477AD0E9468AD55
:1020D600DF01F901EA1BFB0B8F0107C0E42F0E9409
:1020E60077AD0E9468AD0E946DADF8010E940CC2EA
:1020F600269608950E9404ADE0E0E0938500E09303
:1021060084000E948A740E9416AD18950E9404AD40
:10211600E0E0E6BD0E948B740E9416AD18952C97E0
:102126000A930E9482AD0E9487AD0E948CAD0E94E8
:102136008CADEAB1E360EAB9EBB1E360EBB9E091EB
:102146006400EF77E0936400E4E0E093BC00E98587
:10215600FA856B857C850E9495AD0E949AAD0E949A
:102166009FAD0E94A4AD0E94A7ADE051F040604033
:1021760070400E94ACAD0E9499C20E9495AD00E0ED
:102186000E949FADA030E1E0BE07E0E08E07E0E0F0
:102196009E0710F40C94D9100E949FADE4E0F0E085
:1021A60060E070E00E94A4AD0F5FEACFED81E0939E
:1021B600B8000093B90008812D960895E0E0E093F9
:1021C600BC00E0916400E068E0936400EAB1EC7F53
:1021D600EAB9EBB1E360EBB908950E94AFAD0F5FCA
:1021E6001F4F81E38A95F1F7E091BC00E07811F08A
:1021F6000C9404110436E0E01E0714F00C9404114C
:1022060001C001C0ECCF0436E0E01E0714F40C94C4
:102216001011E1E0099119910895E0E009911991F1
:1022260008950E94B4AD022F4093BB00303011F4E4
:102236000C942111E4EAE093BC0003C0E4E8E093C7
:10224600BC000E94F0101E2F113010F40C943011B7
:10225600EAE00E940CC227960895E091B900E87F53
:102266000E1711F40C943F11E4E9E093BC00E1E091
:102276000E940CC227960895E0E00E940CC22796A1
:1022860008950E9407C20E94E110509A51985998E9
:10229600AAE0B0E00E9471C5E9B1E1700E2FE9B184
:1022A600E2701E2F103011F00C94751120E0589832
:1022B6008AE08A95F1F7589A8AE08A95F1F7E9B1AA
:1022C600E2701E2F2F5F103011F00C946F11203228
:1022D60010F00C946F1101C001C0E9CFA2E0B0E08C
:1022E6000E9471C5103011F40C947B110E9492105B
:1022F600A2E0B0E00E9471C50E940EC22396089526
:102306000E9444AD0E94BAAD11F00C948D11077075
:10231600000F202B0E94C5AD11F40C9495110E945C
:10232600D0AD08950E94D5AD11F00C949F11E2E056
:102336000E940BC22F960895313011F00C94A6110D
:102346000E94DEAD0895503011F40C94B2110E9433
:10235600E3AD11F40C94B2110E94ECAD08950E9405
:10236600F1AD11F40C94BA110E94ECAD0895E0E0C1
:10237600EE83EF830E94FAADAE17BF0710F00C9400
:10238600D8110E94FFADAE0FBF1FEC91EA93E0E0BB
:10239600EA93A8E20E9404AE11F40C94D5110E94AF
:1023A60009AE08950E940EAEE5CF0E9414AE0895C0
:1023B6000E941CAE0E9423AE0E9483110E2F013094
:1023C60010F40C94E8110E944411013010F40C949E
:1023D600F2111F5F153010F00C94F21101C001C00C
:1023E600E9CF7894013010F40C94F911E02F0E9493
:1023F6000BC22B9608950E9444AD0E94BAAD11F00F
:102406000C9408120770000F202B0E94C5AD11F422
:102416000C9410120E94D0AD08950E94D5AD11F013
:102426000C941A12E2E00E940BC22F9608953130E6
:1024360011F00C9421120E94DEAD0895503011F473
:102446000C942D120E94E3AD11F40C942D120E94EF
:10245600ECAD08950E94F1AD11F40C9435120E9472
:10246600ECAD08950E942DAEA0E10E9404AE11F4D9
:102476000C9440120E94D0AD089521602A93E0E0AA
:10248600EA93A0E40E9404AE11F40C944D120E944B
:10249600DEAD08954150E0E0EE83EF830E94FAAD91
:1024A600EA17FB0710F40C94A8120E94FAADEA177B
:1024B600FB0711F00C946312E4E8E093BC0003C040
:1024C600E4ECE093BC000E94F010E03011F40C94B0
:1024D6006F120E9409AE0895E091B900E87FE035D9
:1024E60011F00C947E120E94FAADAE17BF0710F0E1
:1024F6000C947E1201C008C00E94FFADAE0FBF1F34
:10250600E091BB00EC931EC0E091B900E87FE8358E
:1025160011F00C9496120E94FAADEA17FB0711F01F
:102526000C94961201C008C00E94FFADAE0FBF1FEB
:10253600E091BB00EC9306C0E4E9E093BC000E9486
:1025460009AE08950E940EAEA9CF0E9414AE08955A
:102556000E941CAE0E9423AE0E94FE110E2F013077
:1025660010F40C94B8120E944411013010F40C942B
:10257600C2121F5F153010F00C94C21201C001C0C8
:10258600E9CF7894013010F40C94D41210E0E88569
:102596001E1710F00C94D4120E9432AEEC931F5FFB
:1025A600F6CFE02F0E940BC22B960895A091C40D82
:1025B600A23010F40C94E412AE3F10F00C94E41226
:1025C60001C005C0E091C40DEF5FE093C40DA0917A
:1025D6002E0EA23010F40C94F512AE3F10F00C94AF
:1025E600F51201C005C0E0912E0EEF5FE0932E0EAE
:1025F600A0915E11A23010F40C940613AE3F10F0B9
:102606000C94061301C005C0E0915E11EF5FE093E4
:102616005E11A091C811A23010F40C941713AE3FAE
:1026260010F00C94171301C005C0E091C811EF5FBC
:10263600E093C81108950A930A2FE02FE13011F0B4
:102646000C942813EFE309910895E23011F00C94ED
:102656002F13EFE209910895E33011F00C9436132D
:10266600E7E109910895E43011F00C943D13EFE091
:1026760009910895E53011F00C944413E7E00991AF
:102686000895E63011F00C944B13E3E00991089598
:10269600EFE5099108950E9437AEE093C000E0E0AF
:1026A600E093C100E093C200E093C500EAE2F3E0E4
:1026B600E093C20DF093C30DA091C20DB091C30D6E
:1026C600139710F00C946D13E3E0F0E0E093C20D65
:1026D600F093C30DA32F0E941E13E093C400E22FB4
:1026E600E13011F00C947D13E091C200E260E093BA
:1026F600C20022C0E23011F00C948713E091C200B0
:10270600E460E093C20018C0E33011F00C9491131A
:10271600E091C200E660E093C2000EC0E43011F022
:102726000C949F13E091C200E660E093C200E09132
:10273600C100E460E093C100E12FE13011F00C9498
:10274600A913E091C200E860E093C200E02FE130F7
:1027560011F00C94B413E091C200E062E093C20061
:1027660009C0E23011F00C94BD13E091C200E063A1
:10277600E093C200E42FE13011F00C94C813E0910D
:10278600C100E861E093C10009C0E23011F00C9489
:10279600D113E091C100E869E093C1000E940CC228
:1027A60029960895E0E0E093C10008950A930A2F60
:1027B600E091C000E07211F00C94E213F9CF00939F
:1027C600C600099108950E94AFAD0E9440AE0E1753
:1027D6001F0710F00C94F613A5E9BAE00E9445AE67
:1027E6000F5F1F4FF2CFE0E0E093BF0DE093C00D07
:1027F600E093C10DE1E0E093C40D099119910895AC
:102806000E944AAE0E9406C2A091C40DA13010F4E7
:102816000C941014E2E0E093C40DE091C100E47062
:1028260011F40C944A140E9440AE32970E9451AEA5
:1028360010F00C943814E091C100E27011F40C947D
:102846002C140E9458AE3197EB56F54FA1E0A083A9
:1028560007C00E9458AE3197EB56F54FA0E0A08313
:102866000E9458AE0E945BAE02C00091C600E09185
:10287600BF0DE2501E2FF0E0EB56F54F0E9463AEFF
:10288600EB56F54FE081F0E02E2B3F2B0EC00E9459
:1028960040AE0E9451AE10F00C9456140E9458AEF1
:1028A6000E945BAE02C00091C600E091C000EC71D0
:1028B6000E2F013010F40C946714A091C10DA030B6
:1028C60011F00C94671401C002C00093C10D0E9460
:1028D6000DC224960E946BAE18950E9472AE0895A2
:1028E6000E9404C2AD01A091BF0DB091C00D4A1760
:1028F6005B0710F00C948114FA0102C00E9472AEBC
:102906009F0100E010E00217130710F00C949414D6
:102916000E9477AEA5E9BAE00E947EAE0F5F1F4F18
:10292600F2CF0E9484AEA436E0E0BE0710F00C940D
:10293600A0140E9472AE0E9489AE0E940BC2289615
:1029460008950E9490AE0E9497AE10F40C94AE14B7
:10295600A22F0E94D913003DE7E01E0710F00C9449
:10296600B914213010F40C94B91401C001C0EBCF96
:1029760078940E940CC2259608950E949FAE00E0AE
:1029860010E00217130710F00C94D214F801E40FAC
:10299600F51FA0810E94D9130F5F1F4FF2CF0E942F
:1029A6000BC2289608950E9437AEE093C800E091C6
:1029B600C900EC79E093C900E091C900E861E093B1
:1029C600C900E091CA00EE73E093CA00E0E0E0932C
:1029D600CD00E4E6F0E0E0932C0EF0932D0EA091EE
:1029E6002C0EB0912D0E139710F00C940015E3E009
:1029F600F0E0E0932C0EF0932D0EA32F0E941E13F1
:102A0600E093CC00E22FE13011F00C941015E09128
:102A1600CA00E2600E94A7AE22C0E23011F00C9418
:102A26001A15E091CA00E4600E94A7AE18C0E33010
:102A360011F00C942415E091CA00E6600E94A7AE3E
:102A46000EC0E43011F00C943215E091CA00E66035
:102A5600E093CA00E091C900E460E093C900E12F69
:102A6600E13011F00C943C15E091CA00E860E09367
:102A7600CA00E02FE13011F00C944715E091CA002E
:102A8600E062E093CA000FC0E23011F00C945115D9
:102A9600E091CA00E063E093CA0005C0E091CA0075
:102AA600EF7CE093CA00E42FE13011F00C9461153D
:102AB600E091C900EF77E093C90009C0E23011F058
:102AC6000C946A15E091C900E068E093C90089E1B9
:102AD6008A95F1F70E940CC229960895E0E0E093EA
:102AE600C90008950A930A2FE091C800E07211F018
:102AF6000C947E15F9CF0093CE00099108950E949B
:102B0600AFAD0E94AFAE0E171F0710F00C949215D2
:102B1600A5ECBDE00E9445AE0F5F1F4FF2CFE0E08F
:102B2600E093290EE0932A0EE0932B0EE093C91151
:102B3600E1E0E0932E0E0991199108950E944AAEA4
:102B46000A93A0912E0EA13010F40C94B015E1E07A
:102B5600E093C911E2E0E0932E0EE091C900E47023
:102B660011F40C94DD150E94AFAE32970E9484AE2C
:102B7600AE17BF0710F00C94DA15E091C900E270A9
:102B860011F40C94CE150E94B4AE3197EB53F24F6C
:102B9600A1E0A08307C00E94B4AE3197EB53F24F79
:102BA600A0E0A0830E94B4AE0E94B7AE02C000911E
:102BB600CE0010C00E94AFAE0E9484AEAE17BF0713
:102BC60010F00C94EB150E94B4AE0E94B7AE02C092
:102BD6000091CE00E091C800EC710E2F013010F488
:102BE6000C94FC15A0912B0EA03011F00C94FC1542
:102BF60001C002C000932B0E09910E946BAE18957E
:102C0600E0912B0EE03011F00C940C160E94BFAE32
:102C16000895E0912B0EE07111F40C941516EFEF68
:102C2600FFEF0895E0912B0EE87011F40C941E1638
:102C3600EEEFFFEF0895E0912B0EE47011F40C9483
:102C46002716EDEFFFEF089508950E9404C2AD0127
:102C56000E9484AE4A175B0710F00C943416FA01F2
:102C660002C00E94BFAE9F0100E010E002171307EA
:102C760010F00C9447160E9477AEA5ECBDE00E94BA
:102C86007EAE0F5F1F4FF2CF0E9484AEA436E0E007
:102C9600BE0710F00C9453160E94BFAE0E9489AE78
:102CA6000E940BC228960895A0912E0EA53010F40E
:102CB6000C946216E0E0E0932E0EE1E00895E0E069
:102CC600089508950E94C4AE00E010E02F81388573
:102CD60040E050E00E945328E03011F00C947A1640
:102CE6004436E0E05E0710F00C947A1601C007C087
:102CF600A1E0B0E00E9471C54F5F5F4FEBCFF801D6
:102D06000F5F1F4FA985BA85AE0FBF1FEC91EE83EB
:102D1600AE810E9475150217130710F00C949416D5
:102D2600D7CF0E940BC22B9608950E949CC30E9487
:102D360005C200E010E020E030E00E945328E030B9
:102D460011F00C94AD162436E0E03E0710F00C941A
:102D5600AD1601C007C0A1E0B0E00E9471C52F5FAB
:102D66003F4FEBCFF8010F5F1F4F0E949FAD0E94B0
:102D7600CAAE6BBF4691413010F40C94C516A42F11
:102D86000E947515003DE7E01E0710F00C94D01662
:102D9600413010F40C94D01601C001C0CCCF789409
:102DA6000E940CC2299608950E9437AEE093D00087
:102DB600E0E0E093D100E093D200E093D500EAE2B0
:102DC600F3E0E0935C11F0935D11A0915C11B0917A
:102DD6005D11139710F00C94F616E3E0F0E0E09323
:102DE6005C11F0935D11A32F0E941E13E093D40093
:102DF600E22FE13011F00C940617E091D200E26068
:102E0600E093D20022C0E23011F00C941017E0914A
:102E1600D200E460E093D20018C0E33011F00C94C5
:102E26001A17E091D200E660E093D2000EC0E430BB
:102E360011F00C942817E091D200E660E093D200DE
:102E4600E091D100E460E093D100E12FE13011F090
:102E56000C943217E091D200E860E093D200E02FA4
:102E6600E13011F00C943D17E091D200E062E0935E
:102E7600D20009C0E23011F00C944617E091D2005E
:102E8600E063E093D200E42FE13011F00C94511787
:102E9600E091D100E861E093D10009C0E23011F081
:102EA6000C945A17E091D100E869E093D1000E9492
:102EB6000CC229960895E0E0E093D10008950A93A4
:102EC6000A2FE091D000E07211F00C946B17F9CF45
:102ED6000093D600099108950E94AFADE0915C1170
:102EE600F0915D110E171F0710F00C948117AFE2D9
:102EF600BEE00E9445AE0F5F1F4FF0CFE0E0E093CB
:102F06005911E0935A11E0935B11E1E0E0935E11F1
:102F16000991199108950E944AAE0A93A0915E11F3
:102F2600A13010F40C949A17E2E0E0935E11E09160
:102F36005C11F0915D110E94CFAEAE17BF0710F085
:102F46000C94B117A9E5B1E10E9450AD3197E15D4E
:102F5600F14FDF01E091D600EC9302C00091D6005C
:102F6600E091D000EC710E2FE0915B11E03011F092
:102F76000C94BF1700935B1109910E946BAE1895D4
:102F86000E94D4AE08950E9404C2AD010E94CFAE45
:102F96004A175B0710F00C94D217FA0102C00E9480
:102FA600D4AE9F0100E010E00217130710F00C9456
:102FB600E5170E9477AEAFE2BEE00E947EAE0F5FDD
:102FC6001F4FF2CF0E94CFAEAA32E3E0BE0710F049
:102FD6000C94F1170E94D4AE0E9489AE0E940BC2D7
:102FE60028960895A0915E11A43010F40C94001850
:102FF600E0E0E0935E11E1E00895E0E008950895D1
:103006000E9490AE0E9497AE10F40C940D18A22F59
:103016000E946217003DE7E01E0710F00C94181896
:10302600213010F40C94181801C001C0EBCF0E9497
:103036000CC2259608950E9438AD00E010E02D815F
:103046003E81F8010F5F1F4F0E94D9AE4C91A42F0D
:103056000E9462170217130710F00C943318F1CF71
:103066000E940CC2299608950E9437AEE093300163
:10307600E0E0E0933101E0933201E0933501E4E6CC
:10308600F0E0E093C611F093C711A091C611B0917C
:10309600C711139710F00C945618E3E0F0E0E09394
:1030A600C611F093C711A32F0E941E13E09334019B
:1030B600E22FE13011F00C946618E0913201E260E3
:1030C600E093320122C0E23011F00C947018E091C6
:1030D6003201E460E093320118C0E33011F00C9441
:1030E6007A18E0913201E660E09332010EC0E430D6
:1030F60011F00C948818E0913201E660E0933201F9
:10310600E0913101E460E0933101E12FE13011F00B
:103116000C949218E0913201E860E0933201E02FBE
:10312600E13011F00C949D18E0913201E062E093D9
:10313600320109C0E23011F00C94A618E091320178
:10314600E063E0933201E42FE13011F00C94B11802
:10315600E0913101E861E093310109C0E23011F0FC
:103166000C94BA18E0913101E869E093310181E3EA
:103176008A95F1F70E940CC229960895E0E0E09343
:10318600310108950E94AFAD0E94DEAE0E171F07F3
:1031960010F00C94D518AFE5B1E10E9445AE0F5F73
:1031A6001F4FF2CFE0E0E093C311E093C411E09328
:1031B600C511E1E0E093C8110991199108950A93A8
:1031C6000A2F003011F40C94EE18E0913101E16001
:1031D600E093310105C0E0913101EE7FE0933101CA
:1031E600099108950A930A2FE0913001E07211F0D7
:1031F6000C94FE18F9CF00933601099108950E94A8
:1032060004AD0E9406C2A091C811A13010F40C941E
:103216000F19E2E0E093C811E0913101E47011F476
:103226000C944C190E94DEAE32970E94E3AE10F069
:103236000C943719E0913101E27011F40C942B19BA
:103246000E94EAAE3197E15AFE4EA1E0A08307C084
:103256000E94EAAE3197E15AFE4EA0E0A0830E949A
:10326600EAAE0E94EDAE02C000913601E091C311B4
:10327600E2501E2FF0E0E15AFE4E0E9463AEE15A84
:10328600FE4EE081F0E02E2B3F2BD9010E94FA3949
:103296001BC00E94DEAE0E94E3AE10F00C945919DA
:1032A6000E94F5AE10F00C94591901C005C00E9499
:1032B600EAAE0E94EDAE02C0009136010E94F5AE64
:1032C60010F40C94671900E0E0913001EC710E2FB8
:1032D600E091C511E03011F00C9473190093C511FB
:1032E6000E940DC224960E9416AD1895BA93AA9311
:1032F6002997E0E0ED83EE830E9404C20B8D1C8DBE
:1033060000FF02C0E1E0EC870436E0E01E0710F0A3
:103316000C949819E1E0EB87E4E6F0E0E01BF10B92
:10332600AF01F695E7959F0108C0E0E0EB870456EC
:103336001040F801F695E7959F012436E0E03E0738
:1033460010F40C94BF19E3E0EA87D901E4E6F0E053
:103356000E9404C3AF014987D9010E94FAAEED87E6
:10336600FE87AD85BE850E94FFAEAD85BE850E94F7
:1033760006AFAF014F831BC02A30E0E03E0710F4D2
:103386000C94D419E2E0EA87E0E0E987D9010E94CB
:10339600FFAED9010E9406AFED87FE87ED85EF836C
:1033A60006C0E1E0EA87E0E0E987E8872F83E98560
:1033B600E05DE9870E940BAFA985A03311F00C945C
:1033C600EC19E0E2E987A885A03311F00C94EC191A
:1033D600E887EC85E03011F40C94F419E5E3EE830C
:1033E60002C0E0E3EE83EA85A98DBA8DEC93E98508
:1033F600AF89B88DEC93E885AD89BE89EC93EF81F2
:10340600AB89BC89EC93EB85A989BA89EC93EE81EB
:10341600AF85B889EC930E940BC26D960895BA9356
:10342600AA9360970E9404C2EB8DE987E98DE8872D
:10343600EA8DEF83E88DEE83EC8DFD8DFA93EA93AA
:10344600EDB7FEB7FA93EA932F93EDB7FEB7FA936B
:10345600EA933F93EDB7FEB7FA93EA934F93EDB72E
:10346600FEB7FA93EA935F93FE017596FA93EA9391
:10347600DE0156960E9479195F914F913F912F91E7
:1034860000E00A3010F00C944E1A0E9412AFE0E0F1
:10349600EC930F5FF6CF00E0E985E03011F40C9471
:1034A6005A1AEB85E03011F40C945A1A01C006C082
:1034B6000E9419AFAE0FBF1FEDE2EC93E885E03036
:1034C60011F40C94761A0E9419AFEA0FFB1F308391
:1034D6000E9419AFEA0FFB1F40830E9419AFEA0F43
:1034E600FB1F508317C0233010F40C947F1A0E94E0
:1034F60019AFEA0FFB1F3083223010F40C94881AA0
:103506000E9419AFEA0FFB1F40830E9419AFEA0F12
:10351600FB1F5083EF81E03011F40C94A61A0E9431
:1035260019AF0E941FAFEA85E03011F40C94A21A7D
:103536000E9419AFAE0FBF1FE5E3EC9304C00E94D3
:1035460019AF0E9424AFEE81E03011F40C94B71A43
:103556000E9419AFAE0FBF1FE8EFEC930E9419AFA0
:10356600AE0FBF1FE3E4EC9300E00E9412AF1C9184
:10357600E02FAE89BF89F0E0EA0FFB1F10830F5FD3
:103586000A3010F00C94CC1A113010F40C94CC1AAA
:1035960001C001C0EACF0E940BC26E9608950E9438
:1035A6009FAE0217130714F00C94F31A0E9429AF6A
:1035B600F801E40FF51FE081EA1711F40C94EC1AF8
:1035C600F801E40FF51FA081AF3311F40C94EC1A47
:1035D60001C003C00E9430AF08950F5F1F4FE1CFB7
:1035E600E1E00E940BC22A9608950E9435AF003092
:1035F600E0EF1E0710F00C94101BF801E20FF31F0A
:10360600E081E03011F00C940D1BF8010E940DC210
:10361600249608950F5F1F4FEACFE0E0F0E00E9486
:103626000DC224960895BA93AA93EF97EF97EF9752
:103636002F970E9404C2DE01AC52BF4F0D90BC9181
:10364600A02D0E94F81A9F01DE01AE52BF4F0D90C9
:10365600BC91A02D0E94F81AAF012436E0E03E0787
:1036660014F00C94461BFE01EC52FF4F0190F081C2
:10367600E02DFA93EA93FE01E459FF4FFA93EA9399
:10368600D9010E94E71B4436E0E05E0714F00C9473
:10369600571BFE01EE52FF4F0190F081E02D0E9474
:1036A6003BAFDA010E94E71B00E010E0E0E00E9479
:1036B60042AFDE01A659BF4FA00FB11FAC91EE81FC
:1036C600EA1711F00C94A31BE1E00E9442AFD80167
:1036D600A40FB51F2A173B0714F00C94751B0E9404
:1036E60047AF0895E0E0DE01A053BF4FED93EC93A2
:1036F6000E944FAFA417B50714F00C94A31BF80152
:103706000E944FAFEA0FFB1FDE01A659BF4FAE0F57
:10371600BF1F1C90FE01E053FF4F0190F081E02D8A
:103726000E9456AFEC91E11511F40C949D1BE0E05C
:103736000E9442AFDE01A053BF4F0E9450ADD8CFCA
:103746000E945BAFE03011F40C94B81BE02F0E948E
:1037560060AFEA0FDE01A253BF4FEC930E940BC28B
:10376600EF96EF96EF9669960895F80131968F01D8
:10377600E217F30714F00C94C11B98CF0E9447AFD1
:1037860008950E949CC30E94AFAD0030E0EF1E0773
:1037960010F00C94E11BF8010E9465AF0E94CAAEBE
:1037A6006BBFE691E03011F00C94DE1BF801198135
:1037B6000881269608950F5F1F4FE7CFE0E0F0E0FF
:1037C60019810881269608950E949FAE022E032A2B
:1037D60011F00C94FC1B0E9429AFA13010F40C943C
:1037E600F91B0E946AAF0F5F1F4FF5CF0E9477AF9C
:1037F6000EC000E010E00217130710F00C94081C2E
:103806000E946AAF0F5F1F4FF6CF0E9477AF0E94EC
:103816000BC22A9608950E949FAE022E032A11F02B
:103826000C94231C0E947DAFE13010F40C94201CF4
:103836000E9485AF0E948AAFF5CF0E9477AF10C075
:1038460000E010E00217130710F00C94311C0E94E0
:1038560085AFD001EC930F5F1F4FF4CF0E9477AF77
:103866000E940BC22A9608950E949FAE022E032A3A
:1038760011F00C944C1C0E9429AFA13010F40C944A
:10388600491C0E948FAF0F5F1F4FF5CF0E949DAF5F
:103896000EC000E010E00217130710F00C94581C3D
:1038A6000E948FAF0F5F1F4FF6CF0E949DAF0E9401
:1038B6000BC22A9608950E9444AD488559852C85E9
:1038C6003D8500E010E00217130710F00C947D1CF4
:1038D600FA01E00FF11FEE83FF83AA85BB85EA0F8D
:1038E600FB1F0F01F801AE85BF850E94A4AF0F5FD5
:1038F6001F4FE9CF0E940BC2609608950E9444AD07
:103906000E851F852A853B8548855985E0E0EE832F
:10391600EF83AE81BF81A417B50710F00C94A71CE6
:10392600EE81FF81E20FF31FAC85BD85EA0FFB1F19
:103936000F01EE81FF81E00FF11FA889B9890E946E
:10394600A4AF0E940EAEE5CF0E940BC26296089508
:103956000E949FAE00240216030610F00C94B51CBC
:10396600215030400E94AAAF6BBFA691A13010F43F
:103976000C94C41C0034E0E01E0710F00C94C41C28
:1039860001C00BC0F901E00FF11FE40FF51F0F0195
:103996000E94AAAF0E94B0AFE5CF0E940BC22C9640
:1039A60008950E9405C29D014D8100E010E000E0EF
:1039B60010E00217130710F00C94E81CF8010E949F
:1039C600B3AF40830F5F1F4FF4CF0E940CC22896FF
:1039D60008950E9435AF0E94B8AF6BBFA691A13083
:1039E60010F40C94FB1C0E94BEAF0E94B0AFF3CF44
:1039F600F801E20FF31FA0E0A0830E940DC22896F3
:103A060008950E9435AF0E94B8AF6BBFA691A13052
:103A160010F40C94131D0E94BEAF0E94B0AFF3CFFA
:103A26000E940DC228960895BA93AA9327970E94DA
:103A360005C230E040E000E0073010F00C94291D8C
:103A4600AC85BD850E94C3AF0F5FF6CF1E852F855F
:103A560000E0012E022A11F00C94351D0E94D0AF11
:103A66000E9424AF222312F00C94471D0E94D0AF6F
:103A7600AE0FBF1FEDE2EC93E12FF22FAFEFBFEFDA
:103A86000E94ECC21E2F2F2F00240116020614F0EE
:103A96000C945A1D0E94D6AFEAE0F0E00E944BC398
:103AA6000E94E2AF0E9417C31E2F2F2FEDCF0024D6
:103AB6000316040614F00C94651D0E94D0AF0E94F4
:103AC600E9AFF5CF0E940CC260960895BA93AA9307
:103AD60026970E9405C230E040E000E0063010F074
:103AE6000C947B1DAB85BC850E94C3AF0F5FF6CFE0
:103AF6001D852E8500E0012E022A11F00C948A1DE8
:103B0600E02F0F5FAB85BC85F0E00E9424AF002458
:103B16000116020610F00C949B1D0E94D6AF0E945F
:103B260006AF0E94E2AF0E9404C31E2F2F2FEFCFD5
:103B360000240316040614F00C94A91DE02F0F5F51
:103B4600AB85BC85F0E00E94E9AFF2CF0E940CC2C3
:103B56002F9608950E94FAAF0C3010F00C94B71D02
:103B66000E9403B00F5FF8CF0E9412B011F00C94C0
:103B7600C01D0E941EB0A0E3A083A885AA2312F050
:103B86000C94D31D0E941EB0ADE2A0830E94A7AD87
:103B9600AFEFBFEF8FEF9FEF0E94F1C20E9495AD8E
:103BA6000E949FAD0E94E5C314F00C94EC1D0E9488
:103BB60024B0FF93EF930E942DB00E945DC3AF9196
:103BC600BF91EC930E942DB00E9440C30E9495AD18
:103BD600E7CF00240116020614F00C94F71D0E948C
:103BE6001EB00E9434B0F5CF0E940CC269960895AB
:103BF6000E94FAAF0C3010F00C94051E0E9403B020
:103C06000F5FF8CF0E9412B011F00C940E1E0E94A6
:103C16001EB0A0E3A0830E949FAD0E94E5C310F0F2
:103C26000C94251E0E9424B0FF93EF930E942DB0A2
:103C36000E9459C3AF91BF91EC930E942DB00E9490
:103C4600A4ADE9CF00240116020614F00C94301E30
:103C56000E941EB00E9434B0F5CF0E940CC2699635
:103C66000895AA93A5970E9404C2E9A9FAA96BA987
:103C76007CA90E9443B0ECA5E88B1DA51B3010F46F
:103C86000C94461E1AE0E889E03011F00C944C1EA4
:103C960010E0A889A03210F40C94561EA03810F03B
:103CA6000C94561E02C0EEE2E88B0EA50D3010F401
:103CB6000C945E1E0CE0E0E0EE87EF87AE85BF85D4
:103CC6001D9714F00C94741E0E9448B00E9424AFF5
:103CD600EE85FF85DE015E960E9424AF0E944DB000
:103CE600EDCF0E9453B00E945AB00E94F81AEA879C
:103CF600FB87AA85BB851B9714F40C94861EEAE005
:103D0600F0E0EA87FB87EA85FB85309711F00C9493
:103D1600921EE0E3E98BE1E0F0E0EA87FB8750E002
:103D2600113010F40C94201FEA85FB85A12FB0E01A
:103D3600AE17BF0714F40C94ED1EE0E3EE8FE8898E
:103D4600EF8FE2E0F0E0EE87FF875E5FAA85E12F66
:103D5600EA1B2E2F520F213010F40C94BB1E0E942A
:103D66004DB03197DE015E960E9424AF2150F3CF0D
:103D7600E0E0EC87ED87AE85BF851C9714F00C94C8
:103D8600D51E0E944DB031970E9461B00F01EC859F
:103D9600FD853196EC87FD873197DE0151960E94AD
:103DA600A4AFE9CFE0E0EE87EF87AE85BF851C972D
:103DB60014F00C94EC1E0E9448B0EA0FFB1F0F0192
:103DC600EE85FF85DE015E960E94A4AF0E944DB08F
:103DD600ECCF2BC0EA85E11B2E2FEBE0F0E0EE875F
:103DE600FF87E22FAE85BF85F0E0EA17FB0714F0E8
:103DF6000C940F1F0E9448B0EA0FFB1F0F01EE85BF
:103E0600FF853197DE0151960E94A4AFEE85FF85AE
:103E16003197EE87FF87E5CFE22FF0E0DE0151967E
:103E2600EA0FFB1FA889A0835F5FE52FAA85BB85E4
:103E3600F0E0EA0FFB1FEA87FB87EBA5E03011F401
:103E46000C94271F40E301C040E2EA85FB85A02FC2
:103E5600B0E0EA17FB0714F00C94671FAA85E02F61
:103E6600EA1B3E2FEBE0F0E0EE87FF870E9448B0AA
:103E7600EA0FFB1FBF010E9466B00E94A1C3EA1BA6
:103E8600FB0BDE0151960E946BB0EE85FF853197E4
:103E9600EE87FF870E9466B0AE17BF0714F40C9436
:103EA600551FE4CFE0E0EE87EF870E9466B0AE17BD
:103EB600BF0714F00C94671F0E9448B0EA0FFB1F5F
:103EC60040830E944DB0F1CFE0E0EE87EF87AE85EC
:103ED600BF851C9714F00C947E1FEE85FF85AFA559
:103EE600B8A9EA0FFB1F0F010E9448B00E94A4AFB9
:103EF6000E944DB0ECCF0E940BC2E59608950E9439
:103F0600C4AE3D854C855B85383110F40C948C1F0E
:103F160030E04C3310F40C94911F40E05C3310F405
:103F26000C94961F50E0E985EE8310E020E01C30EB
:103F3600E0E02E0714F00C94A91FE12FF22F0E9447
:103F4600D9AEE0E0EC931F5F2F4FF1CF0A8500302A
:103F560011F40C94D61F303011F40C94B71F3C307A
:103F660011F40C94B71F08C0AF81B885E1E3EC9358
:103F76001196E2E3EC9316C03C3010F00C94C61F89
:103F86000E9471B00FC0A32FAC500E9483B0AF81C6
:103F9600B885EC93A32FAC500E9488B0AF81B8854A
:103FA6001196EC9302C00E9471B0AF81B88512964B
:103FB600EAE3EC93A42F0E9483B0AF81B8851396F1
:103FC600EC93A42F0E9488B0AF81B8851496EC9329
:103FD60015E020E0EE81E03011F40C9408200E94F8
:103FE6008DB00E94D9AEEAE3EC930E948DB00E9498
:103FF60092B00E9483B0DB01EC930E948DB00E94C8
:1040060092B00E9488B0DB01EC93003011F40C945E
:1040160029200E948DB00E94D9AEE0E2EC933C309C
:1040260010F00C941D200E948DB00E94D9AEE1E4E0
:10403600EC9306C00E948DB00E94D9AEE0E5EC93E9
:104046000E948DB00E94D9AEEDE4EC93E1E00E94AF
:104056000BC22E960895BA93AA9326970E9404C27D
:10406600E989EF70E05DE987E989E07FE295EF7025
:10407600E05DEA870B891A8928891D3010F00C94B7
:104086004920103011F40C94492001C011E000328F
:1040960010F00C945320003011F40C94532001C0FE
:1040A60001E0233310F00C945D202B3010F40C94B7
:1040B6005D2001C021E0EE85E03011F00C94662011
:1040C600EEE2EE830FC0AE85A13011F00C946E20A7
:1040D600EFE2EE8307C0AE85A03210F40C94752093
:1040E600EE85EE83A02FEAE00E94F6C23E2FA02FB7
:1040F600EAE00E9445C34E2FA12FEAE00E94F6C2D5
:104106005E2FA12FEAE00E9445C3EB870E9499B07B
:10411600E8870E949EB0EF83305D405D505DEB8581
:10412600E05DEB870E940BAFEF85E03011F00C9459
:10413600A7200E94A3B0EC85FD855383EB850E94E2
:10414600AFB00E94B4B04DC0E13011F00C94B42071
:104156000E94CEB0EC85FD85338344830E94B4B0C3
:1041660040C0E23011F00C94C5200E94DCB0EC8512
:10417600FD855583EB850E94F1B03087EC85FD8582
:1041860041872FC0E33011F00C94D2200E94A3B0D7
:104196000E94FDB00E9404B10E940BB122C0E4301F
:1041A60011F00C94E1200E94CEB00E94FDB00E9456
:1041B60004B13087EC85FD85418713C0E53011F0E9
:1041C6000C94F4200E94DCB0EC85FD853583468393
:1041D600EE81AC85BD851796EC93EC85FD850E9436
:1041E6000BB1AC85BD851A96E0E0EC930E940BC23C
:1041F600649608950E9444ADA885B9850E94F81A70
:10420600EE83FF83AE81BF81A030E1E0BE0710F4EC
:104216000C941121EFEFF0E0EE83FF830E9412B1C0
:104226000E94C41B5E2F00E010E00E9417B110F040
:104236000C9464210E9429AF0E941CB16BBFE691C9
:10424600EA1711F00C946121E52FF0E0E00FF11F61
:10425600DF01EE81FF81EA17FB0710F00C9438218D
:10426600E0E00E940BC22E96089520E030E040E088
:10427600451710F00C945521E42FF0E0E00FF11FE4
:10428600A885B985AE0FBF1F0C90E42F0E9412B10E
:104296000E9421B1E01511F40C94532121E030E085
:1042A6004F5FE6CF022E032A11F00C946121E02F16
:1042B600E40F5E2F0E940BC22E9608950F5F1F4FCC
:1042C600B4CFE0E00E940BC22E9608950E9407C26A
:1042D6002A2F022F02950F700F70AAE00A9F002D59
:1042E600E22FEF701E2F010F0E9433AD08950E943A
:1042F60006C23A2F032FA02FEAE00E94F6C21E2F15
:104306001295107FA02FEAE00E9445C32E2F120FB0
:10431600E12F0E940DC2249608950A930A2F0033B6
:1043260010F40C949B210A3310F00C949B2101C0CD
:1043360003C0E1E009910895E0E00991089509912B
:1043460008950A930A2F0E949021E03011F40C94EC
:10435600B021E02FE05309910895E0E00991089516
:10436600099108950E9404C24A2F5E81F52FE0E06C
:104376008F010070E42FF0E0F0709F01022B132BE9
:10438600F8010E940BC22796089528970E9406C23C
:104396000A2F1C852D853E85E32F0E9429B10E9498
:1043A60031B10E9436B10E943BB1E22F0E9429B181
:1043B6000E943FB1E12F0E9429B10E943FB1E02F38
:1043C6000E9429B1EC83FD836E837F830E9436B100
:1043D6000E942AC20E9431B1E885F9856A857B85EB
:1043E6000E940DC22F9608950E9406C22A2F3C8174
:1043F600E22FE0531E2FE32FE0530E2FAAE00A9F71
:10440600002D010FE02F0E940DC225960895BA9344
:10441600AA932B970E9404C2A989BA890E94F81A06
:104426001E2FE989FA890E944CB1A6E0B0E00E94ED
:10443600E71B10E0E0E0E88B0E9453B1A03310F4D4
:104446000C942C220E9453B1AA3310F00C942C2207
:1044560002C0E1E0E88BE889E03011F00C943422E8
:104466001F5F153010F00C943E22A889A03011F081
:104476000C943E2201C001C0DFCF163010F00C9420
:104486004922103011F40C94492204C00E945CADFC
:1044960063960895153011F00C946522E989FA891E
:1044A600E481E88BA989BA8913965C91A989BA89AE
:1044B60012964C91A989BA8911963C91A989BA8913
:1044C6002C9147C0143011F00C947A22E989FA89AC
:1044D600E381E88BA989BA8912965C91A989BA8980
:1044E60011964C91A989BA893C9120E332C01330C8
:1044F60011F00C948C22E989FA89E281E88BA9896A
:10450600BA8911965C91A989BA894C9130E320E366
:1045160020C0123011F00C949B22E989FA89E181BE
:10452600E88BA989BA895C9140E330E320E311C0A6
:10453600113011F00C94A822A989BA89EC91E88B64
:1045460050E340E330E320E304C00E945CAD639691
:104556000895E22FE0530E2F0A3010F40C94B42283
:1045660000E00E945AB1A0E1B7E20E945FB1EE837B
:10457600FF83E32FE0530E2F0A3010F40C94C4226D
:1045860000E00E945AB1A8EEB3E00E945FB10E941B
:10459600B3AFEE83FF83E42FE0530E2F0A3010F4FF
:1045A6000C94D62200E00E9464B1E4E60E946BB14E
:1045B600EE83FF83E52FE0530E2F0A3010F40C94A0
:1045C600E52200E00E9464B1EAE00E946BB1EE834E
:1045D600FF83E889E0530E2F0A3010F40C94F4227E
:1045E60000E00E945AB10E94B3AFEE83FF830E949F
:1045F6000BC263960895BA93AA932A970E9404C29F
:104606005A890B891C8930E0E52FE1502E2F28307E
:1046160010F40C940F2327E0422FE22F2150F0E0F4
:104626000E9456AFE02FEF70EC93F8010E9490C203
:104636008F013F5F341710F00C942223EECF0E94B7
:1046460070B1EA0FFB1F00834F5FE42FF0E00E947A
:1046560056AFE0E0EC9330E00E9475B1AC91AA3021
:1046660010F40C943B230E9475B1EC91E95FEC9336
:10467600E32FA889B9890E9478B10E9475B1EC919F
:10468600E05DD001EC933F5F341710F00C944C239F
:10469600E3CFA889B989EE27A30FBE1FEC930E942A
:1046A6000BC2659608950E947DB10217130710F09C
:1046B6000C945F23F80101C0F9010E940DC22696F1
:1046C60008950E9483B111F00C947923E02FE370D2
:1046D60011F40C947323ECE1198108812396089553
:1046E600EDE1198108812396089527C0113011F450
:1046F6000C949623133011F40C949623153011F470
:104706000C949623173011F40C949623183011F458
:104716000C9496231A3011F40C9496231C3011F441
:104726000C94962305C0EFE119810881239608951C
:10473600EEE119810881239608951981088123964F
:104746000895AA9321970E9489B1498528853F81BA
:10475600203011F40C94C0232D3010F00C94C0239B
:10476600303011F40C94C023303210F00C94C02376
:10477600443610F00C94C02304C00E945CAD2A9607
:10478600089551E0223010F40C94D4235A93A42FA8
:104796000E946423EE83F0E00E0F1F1F21505F5F1F
:1047A600F1CFE32F0E948EB10E940BC22A96089584
:1047B6000A930A2FE02FE37011F00C94E523E1E051
:1047C60009910895E0E009910895AA931A930A932E
:1047D6000A81102FE02FEC5F1E1710F00C94FF23B8
:1047E600E12FE37011F00C94FD23E12F198108816C
:1047F600239608951F5FEECF1981088123960895A9
:10480600AA931A930A930A81043010F00C94102488
:10481600E0E01981088123960895E02FE37011F0F6
:104826000C941A24E02F19810881239608950450C8
:10483600102FE02FEC5F1E1710F00C942E24E12FA2
:10484600E37011F00C942C24E12F19810881239632
:1048560008951F5FEECF1981088123960895AA93C4
:104866001A930A931B81EB81E1500E2FA8E10A9F50
:10487600002DEA810E0FE02F1981088124960895F4
:104886000E94B4AD4A93A32F0E9432240E2F112703
:104896000E9493B10E940CC2279608950E9406C2F8
:1048A6002A2F3C81E32FE1500E2F11270E949BB146
:1048B6000E940DC2259608950E94B4AD4A93A32F77
:1048C6000E9451248F010E9493B10E940CC2279628
:1048D60008950E9404C22A2F3E814F8158855A931B
:1048E6004A93A32F0E94A4238F01015010400E94D7
:1048F6009BB10E940BC22996089524970E9405C277
:104906000A2F19852A853B854C854A933A932A9323
:10491600A12F0E946C240E94A3B131976040704081
:104926000E94ACAD0E94A6B10E9495AD0E94ADB1A9
:104936000E94ACAD0E940CC22D960895AA930E94C7
:1049460006C22D813E810D811E81EC81E03011F47D
:104956000C94B424012F1127E02F0E940DC2279634
:104966000895E02F0E940DC2279608950E940DC259
:1049760027960895AA9324970E94A7AD0E94B6B1E0
:10498600EC81E03011F00C94CB24E881299608954F
:104996000E94B9B1A13011F00C94D424E881299673
:1049A60008950E94B9B1A23011F00C94DD24E8817B
:1049B600299608950E948DC3E8E00E9470C20E9465
:1049C600B6B1E881299608950E9405C24A2F242F80
:1049D600332700240216030614F00C94F424215005
:1049E600304000E010E00217130714F00C94132572
:1049F600F801AD81BE81AE0FBF1F0C903196AD811F
:104A0600BE81AE0FBF1FEC91E01511F40C9410257A
:104A1600E0E00E940CC2279608950F5F1F4FE3CF78
:104A2600E1E00E940CC2279608950E9407C21A2F41
:104A36002B81A22F0E949021E03011F00C942825A2
:104A4600EFEF0E940EC224960895A12F0E94902196
:104A5600E03011F40C943B25A22F0E94A4210E2FC6
:104A6600AAE00A9F002DA12F0E94A4210E0F04C0C8
:104A7600A22F0E94A4210E2FE02F0E940EC2249680
:104A86000895AA930E9405C23D81AE81BF810E940E
:104A9600F81A2E2FE31B1E2F112311F00C94582504
:104AA600E1E00E940CC22896089500E0011710F07C
:104AB6000C947325E32FE00F4E2F421710F00C9441
:104AC6007125E02FAE81BF810E9478B1AE81BF8192
:104AD600EE27A40FBE1FEC91D001EC930F5FE6CF3B
:104AE600012F021710F00C948125AE81BF81EE27AD
:104AF600A00FBE1FE0E2EC930F5FF3CFE0E00E9451
:104B06000CC22896089524970E94C2B12AE010E0AC
:104B16001A3010F00C949D25A32FB42FEE27A10F69
:104B2600BE1F0E94C7B111F00C949B25212F02C015
:104B36001F5FEECF213010F40C94A6252B3010F019
:104B46000C94A62504C00E94CCB12996089510E0C5
:104B5600E0E0ED83EE83EF83E8870E94A7ADAAE04D
:104B6600B0E080E090E00E94C6C20E9495ADE12FC1
:104B76001F5FF0E0E30FF41FA0810E94A4210E2F17
:104B86000E94ADB10E9495AD121710F00C94CC2581
:104B9600E4CF0E94A7AD0E940CC2299608950E94F8
:104BA60006C28D012C813D811A930A930E94D3B1CE
:104BB600E32FE13011F00C94F625213011F00C941E
:104BC600EB25E6EFF0E060E070E00E94D9B10AC0A4
:104BD600223011F00C94F525EDEFF0E060E070E086
:104BE6000E94D9B19BC0E23011F00C9410262130FE
:104BF60011F00C940526E4E0F1E060E070E00E941C
:104C0600D9B10AC0223011F00C940F26EDE0F1E084
:104C160060E070E00E94D9B181C0E33011F00C94DD
:104C26002A26213011F00C941F26E5E1F1E060E020
:104C360070E00E94D9B10AC0223011F00C942926E6
:104C4600EEE1F1E060E070E00E94D9B167C0E430C7
:104C560011F00C944426213011F00C943926E8E228
:104C6600F1E060E070E00E94D9B10AC0223011F094
:104C76000C944326E3E3F1E060E070E00E94D9B1D2
:104C86004DC0E53011F00C945E26213011F00C94E5
:104C96005326ECE3F1E060E070E00E94D9B10AC06F
:104CA600223011F00C945D26E4E4F1E060E070E05F
:104CB6000E94D9B133C0E63011F00C947826213029
:104CC60011F00C946D26EBE4F1E060E070E00E94D8
:104CD600D9B10AC0223011F00C947726E3E5F1E051
:104CE60060E070E00E94D9B119C0E73011F00C9471
:104CF6009126213011F00C948726ECE5F1E060E076
:104D060070E00E94D9B10AC0223011F00C949126AD
:104D1600E4E6F1E060E070E00E94D9B10E940DC2C5
:104D2600269608950E94DEB140E050E841E050E04A
:104D360020E030E02031E0E03E0710F00C94B6268B
:104D4600F901AE81BF810E94E1B10E9484C30E9435
:104D5600D9C310F00C94B126042B152B440F551F04
:104D66002F5F3F4FE7CFF8010E940BC228960895A8
:104D7600BA93AA93EF9763970E9405C240E0403129
:104D860010F00C94D72620E0253010F00C94D52690
:104D96000E94E6B1AE0FBF1FEE27A20FBE1FEC9317
:104DA6002F5FF2CF4F5FEBCF10E00E94ECB1EE2702
:104DB600A10FBE1F3C911F5F103510F00C94E82622
:104DC6003B3511F40C94E82601C001C0EECF40E05B
:104DD60020E0012F003510F00C9414270E94ECB14E
:104DE600EE27A00FBE1F3C913C3211F00C94FE261C
:104DF6004F5F20E014C0403110F00C940727253097
:104E060010F00C94072701C00AC00E94E6B1AE0F4D
:104E1600BF1FE22F2F5FF0E0EA0FFB1F30830F5F0B
:104E2600D9CF40E02FE00E94E6B1AE0FBF1F0E942F
:104E36000A22ED83FE83E22FDE01A95ABF4F0D90B1
:104E4600BC91A02D0E94F3B1AD81BE81A083B18338
:104E56004F5F2150403110F00C943227E4CF0E946E
:104E66000CC2EF966C960895759A749A769A779A0C
:104E7600E0910401E068E09304015D9A559A5D981B
:104E86005F9A579A5F980895E0E00895E0E0E1B9E7
:104E9600E2B9E4B9E5B9E7B9E8B9EAB9EBB9EDB908
:104EA600EEB9E0BBE1BBE3BBE4BBE0930101E093F9
:104EB6000201E4E1E0930401E0930501E0E0E09300
:104EC6000701E0930801E0930A01E0930B010895BE
:104ED6000A930A2F00FF03C05D9A559A01C05D9898
:104EE600099108950A930A2F00FF03C05F9A579A03
:104EF60001C05F98099108950A930A2F6B9A0030B2
:104F060011F40C948827739A01C073980991089537
:104F1600639B02C0E1E00895E0E008950E94F9B1C4
:104F2600E860E0930101003011F40C94A027E091B1
:104F36000201E860E093020105C0E0910201E77F0B
:104F4600E0930201099108956F980E94FEB1679B54
:104F560002C0E0E00895E1E008951A930A9300E0A4
:104F660010E0649901C011E0A49B01C010E010306C
:104F760011F40C94BF270061659901C0006266991F
:104F860001C00064679901C00068E02F099119917A
:104F960008950A930A2F9A9A003011F40C94D52793
:104FA600A29A01C0A298099108950A930A2F003087
:104FB60011F40C94E227A0E00E94CC2703C0A1E0E4
:104FC6000E94CC27099108959A9B03C0A29B01C019
:104FD60001C002C0E1E00895E0E008956E980E94E5
:104FE600FEB1669B02C0E0E00895E1E008950E94EC
:104FF600F9B1E061E0930101003011F40C94092845
:10500600E0910201E061E093020105C0E091020136
:10501600EF7EE093020109910895E0910001E071AD
:1050260011F40C941828E1E00895E0E008950E9438
:1050360002B2E064E0930A01003011F40C942928CE
:10504600E0910B01E064E0930B0105C0E0910B01D8
:10505600EF7BE0930B0109910895E0910901E0745B
:1050660011F40C943828E1E00895E0E008950A93DD
:105076000A2F0E947115539A003011F40C9445289A
:105086005B9A01C05B98099108950E947115529828
:105096000E94FEB14A9B02C0E1E00895E0E0089557
:1050A6000E94A42EE03011F00C945B28E0E00895F5
:1050B60023980E94FEB11B9B02C0E0E00895E1E048
:1050C600089523980E94FEB11B9B02C0E1E008955B
:1050D600E0E008950A930A2F249A003011F40C9404
:1050E60076282C9A01C02C98099108950A930A2FC4
:1050F600229A003011F40C9482282A9A01C02A9828
:10510600099108950E9402B2E062E0930A0100301C
:1051160011F40C949428E0910B01E062E0930B01EA
:1051260005C0E0910B01EF7DE0930B010991089515
:10513600E0910901E07211F40C94A328E1E00895CE
:10514600E0E008950A930A2F0E945E17E09101019C
:10515600E260E0930101003011F40C94B828E0916C
:105166000201E260E093020105C0E0910201ED7FD9
:10517600E0930201099108950E945E17E0910101F2
:10518600EE7F0E9407B2E0910001E17011F40C94E9
:10519600CE28E1E00895E0E008950E94F9B1E064C8
:1051A600E0930101003011F40C94DF28E091020134
:1051B600E064E093020105C0E0910201EF7BE09319
:1051C600020109910895E0910101EF7D0E9407B265
:1051D600E0910001E07211F40C94F328E0E00895E8
:1051E600E1E0089538980E94FEB1309B02C0E0E0ED
:1051F6000895E1E008950A930A2F399A003011F4D0
:105206000C940729419A01C0419809910895419B40
:1052160002C0E1E00895E0E008953A980E94FEB1E8
:10522600329B02C0E1E00895E0E00895E0910101BB
:10523600EF770E9407B2E0910001E07811F40C9438
:105246002629E1E00895E0E008950E9419290895CD
:105256000A930A2F0E94C118E0910401E260E093CC
:105266000401003011F40C943E29E0910501E2603E
:10527600E093050105C0E0910501ED7FE09305018E
:10528600099108950E94C118E0910401EE7FE09310
:1052960004010E94FEB1E0910301E17011F40C9447
:1052A6005629E1E00895E0E008950A930A2F279A27
:1052B600003011F40C9461292F9A01C02F9809919E
:1052C60008952F9B03C0279B01C001C002C0E1E0E7
:1052D6000895E0E008950A930A2F9C9A003011F48D
:1052E6000C947729A49A01C0A49809910895A49BC7
:1052F60002C0E0E00895E1E008956C980E94FEB1D6
:10530600649B02C0E0E00895E1E008950A930A2F45
:105316009B9A003011F40C949229A39A01C0A39889
:10532600099108956D98759A0E94FEB1659B02C019
:10533600E0E00895E1E008950A930A2F269A0030E6
:1053460011F40C94A8292E9A01C02E98099108955B
:105356002E9B03C0269B01C001C002C0E1E0089558
:10536600E0E008950A930A2F259A003011F40C9470
:10537600BE292D9A01C02D98099108951D9B02C042
:10538600E1E00895E0E008950A930A2F569A003066
:1053960011F00C94D0295E9805C0013011F00C94E0
:1053A600D5295E9A099108954E9B02C0E1E00895C1
:1053B600E0E008950E9402B2E068E0930A0100303E
:1053C60011F00C94EC29E0910B01EF77E0930B01BF
:1053D60009C0013011F00C94F529E0910B01E06849
:1053E600E0930B0109910895E0910901E07811F429
:1053F6000C94FF29E1E00895E0E0089554980E9496
:10540600FEB14C9B02C0E1E00895E0E008950A93E6
:105416000A2F3B9A003011F40C94132A439A01C0C8
:105426004398099108953C980E94FEB1349B02C0AE
:10543600E1E00895E0E008950A930A2F003011F0A4
:105446000C94282A3D9845980DC0013011F00C9413
:105456002F2A3D9A459806C0023011F00C94352A41
:105466003D98459A099108953D98459A0E94FEB146
:10547600359B02C0E0E00895E1E008950A930A2F03
:10548600003011F00C944A2A3E9846980DC001301F
:1054960011F00C94512A3E9A469806C0023011F03B
:1054A6000C94572A3E98469A099108950A930A2F12
:1054B6003E9A003011F40C94622A469A01C046982E
:1054C600099108953E98469A0E94FEB1369B02C005
:1054D600E0E00895E1E008950A930A2F003011F004
:1054E6000C94782A9898A0980DC0013011F00C946D
:1054F6007F2A989AA09806C0023011F00C94852A4B
:105506009898A09A099108950A930A2F989A0030BC
:1055160011F40C94902AA09A01C0A09809910895BC
:105526009898A09A0E94FEB1909B02C0E0E0089570
:10553600E1E008950A930A2F003011F00C94A62A90
:105546009998A1980DC0013011F00C94AD2A999A42
:10555600A19806C0023011F00C94B32A9998A19A2A
:10556600099108950A930A2F999A0E94FEB1003074
:1055760011F40C94C02AA19A01C0A198099108952A
:105586009998A19A919B02C0E0E00895E1E0089500
:105596000A930A2F003011F00C94D42A0B98139812
:1055A6000DC0013011F00C94DB2A0B9A139806C03B
:1055B600023011F00C94E12A0B98139A0991089580
:1055C6000A930A2F0B9A003011F40C94EC2A139AC2
:1055D60001C01398099108950B98139A0E94FEB181
:1055E600039B02C0E0E00895E1E008950A930A2FC4
:1055F600003011F00C94022B099811980DC001305F
:1056060011F00C94092B099A119806C0023011F07A
:105616000C940F2B0998119A099108950A930A2F51
:10562600099A003011F40C941A2B119A01C01198A2
:10563600099108950998119A0E94FEB1019B02C032
:10564600E0E00895E1E008950E9402B2E260E0938E
:105656000A01003011F40C94362BE0910B01E26044
:10566600E0930B0105C0E0910B01ED7FE0930B0188
:1056760009910895E0910901E27011F40C94452B0B
:10568600E1E00895E0E008950E9402B2E460E0934C
:105696000A01013011F00C94562BE0910B01E460E5
:1056A600E0930B0105C0E0910B01EB7FE0930B014A
:1056B60009910895E0910901E47011F40C94652BA9
:1056C600E1E00895E0E008953D98459A3D98459AB1
:1056D600E0E008950A930A2F3D98459AE0910A0161
:1056E600E061E0930A01003011F40C94802BE09104
:1056F6000B01E061E0930B0105C0E0910B01EF7E29
:10570600E0930B01099108950E9402B2E061E093D3
:105716000A01003011F40C94962BE0910B01E06124
:10572600E0930B0105C0E0910B01EF7EE0930B01C6
:10573600099108950E9402B2E860E0930A010030E0
:1057460011F40C94AC2BE0910B01E860E0930B0193
:1057560005C0E0910B01E77FE0930B0109910895E5
:10576600E0910901E87011F40C94BB2BE1E0089577
:10577600E0E0089508950E9402B2E160E0930A0114
:10578600013011F00C94CD2BE0910B01E160E09318
:105796000B0105C0E0910B01EE7FE0930B0109912F
:1057A6000895E0910901E17011F40C94DC2BE1E01D
:1057B6000895E0E008950A930A2F829A839A0130A9
:1057C60011F00C94E92B8B988A9A09C0023011F0DB
:1057D6000C94F02B8A988B9A02C08A988B98099120
:1057E60008950A930A2FA1E00E942C2EA02F0E9452
:1057F600DE2B099108950A9300E07B9B01C00160AE
:105806007A9B01C00260E02F099108950A930A2F3E
:10581600829A003011F40C94122C8A9A01C08A984C
:105826000991089583988B9A0E94FEB17B9B02C0D2
:10583600E1E00895E0E008950E940AB2E0910701D0
:10584600E260E0930701013011F00C94332CE091F3
:105856000801E1600E9412B2ED7FE093080115C0D5
:10586600023011F00C94402CE0910801EE7F0E946A
:1058760012B2E260E093080108C0E0910801EE7FF1
:105886000E9412B2ED7FE0930801099108950A93F0
:1058960000E0E0910601E27011F40C94532C0160D3
:1058A600E0910601E17011F40C945A2C0260E02F8D
:1058B600099108950E940AB2003011F40C94692CE3
:1058C600E0910801E160E093080105C0E09108015C
:1058D600EE7FE093080109910895E0910701ED7FBD
:1058E6000E9417B2E260E0930801E0910601E270BF
:1058F60011F40C94802CE1E00895E0E008950E94F4
:105906001CB2E064E0930701003011F40C94912C72
:10591600E0910801E064E093080105C0E091080108
:10592600EF7BE093080109910895E0910801E07486
:1059360011F40C94A02CE1E00895E0E00895E091C4
:105946000701EF770E9417B2E0680E9421B2E0914A
:105956000601E07811F40C94B22CE1E00895E0E041
:105966000895E0910701EB7F0E9417B20E9424B2CE
:1059760011F40C94C02CE0E00895E1E00895E09164
:105986000701EB7F0E9417B20E9424B211F40C9417
:10599600CE2CE1E00895E0E00895E0910701E77F6D
:1059A6000E9417B2E8600E9421B2E0910601E870F9
:1059B60011F40C94E02CE1E00895E0E008950E94D3
:1059C6001CB2E860E0930701003011F40C94F12C4E
:1059D600E0910801E860E093080105C0E091080144
:1059E600E77FE093080109910895E0910701EF7EB2
:1059F6000E9417B2E0610E9421B2E0910601E071B7
:105A060011F40C94082DE0E00895E1E008950E9459
:105A16001CB2E061E0930701003011F40C94192DDB
:105A2600E0910801E061E093080105C0E0910801FA
:105A3600EF7EE093080109910895E0910701EF7D5B
:105A46000E9417B2E0620E9421B2E0910601E07264
:105A560011F40C94302DE1E00895E0E008950A93E6
:105A66000C98149A0E94FEB100B104FF03C0E1E055
:105A760009910895E0E0099108950A930D98159A01
:105A86000E94FEB100B105FF03C0E1E0099108954F
:105A9600E0E0099108950A930A2F0D9A003011F457
:105AA6000C94572D159A01C01598099108950A93DB
:105AB6002098289A0E94FEB103B100FF03C0E0E0DF
:105AC60009910895E1E0099108950A930A2F209A11
:105AD600003011F40C94712D289A01C02898099170
:105AE60008950A932198299A0E94FEB103B101FFF5
:105AF60003C0E0E009910895E1E0099108950A9351
:105B06000A2F219A003011F40C948B2D299A01C08A
:105B16002998099108950F98179A0E94FEB1079B3C
:105B260002C0E0E00895E1E008950E942FB2E06827
:105B3600E0930401013011F00C94A72DE0910501CA
:105B4600E068E093050105C0E0910501EF77E09379
:105B5600050109910895E0910301E07811F40C9490
:105B6600B62DE1E00895E0E008950E942FB2E064CA
:105B7600E0930401003011F40C94C72DE091050167
:105B8600E064E093050105C0E0910501EF7BE09339
:105B9600050109910895E0910301E07411F40C9454
:105BA600D62DE1E00895E0E008950E942FB2E0626C
:105BB600E0930401003011F40C94E72DE091050107
:105BC600E062E093050105C0E0910501EF7DE093F9
:105BD600050109910895E0910401EF7DE093040128
:105BE600E0910501E062E0930501E0910301E072B6
:105BF60011F40C94002EE1E00895E0E00895E091A0
:105C06000301E07211F40C940A2EE1E00895E0E03D
:105C160008950E942FB2E061E0930401003011F470
:105C26000C941B2EE0910501E061E093050105C08F
:105C3600E0910501EF7EE093050109910895E09159
:105C46000501E07111F40C942A2EE1E00895E0E0DC
:105C560008950E942FB2E860E0930401003011F429
:105C66000C943B2EE0910501E860E093050105C028
:105C7600E0910501E77FE093050109910895E09120
:105C86000301E87011F40C944A2EE1E00895E0E077
:105C960008950E942FB2E460E0930401003011F4ED
:105CA6000C945B2EE0910501E460E093050105C0CC
:105CB600E0910501EB7FE093050109910895E091DC
:105CC6000401EB7FE09304010E94FEB1E091030121
:105CD600E47011F40C94712EE1E00895E0E008956B
:105CE6000A930A2F003011F40C947B2E479A01C0B8
:105CF60047983F9A09910895479B02C0E1E00895AD
:105D0600E0E008953F9847980E9434B2379B02C05E
:105D1600E1E00895E0E008956A980E94FEB1629B72
:105D260002C0E1E00895E0E008950E94E6280895A3
:105D36000A930A2F0E94732E099108950E94622EDB
:105D460008959D980E94FEB1959B02C0E1E00895DA
:105D5600E0E00895E0910101EB7F0E9407B2E09137
:105D66000001E47011F40C94BA2EE1E00895E0E02D
:105D760008950A98129A0E94FEB1029B02C0E1E0C1
:105D86000895E0E008950A930A2F089A003011F466
:105D96000C94D22EA1E00E942C2E109A01C01098CD
:105DA600099108950898109A0E94FEB1009B02C0BE
:105DB600E1E00895E0E00895A1E00E942C2E089508
:105DC6000A930E94A42E0E2F003011F00C94EE2E92
:105DD600E3E6099108950E98169A0E94FEB1069B75
:105DE60003C0E0E009910895E1E0099108950E9855
:105DF600169A0E94FEB1069B02C0E0E00895E1E01B
:105E060008950E9438B208950E949CC3A1971A93E0
:105E16000A930E9438B20E943EB2ABA1BCA18DA1EA
:105E26009EA10E9444B210F40C941A2F10E200E0D6
:105E3600011710F00C942D2F0E9449B20E944EB209
:105E4600ABA1BCA18DA19EA10E9421B1D001EC9372
:105E56000F5FEECF0E9453B20E94A41419810881ED
:105E6600A7960895EF9723970E9406C29D010E9468
:105E760038B20E943EB20E945EB20E9444B210F452
:105E86000C94462F10E200E0011710F00C94592FE5
:105E96000E9467B2FF93EF93E02F0E945EB20E94CA
:105EA60021B1AF91BF91EC930F5FEECF0E946EB21E
:105EB600D9010E94F81A1E2F113410F40C94642F85
:105EC60010E400E0011710F00C946F2F0E9467B2E7
:105ED6000E947AB20F5FF6CF0E946EB20E940DC288
:105EE600EF962B9608950E9407C211E020E02A3013
:105EF60010F00C94942FA0E00E94CC27AFE00E94F3
:105F060083B211F40C94882F10E0A1E00E94CC27F4
:105F1600A3E00E9483B211F00C94922F10E02F5F41
:105F2600E6CFE12F0E940EC223960895EF97A5971C
:105F36000E948BB20E9490B20E944E13A1E00E9472
:105F4600FA270E9496B2ACE6B1E080E090E00E94AB
:105F5600072FA0E8B1E080E090E00E94072F0E94A2
:105F66009AB2E1EAF1E060E070E00E94A6B20E9417
:105F7600EC1CE7EBF1E060E070E00E94A6B20E9444
:105F8600352F0E949AB2E3ECF1E060E070E00E94E7
:105F9600A6B20E94EC1CE0EDF1E060E070E00E9429
:105FA600A6B20E94352F0E949AB2ECEDF1E060E0B5
:105FB60070E00E94A6B20E94EC1CE9EEF1E060E0FF
:105FC60070E00E94A6B20E94352F0E94042FEF9621
:105FD600A5960895AA93EF972F970E94ABB240E03B
:105FE6000E94B0B2E03011F40C940030A5EFB1E09D
:105FF60080E090E00E94B5B206C0AFEFB1E080E06D
:1060060090E00E94072F0E94BAB2523010F40C940E
:1060160017300E9496B20E94C1B2A3E00E94C550FA
:106026000E9496B20E94BAB2503011F00C945630CB
:10603600FE01EB5BFF4FE081EA930E94CFB2EA9349
:10604600FE01EA5BFF4FE081EA930E942DAEDE017E
:10605600D4960E94821FE6E0F2E060E070E00E94C3
:10606600D4B2FE01E85BFF4FE081EA93FE01E85BF4
:10607600FF4FE081EA93E0E2EA93FE01E75BFF4F20
:10608600E081EA930E942DAEDE01D5960E942E2075
:10609600E3E1F2E060E070E00E94D4B20E94CFB289
:1060A600E093D91106C0A0E2B2E080E090E00E9441
:1060B600B5B2A2E00E9417510E94DAB20E9455378B
:1060C6000E94E0B2DE01AF5BBF4FAC91A13010F48D
:1060D6000C947430AEE2B2E080E090E00E94B5B27B
:1060E60006C0A2E4B2E080E090E00E94072FA1E0A3
:1060F6000E947527A0E00E946B27FE017D960E94F4
:10610600E5B20E9492515E2F503011F40C948E30FD
:106116004F5FE1E0EE83E0E0EDA7E3E5F2E060E06B
:1061260070E00E9497C3DE0191960E94352FE0E051
:10613600EB8FE4E6F2E060E070E00E9497C3DE01D8
:106146001B960E94352FA1E00E94B2370E94E0B252
:106156000E94EAB2E03011F00C94B330E1E0EE8335
:10616600A1E00E946B27AAE00E94DD0FA0E00E943A
:106176001C53AAE00E94F40F8F010436E0E01E07CC
:1061860010F00C94C730F2CF0E94D4520E941754DC
:106196009F010E9417549F010E9417549F012A5F76
:1061A60030402031E7E23E0710F40C94E13021380C
:1061B600EEE33E0710F00C94E13007C0A5E7B2E02D
:1061C60080E090E00E94B5B20DC03A932A93DE01BA
:1061D600AC5BBF4F0E94171DE3E8F2E060E070E0A1
:1061E6000E94EFB20E9407549F012A503040283285
:1061F600E0E03E0710F40C9407312530E1E03E075D
:1062060010F00C94073107C0A9E9B2E080E090E0F5
:106216000E94B5B20FC03A932A930E94F6B2DE01ED
:10622600A85BBF4F0E94121AEBEAF2E060E070E052
:106236000E94EFB2A1E00E9475270E94BA310E9427
:10624600E0B2DE01AF5BBF4FAC91A13010F40C940D
:106256003F310E94EAB2F0E0FA93EA93DE01AC5BCA
:10626600BF4F0E94171DEFEBF2E060E070E00E9466
:10627600EFB2E1E0EE8306C0A6EDB2E080E090E08A
:106286000E94072FA1E00E942310A1E00E943F1068
:106296008F01E091D9110E94E0B20E94BAB250304B
:1062A60011F00C945A310E94CFB20E94E0B2023033
:1062B600E0E01E0710F00C946D31503011F00C9494
:1062C6006D310E94EAB2A091D911EA1711F00C942F
:1062D6006D3101C001C0D9CF0230E0E01E0710F4D5
:1062E6000C947C31A8EEB2E080E090E00E94B5B25A
:1062F60019C0503011F40C948731A8EFB2E080E059
:1063060090E00E94B5B20EC00E94EAB2A091D911E7
:10631600EA1711F40C949531A6E0B3E080E090E022
:106326000E94072FEE81E03011F00C94A131A5E117
:10633600B3E080E090E00E94072F06C0A5E2B3E03C
:1063460080E090E00E94072FEE810E940BC2EF963C
:10635600669608950A930A2F003011F00C94B63110
:106366000E94DAB202C00E94FEB2099108950E940C
:1063760007C20E94A727E093DA11A1E00E9423102A
:106386000E94FEB20E948F2EE03011F00C94CE31A6
:106396000E9404B308950E94A42EE03011F00C94DC
:1063A600D7310E9409B308950E94AD2EE03011F056
:1063B6000C94E231E3E00E940EC223960895A0E019
:1063C6000E940EB311F40C94ED31E4E00E940EC26B
:1063D60023960895A1E00E940EB311F00C94F831B3
:1063E600E5E00E940EC223960895A1E00E94FA27D6
:1063F600A0E00E943A28A0E00E941A280E94F736E0
:106406000E9416B311F40C940D32EBE00E940EC2FA
:10641600239608950E9420B311F00C941732ECE0F5
:106426000E940EC223960895A1E00E941A280E9497
:1064360016B311F40C942432EDE00E940EC223969A
:1064460008950E9420B311F00C942E32EEE00E94C3
:106456000EC2239608950E945E170E942AB3A0E0FA
:106466000E9430B3A0E00E9437B311F40C9440327E
:10647600EFE00E940EC223960895A1E00E9437B372
:1064860011F00C944B32E0E10E940EC2239608955F
:10649600A0E00E948528A1E00E9430B30E94BF2898
:1064A6000E2F003011F40C945D32E1E10E940EC211
:1064B60023960895A1E00E9437B311F00C94683238
:1064C600E2E10E940EC2239608950E9440B30E9404
:1064D60045B311F00C947432E3E10E940EC2239688
:1064E6000895A0E00E9445B311F40C947F32E3E1D5
:1064F6000E940EC223960895A2E00E94412A0E949D
:10650600EE2DA1E00E94D0280E9496B20E94C118EA
:10651600A0E00E945829A1E00E940A2A0E944EB3D8
:106526000E9455B311F40C949D32E4E10E940EC210
:10653600239608950E945AB30E9455B311F00C9405
:10654600A932E5E10E940EC2239608950E94652AAB
:106556000E2F003011F00C94B532E6E10E940EC207
:1065660023960895A0E00E94D028A0E00E940A2A5F
:106576000E9496B20E945FB30E9455B311F00C942C
:10658600C932E7E10E940EC2239608950E94652A49
:106596000E2F003011F40C94D532E8E10E940EC2A1
:1065A60023960895A0E00E94FE28A4E1B0E00E9490
:1065B600650F0E9464B311F40C94E632E9E10E947F
:1065C6000EC223960895A1E00E94FE280E94F73687
:1065D6000E9464B311F00C94F532EAE10E940EC2F7
:1065E60023960895A0E00E94FE280E9469B30E94A7
:1065F600F5280E2F003011F00C940633EBE10E94C3
:106606000EC223960895A1E00E94FE280E9496B22B
:106616000E94F5280E2F003011F40C941733ECE18C
:106626000E940EC223960895A0E00E94FE280E94B2
:10663600852E0E946DB3A1E00E940A2A0E946DB3C6
:106646000E94162A0E2F003011F00C942F33EDE124
:106656000E940EC223960895A0E00E940A2A0E9474
:10666600F7360E9469B30E94162A0E2F003011F4E5
:106676000C944233EEE10E940EC2239608950E94C6
:1066860040B30E940C2EA0E00E946E290E94EE2DBF
:106696000E9471B3A1E00E9478B311F40C945833B0
:1066A600EFE10E940EC223960895A0E00E9478B3FF
:1066B60011F00C946333E0E20E940EC22396089513
:1066C6000E945AB30E947DB311F00C946F33E1E23D
:1066D6000E940EC2239608950E945FB30E947DB366
:1066E60011F40C947B33E2E20E940EC223960895C5
:1066F600A0E00E9489290E94F7360E947DB311F41A
:106706000C948A33E3E20E940EC2239608950E94F7
:1067160071B30E9496B2A0E00E9482B311F40C9469
:106726009933E4E20E940EC223960895A1E00E94E6
:1067360082B311F00C94A433E5E20E940EC22396B4
:1067460008950E948BB3A0E00E946E290E9469B34F
:106756000E94852E0E2F003011F00C94B733E6E21E
:106766000E940EC223960895A1E00E946E290E94FF
:1067760092B30E94852E0E2F003011F40C94C8336C
:10678600E7E20E940EC223960895A0E00E946E29B9
:10679600A1E00E948929A0E00E945829A0E00E9459
:1067A6000A2AA2E00E946F2A0E9469B30E945AB385
:1067B6000E947DB311F00C94E533E8E20E940EC20C
:1067C600239608950E945FB30E947DB311F40C9442
:1067D600F133E9E20E940EC2239608950E94932A9D
:1067E6000E2F003011F40C94FD33EAE20E940EC223
:1067F600239608950E948BB30E9469B30E945AB3F0
:106806000E947DB311F00C940D34EBE20E940EC28F
:10681600239608950E945FB30E947DB311F40C94F1
:106826001934ECE20E940EC2239608950E94932A20
:106836000E2F003011F00C942534EDE20E940EC2AA
:1068460023960895A0E00E940A2A0E9469B3A0E058
:106856000E949D2A0E94C32A0E2F0E9495B30E9471
:10686600872BA1E00E94BE2B0E9492B30E94A3B385
:1068760011F00C944334EEE20E940EC22396089562
:10688600A0E00E94BE2B0E9492B30E94A3B311F413
:106896000C945234EFE20E940EC223960895A1E0B2
:1068A6000E94272B0E9492B30E94A3B311F00C946E
:1068B6006134E0E30E940EC223960895A0E00E9490
:1068C600272B0E9492B30E94A3B311F40C94703448
:1068D600E1E30E940EC223960895A1E00E94472B91
:1068E6000E9492B30E94A3B311F00C947F34E2E3AA
:1068F6000E940EC223960895A0E00E94472B0E9494
:1069060092B30E94A3B311F40C948E34E3E30E9475
:106916000EC223960895A1E00E949D2B0E9492B379
:106926000E94A3B311F00C949D34E4E30E940EC2BE
:1069360023960895A0E00E949D2B0E9492B30E9488
:10694600A3B311F40C94AC34E5E30E940EC2239673
:106956000895A1E00E94872B0E9434B20E94F73668
:106966000E94A3B311F00C94BD34E6E30E940EC25C
:1069760023960895A0E00E94872B0E9434B20E94BD
:10698600A3B311F40C94CC34E7E30E940EC2239611
:106996000895A0E00E941F2AA1E00E94C7290E9434
:1069A6006DB30E94372A0E2F003011F40C94E03498
:1069B600E8E30E940EC223960895A0E00E94C7292C
:1069C6000E946DB30E94372A0E2F003011F00C94EE
:1069D600F134E9E30E940EC223960895A1E00E94D5
:1069E600DD290E9469B30E94012A0E2F003011F0A2
:1069F6000C940235EAE30E940EC2239608950E9483
:106A06005FB30E9455B311F00C940E35EBE30E9470
:106A16000EC2239608950E945AB30E9455B311F4EC
:106A26000C941A35ECE30E940EC223960895A0E05A
:106A36000E94DD290E9496B20E94F7360E94012A22
:106A46000E2F003011F40C942D35EDE30E940EC28A
:106A5600239608950E945FB30E9455B311F00C94DB
:106A66003935EEE30E940EC2239608950E945AB36A
:106A76000E9455B311F00C944535EFE30E940EC207
:106A860023960895A1E00E94A8B311F00C94503506
:106A9600E0E40E940EC223960895A0E00E94A8B3E7
:106AA60011F40C945B35E1E40E940EC2239608951E
:106AB600A1E00E94B1B311F00C946635E2E40E94A5
:106AC6000EC223960895A0E00E94B1B311F40C946F
:106AD6007135E3E40E940EC223960895A1E00E9458
:106AE600BAB311F40C947C35E4E40E940EC22396EA
:106AF6000895A0E00E94BAB311F00C948735E5E43E
:106B06000E940EC223960895A1E00E94C3B311F01D
:106B16000C949235E6E40E940EC223960895A0E0F6
:106B26000E94C3B311F40C949D35E7E40E940EC293
:106B360023960895A1E00E94CCB311F00C94A835D9
:106B4600E8E40E940EC223960895A0E00E94CCB30A
:106B560011F40C94B335E9E40E940EC2239608950D
:106B6600A1E00E94D5B311F00C94BE35EAE40E9470
:106B76000EC223960895A0E00E94D5B311F40C949A
:106B8600C935EBE40E940EC223960895A1E00E9447
:106B9600DEB311F00C94D435ECE40E940EC22396B9
:106BA6000895A0E00E94DEB311F40C94DF35EDE405
:106BB6000E940EC223960895A1E00E94E7B311F049
:106BC6000C94EA35EEE40E940EC223960895A0E0E6
:106BD6000E94E7B311F40C94F535EFE40E940EC25F
:106BE60023960895A1E00E94F0B311F40C940036A8
:106BF600E0E50E940EC223960895A0E00E94F0B33D
:106C060011F00C940B36E1E50E940EC2239608950E
:106C1600A1E00E94F9B311F40C941636E2E50E9445
:106C26000EC223960895A0E00E94F9B311F00C94C9
:106C36002136E3E50E940EC2239608950E94EE2DAA
:106C46000E944EB30E94EE2D0E2F003011F40C94CC
:106C56003136E4E50E940EC2239608950E945AB387
:106C66000E94EE2D0E2F003011F00C943F36E5E514
:106C76000E940EC223960895A1E00E9402B411F06C
:106C86000C944A36E6E50E940EC223960895A0E0CB
:106C96000E9402B411F40C945536E7E50E940EC228
:106CA60023960895A0E00E946E290E940BB411F469
:106CB6000C946236E8E50E940EC2239608950E945F
:106CC6000BB411F40C946C36E9E50E940EC22396BF
:106CD6000895A1E00E94FA27A1E00E9415B411F0E0
:106CE6000C947A36EAE50E940EC223960895A0E037
:106CF6000E9415B411F40C948536EBE50E940EC281
:106D060023960895A0E00E94B529A1E00E949F293C
:106D16000E9496B20E941EB411F00C949736ECE5D0
:106D26000E940EC223960895A0E00E949F290E9409
:106D360096B20E941EB411F40C94A636EDE50E949C
:106D46000EC223960895A0E00E949F29A1E00E940A
:106D5600B5290E9496B20E941EB411F00C94B83662
:106D6600EEE50E940EC223960895A0E00E94B52982
:106D76000E9496B20E941EB411F40C94C736EFE539
:106D86000E940EC223960895A1E00E943F101E2F76
:106D96002F2F0E94A7270E2F1230E0E02E0710F0AB
:106DA6000C94DC36A091DA110A1711F00C94DC363B
:106DB60001C001C0E9CF0E94A7270E2FA091DA11CA
:106DC6000A1711F00C94EE361031E0E02E0710F0A1
:106DD6000C94EE3601C005C0E0E60E940EC2239672
:106DE60008950E9423B408950E9428B40895EF9749
:106DF600EF97EF9765970E9405C24A2F00E0242F70
:106E06003327D901E6E00E9448C29F0110E0103402
:106E160010F00C9415370E942CB4E12FED5FEC9323
:106E26001F5FF5CF0E9434B4DE01AB56BF4F0E9400
:106E3600160E0E9434B4DE01A15BBF4F0E94540EB1
:106E46000E9434B20E943BB4E0E0EA93A6E40E94BA
:106E560040B4E0E4F0E00E94E5B20E94160E10E0B5
:106E6600103410F00C9444370E942CB40C90E12F8F
:106E76000E9446B4E01511F40C94423701E01F5FFE
:106E8600EFCF0E9434B4DE01AB56BF4F0E94540EC2
:106E96000E9434B2E02F0E940CC2EF96EF96EF9656
:106EA6006A9608951A930A931FE3A12F0E94FA3651
:106EB6000E2F003011F40C946437E1E0099119911A
:106EC6000895E0E009911991089528970E9405C256
:106ED6004A2F10E0413011F00C94723716EA423016
:106EE60011F00C9477371EEA2CEF3FEE0E944DB45A
:106EF600E1E2F3E465E070E00E94ACAD0E9458B4B4
:106F060011F00C9492370E944DB40E946AB411F0AD
:106F16000C949237E2E00E940CC22D9608952CEF55
:106F26003FE70E944DB4E4E3F2E160E070E00E94C6
:106F3600ACAD0E9458B411F00C94AD370E944DB41C
:106F46000E946AB411F00C94AD37E1E00E940CC2C5
:106F56002D960895E0E00E940CC22D960895AA93FE
:106F66000E9407C22B81A0E00E949127A1E00E9407
:106F760068370E2F003011F00C94CA37A5E3B3E042
:106F860080E090E00E94072F0E9473B408950130BC
:106F960011F00C94DD37203011F40C94D837A7E4A7
:106FA600B3E080E090E00E94072FE1E00E940EC26D
:106FB60024960895A2E00E9468371E2F103011F023
:106FC6000C94F437203011F40C94EF37ACE5B3E0B1
:106FD60080E090E00E94072FE2E00E940EC2249615
:106FE6000895113011F00C940538203011F40C94EA
:106FF6000238A1E7B3E080E090E00E94072F0E94EC
:1070060073B40895123011F00C941838203011F42E
:107016000C941338A9E8B3E080E090E00E94072FB3
:10702600E3E00E940EC2249608950E9473B4089568
:10703600A0E00E94F5180895AFEF0E94F518089594
:107046000A9300E0023010F00C944C38ABE20A9F31
:10705600F001E55DFD4E0E9478B4E45DFD4E0E94B0
:1070660078B4E35DFD4E0E9478B4E25DFD4E0E9469
:1070760078B4E15DFD4E0E9478B4E05DFD4E0E945D
:1070860078B4EF5CFD4E0E9478B40E947EB40F5F28
:10709600D9CFE1E0E03011F40C945638E03011F429
:1070A6000C94563801C006C0E1E0E0932B12EBE7E2
:1070B600E0932C12E0E0E0932812E0932A12E0938A
:1070C600291200E0063210F00C947138E02F0F5FA1
:1070D6000E9483B40E9487B40F5FF4CFE0E0E09390
:1070E6002712099108950E9407C2E0912912E03003
:1070F60011F00C9481380E948CB408950E94553A80
:10710600E03011F00C948A380E948CB40895E09116
:107116002A12E03011F00C94AF38E0E0E0938212CE
:10712600E09381120E94F93A0E2F003011F40C946C
:10713600AF380E94373BA09128120E94BE3B1E2FFB
:10714600103011F00C94AB38E1E0E0932A1204C041
:1071560020E00E9423B40895A0912A12A13011F0D4
:107166000C94FF380E94843C0E2F013011F00C94D1
:10717600CB380E9495B40E949EB40E94A3B40E948C
:10718600A9B40E94AEB4EE5CFD4EA1E0A0831FC080
:10719600023011F00C94D938E2E0E0932A12A0EA0A
:1071A600B3E080E090E00E94799A11C0033011F0BC
:1071B6000C94E138E3E0E0932A1209C0E2E0E093A0
:1071C6002A12ACEAB3E080E090E00E94799A03309C
:1071D60011F40C94FE3820E0263210F00C94FB38A3
:1071E600E22F2F5F0E9483B40E9487B42F5FF4CFF3
:1071F600E0E0E093271286C0A0912A12A23011F097
:107206000C943E39E0918212EF5FE0938212A091D6
:107216008212A33010F40C942A390E94A3B4EE5CB7
:10722600FD4EA2E0A0830E94A3B40E94A9B40E94CE
:10723600AEB4E15DFD4EA0E0A083E0E0E0932A124B
:10724600ABEBB3E080E090E00E94799A13C0A09186
:1072560028120E94303C1E2F103011F00C94393940
:10726600E1E0E0932A120E9404B3089520E00E9410
:1072760023B4089547C0A0912A12A33011F00C94AC
:107286008539E0918112EF5FE0938112A09181121E
:10729600A33010F40C945D390E94A3B4EE5CFD4E4D
:1072A600A3E0A0830E94A3B40E949EB40E9495B45A
:1072B6000E94B3B40E944C3B0E2F003011F40C9484
:1072C6006839E1E0E0932A120DC0A09128120E94CD
:1072D600923B0E94A3B4EE5CFD4EA4E0A083E0E0E6
:1072E600E0932A1220E0263210F00C948239E22F25
:1072F6002F5F0E9483B40E9487B42F5FF4CFE0E033
:10730600E09327120E9404B30895A1E00E942B295E
:10731600AEE6B0E00E94650FA0E00E942B2908951A
:107326000A930E94AD2E0E2F003011F40C94A23950
:10733600E0912912E03011F40C94A23901C003C087
:10734600E1E009910895E0E009910895A0E00E9426
:107356008929A0E00E946E290E94C118E0E0E0930E
:107366002912A7ECB3E080E090E00E94799A089594
:10737600A0E00E9458290E9440B30E940C2EA1E072
:107386000E946E290E948BB2E4E00E94B8B40E946B
:1073960037180E94C518E1E0E0932912AFECB3E07C
:1073A60080E090E00E94799AE1E008950A930A2F1E
:1073B600013011F00C94E339A1E00E946E2915C04A
:1073C600023011F00C94F539A1E00E946E290E945A
:1073D60034B2A0E00E946E290E9434B2A1E00E945D
:1073E6006E2903C0A0E00E946E29099108950E94AB
:1073F6002EADA0912712A63210F00C940E3AE09111
:107406002712EF5FE0932712E150ABEDB1E10E9446
:10741600F3B1108321831030E1E02E0714F40C94AD
:107426001B3AA0912712A13011F00C941B3A01C00F
:1074360003C0009127120F5F0E940EC22396089583
:107446000E9483B110F00C94513A003011F40C9460
:107456003A3AABE21A9FF001E35DFD4EA1E0A0834C
:10746600A6EDB3E080E090E00E94799A17C0ABE207
:107476001A9FF001E35DFD4E0E94BDB40E94B3B4B5
:107486000E94C3B40E94BDB40E949EB40E94C9B4B7
:10749600A8EEB3E080E090E00E94799A1981088115
:1074A600239608950A9300E0023010F00C94683A8F
:1074B600ABE20A9FF0010E94CDB411F40C94663A37
:1074C600E1E0099108950F5FEFCFE0E0099108959B
:1074D6000E9483B110F00C947A3AABE21A9FF00145
:1074E600E25DFD4E00830E94C3B4A0E0A083198133
:1074F6000881239608950E9405C28D012D813E8143
:107506004F811A930A93ABE24A9FF001ED5CFD4E60
:10751600FA93EA93A22FBB270E94E71B423010F092
:107526000C94A03AABE24A9FF001E25DFD4E308337
:107536004A9FF001E05DFD4E20830E940CC2289612
:1075460008951A930A931A2F123010F00C94BC3A2D
:1075560000E0033210F00C94BC3AABE21A9FF00143
:10756600ED5CFD4EDF01EE27A00FBE1FEC930F5F13
:10757600F0CF0E94C3B40E94BDB40E949EB40E9484
:10758600C9B40991199108951A930A931A2FABE277
:107596001A9FF001EE5CFD4E00810E94C9B4E02FF7
:1075A6000991199108950A930A2FABE20A9FF001F7
:1075B600EF5CFD4EE081099108950E9407C28D019E
:1075C6002B81ABE22A9FF001ED5CFD4EFA93EA9324
:1075D6001A930A932A9FF001EF5CFD4EA081B0E05A
:1075E6000E94E71B0E940EC2249608950E9406C2BE
:1075F6002FE030E0A9E00E94F40F8F010217130775
:1076060010F00C940B3BE0E00E940DC22496089506
:10761600A9E00E94DD0F20E030E0E0912812EF5F44
:10762600E0932812A0912812A23010F40C941E3B6D
:10763600E0E0E09328120E94A3B40E94CDB411F4B6
:107646000C942A3BE1E00E940DC224960895F901AC
:1076560031969F01339710F00C94323BDECFE0E079
:107666000E940DC2249608950E94AFAD0632E0E056
:107676001E0714F00C94473BF8010E94D2B40E94F6
:1076860087B40F5F1F4FF2CF0E94C5180991199159
:10769600089522970E9404C2A0912712A13010F4E7
:1076A6000C945C3BE0912712E150F0E0EE83FF83FF
:1076B60003C0E0E0EE83EF8300E010E020E030E07E
:1076C600EE81FF812E173F0710F00C94723BF901F3
:1076D6000E94D2B40E94D5B42F5F3F4FF1CF1070F5
:1076E600EE81FF810E94D2B44D915C91507040179B
:1076F600510711F40C94893BE0E0E093DB11E09331
:10770600DC11E1E00E940BC228960895EE81FF810C
:107716000E94D2B40E9487B40E94DAB408950E94EF
:1077260007C22A2F10912712113010F40C949C3B9B
:10773600115000E0011710F00C94B43BABE22A9F05
:10774600F001ED5CFD4EDF01E02F0E9478B1E02FE5
:10775600ABEDB1E1F0E0EE0FFF1F0E94A4AF0F5FAB
:10776600E9CFABE22A9FF001EF5CFD4E10830E9449
:107776000EC2239608950E94DFB411F00C94C83B04
:10778600E1E00E940BC2AD9608950E94EDB40E94FE
:10779600CDB411F00C94D43BE2E00E940BC2AD963E
:1077A60008950E94EDB4E25DFD4E1081113010F493
:1077B6000C94E73B0E94EDB4E15DFD4E10830E9400
:1077C600EDB40E94B3B40CC00E94EDB4E15DFD4E71
:1077D600BF010E94EDB4E45DFD4EE081DB01EC9358
:1077E6000E94F2B4BF010E94EDB40E94FAB4E05DBB
:1077F600FD4E2081103011F00C94023C20E0243222
:1078060010F40C94073C23E20E8140E050E0E22F96
:107816000E9400B514F00C94193C0E94EDB40E942D
:1078260005B51083010F4F5F5F4FF1CF0E94F2B491
:1078360000830E9475B10E940BB5E32F0E9400B52C
:1078460014F00C942B3C0E941BB54F5F5F4FF5CF95
:10785600E0E00E940BC2AD9608950E94DFB411F0DD
:107866000C943A3CE1E00E940BC2AD9608950E944A
:10787600EDB40E94CDB411F00C94463CE2E00E94B7
:107886000BC2AD960895A9EFB3E080E090E00E94A8
:10789600799A0E94F2B4BF010E94EDB40E94FAB434
:1078A600E05DFD4E2081243210F40C945B3C23E213
:1078B6000E8140E050E0E22F0E9400B514F00C94D7
:1078C6006D3C0E94EDB40E9405B51083010F4F5F19
:1078D6005F4FF1CF0E94F2B400830E9475B10E94FF
:1078E6000BB5E32F0E9400B514F00C947F3C0E9468
:1078F6001BB54F5F5F4FF5CFE0E00E940BC2AD9620
:10790600089525970E9422B5E0E0EC830E9489B194
:10791600EAEFF0E0EE83FF830E9428B4A0912712DD
:10792600A13010F40C94BF3CE885EA1710F00C94D3
:10793600A53CEE81FF81EC59FF4FEE83FF83E0917A
:107946002712E88720E030E0E0912712D901F0E025
:10795600AE17BF0710F00C94BF3CF9010E94D2B4D9
:107966000E9484C3F17011F40C94BC3CE22FEF5FCB
:10797600EA872F5F3F4FE8CF0F5F1F4F0E9417B177
:1079860010F00C94D23CA0912712A83210F00C945F
:10799600D23CAA85A03011F00C94D23C01C001C0A3
:1079A600BBCFA091DB11B091DC11A030E1E0BE07A6
:1079B60011F00C94E53CA0912712A13011F00C9423
:1079C600E53C01C005C0E1E00E940BC22B9608957C
:1079D600AA85A03011F40C94FC3C0E9417B110F05B
:1079E6000C94FC3CA0912712A03011F40C94FC3CA2
:1079F60005C0E2E00E940BC22B9608954091271223
:107A0600552750704150504020E030E0241735078C
:107A160010F00C94183DF9010E94D2B4EC91A9859E
:107A2600EA0FE9872F5F3F4FF1CFE0912712E15030
:107A3600ABEDB1E10E9426B5F070A985B0E0EA177A
:107A4600FB0711F40C942E3D0E941F38E2E00E94C1
:107A56000BC22B9608950E941B38E3E00E940BC2CE
:107A66002B9608950E940BC22B9608950A9300E068
:107A7600083010F00C94503DA3E00A9FF001EF533C
:107A8600FD4E0E942AB5EE53FD4E0E942AB5ED53D7
:107A9600FD4EA0E0A0830F5FEBCFE0E0E093D912AC
:107AA600E093DB12E3E6E093DA12E0E0E093DD1226
:107AB600E093DC1209910895E3E6E093DA120E945E
:107AC60030B5A4E0B4E080E090E00E94799A089591
:107AD600AA970E9404C2A091DA12A33611F00C9460
:107AE600793DE0E00E940BC2E0960895E091DA123B
:107AF600E03011F00C94943D0E949339E03011F47B
:107B06000C948D3D0E9435B510F40C948C3D0E946A
:107B16003DB502C00E9443B5E0E00E940BC2E0966C
:107B26000895A091DA12A13011F00C94A23D0E94A2
:107B3600393DE2E0E093DA120E9449B535C2A091E0
:107B4600DA12A23011F00C94B33D0E9435B510F450
:107B56000C94B23DE0E0EA93A8E70E9452B524C235
:107B6600A091DA12A33011F00C94EF3D0E9458B5A3
:107B7600013011F40C94C43D043011F40C94C43D4E
:107B860004C00E943DB50E9443B50E945DB54536CE
:107B9600E0E05E0710F40C94E53D0E9462B5A63065
:107BA60010F40C94E23D0E9430B5E0E0E093DC1264
:107BB600E9ECE093E912E0E0E093DA1203C0E1E0D9
:107BC600E093DA120E949339E03011F00C94EE3D06
:107BD600E0E0E093DA12E8C1A091DA12A43011F0E5
:107BE6000C94003E0E945DB54333E0E05E0710F45E
:107BF6000C94FF3D0E943DB5D7C1A091DA12A53085
:107C060011F00C940C3EE0E0EA93A9E70E9452B50D
:107C1600CBC1A091DA12A63011F00C94CC3E0E9492
:107C26005DB54536E0E05E0710F40C942D3E0E94EB
:107C360062B5A43010F40C94273E0E9430B50E9421
:107C46006AB50E9474B50895E4E0E093DA120E94E2
:107C560074B508950E9458B5043011F00C94C23ED4
:107C66000E9479B5153010F00C944B3E0E9462B517
:107C7600A53610F40C94443E0E9430B50E946AB5B5
:107C860006C0A5E10E94DD0FE4E0E093DA1277C0BA
:107C96000E947EB5E985EA93AB850E94B521E09303
:107CA6008712F0938812EB85E0938312EC85E093BC
:107CB6008412ED85E093851220E0283010F00C94B4
:107CC6006F3EE22FE25F0E9484B5F0E0EA0FFB1FF1
:107CD600AE81A0832F5FF1CF20E0283010F00C9406
:107CE600803EE22FE95F0E9484B5E85FF0E0EA0F8C
:107CF600FB1FAE81A0832F5FF0CFA6E4B0E00E9409
:107D0600ACC32E2F213010F40C948E3E213110F08E
:107D16000C948E3E01C008C02150ABE8B2E1EE27BC
:107D2600A20FBE1FE3E0EC93E1E0E0939B120E94FA
:107D36003DB5A5E10E94DD0FE1E0E093E912E09197
:107D46008712F0918812EE83FF83ECE0F4E060E0A6
:107D560070E00E9497C3AA85BB850E9491B53091B9
:107D66008312EAE1F4E060E070E00E9495B530919C
:107D76008412E6E2F4E060E070E00E9495B50E94AD
:107D86009339E03011F00C94CB3EE0E0E093DA1248
:107D96000BC1A091DA12A73011F00C94DA3EE0E0A4
:107DA600EA93A9E70E946B3A0E943DB5FDC0A091F7
:107DB600DA12A83011F00C94183FE091DC12E03092
:107DC60011F40C94F33EE091DD12E03011F00C94C6
:107DD600F33EA091D912A83010F00C94F33E01C0E6
:107DE60003C0E9E0E093DA12E091DC12E03011F42E
:107DF6000C940A3FE091DD12E03011F40C940A3F36
:107E0600A091D912A83010F00C940A3F01C003C00B
:107E1600EAE0E093DA120E949339E03011F00C9414
:107E2600173FE0E0E093DA12BFC0A091DA12A93062
:107E360011F00C94593FE091DC12E03011F00C94F3
:107E4600273FEAE5E093DA12E091DD12E03011F423
:107E56000C94303FEAE0E093DA120E949339E03066
:107E660011F00C94393FE0E0E093DA12A091D912B8
:107E7600A83010F40C94423FEAE5E093DA120E942F
:107E860058B5043011F00C94583F0E9479B5113062
:107E960010F40C94583F0E947EB51A93DE01199691
:107EA6000E94DD41EAE5E093DA127EC0A091DA1283
:107EB600AA3011F00C94973FE091DC12E03011F0FB
:107EC6000C94683FEAE5E093DA12E091DD12E030C7
:107ED60011F00C94713FEBE0E093DA120E949339B3
:107EE600E03011F00C947A3FEAE5E093DA12A091C3
:107EF600D912A83010F40C94833FEAE5E093DA1225
:107F06000E9458B5043011F00C94963F0E9479B542
:107F1600113010F40C94963F0E947EB51A93DE0140
:107F260019960E94DD4140C0A091DA12AB3011F0E3
:107F36000C94A33FA5E10E94DD0F0E943DB534C01D
:107F4600A091DA12AC3011F00C94BA3F0E945DB5E4
:107F56004536E0E05E0710F40C94B93F0E9430B558
:107F6600E0E0E093DC12EAE5E093DA121DC0A091AE
:107F7600DA12AA3511F00C94C63FA5E10E94DD0F76
:107F86000E943DB511C0A091DA12AB3511F00C94E8
:107F9600D73F0E945DB54536E0E05E0710F40C94CD
:107FA600D73FE3E6E093DA120E9474B508950E9483
:107FB60004C2AD01EF81F885E0939D12F0939E1205
:107FC600EE81E0939F1200E010E00031E0E01E0732
:107FD60010F00C940040F801DA010E94E1B12D91F5
:107FE6003C91A1EAB2E1F8010E949DB5208331835C
:107FF60021E030E00F5F1F4FE8CFE1E0E0939B12F6
:108006000E94A2B50895A4970E9407C220E02231DB
:1080160010F00C941840E22FF0E0DE0113960E9457
:10802600E1B10E9487B42F5FF2CFE5E0F0E0E98F7F
:10803600FA8FEAE0F0E0E98FFA8FE4E1F0E0EB8F07
:10804600FC8FE2E3F0E0ED8FFE8FE4E6F0E0EF8FE9
:10805600F8A3E8ECF0E0E9A3FAA30FEF1FEF1A93F9
:108066000A930E94A7B50E94DA3FE0E00E940EC282
:10807600A79608950E949339E03011F00C94484079
:10808600E0E0E093DA12E1E00895E0E00895E0919F
:10809600DA1208950A930A2FA091DA12A33611F084
:1080A6000C945840E0E0E093DA12A091DA12A63080
:1080B60010F00C946140E0E009910895003011F051
:1080C6000C946C400E9430B5E0E0E093DC1209911C
:1080D60008950E9449B5E1E00991089526971A93FB
:1080E6000A93A091DA12A33611F00C947D40E0E0D9
:1080F600E093DA12A091DA12A63010F00C948840C0
:10810600E1E01981088128960895E091DC12E030BB
:1081160011F00C949340E2E01981088128960895A5
:1081260000919D1210919E12002E012A11F00C94BE
:10813600A440E0E0E093DD12E3E01981088128968F
:108146000895E1E0E093DD120E94ACB50E94C3B54C
:10815600DE0115960E947E3AA5E3B4E080E090E049
:108166000E94799AE0E01981088128960895269759
:10817600A091DA12A63010F00C94C440E1E02696E5
:1081860008950E94CAB50E94C3B5DE0113960E94E7
:108196007E3AE0E0E093DD12A4E4B4E080E090E013
:1081A6000E94799AE0E0269608950E94DEB1003496
:1081B600E0E01E0710F00C94E640F8010E9489AE3C
:1081C6000F5F1F4FF4CFE0919B12AE81BF81EC93FE
:1081D600E091DA12AE81BF811196EC93E09185129F
:1081E600AE81BF811296EC9300918712109188128E
:1081F6000E94D3B5E0918312AE81BF811596EC93B0
:10820600E0918412AE81BF811696EC9300919D1287
:1082160010919E120E94E6B5E0919F12AE81BF8139
:108226005996EC93E091DC12AE81BF815A96EC939D
:10823600E091DD120E94EDB50031E0E01E0710F07E
:108246000C943741A1EAB2E1F8010E94E1B14D91E7
:108256005C910E94F6B54083452F55270E94F6B5DE
:1082660040830F5F1F4FE8CFE0E40E940BC22896C1
:108276000895E091D91208950E9438AD20E030E0CB
:10828600AD85BE85E0E00E94FAB5EFEFEC93AF81D5
:10829600B885E0E0EC93AD81BE81EC93E091D91214
:1082A600E03011F00C945C41E1E00E940CC22F9684
:1082B6000895E091D912E150E093D9120E9402B6D6
:1082C600E03011F40C94AF410E9402B6AD85BE8534
:1082D6000E940BB6EE53FD4EE081A985BA850E9439
:1082E6000BB6ED53FD4E4081AB85BC854C934031BA
:1082F60010F00C949D41A1EAB2E1E42FF0E00E9457
:10830600E1B10D911C9100240016010610F00C94A9
:108316008E41980107C0ABE8B2E1EE27A40FBE1F5D
:108326002C913327AF81B8852C93E32FF070AD8164
:10833600BE81EC930E9412B6EF53FD4EA0E0A083DF
:108346000E9412B6EE53FD4EA0E0A0830E9412B624
:10835600ED53FD4EA0E0A083E0E00E940CC22F96F4
:1083660008951A930A930A2F1A81A091D912A83058
:1083760010F40C94C341E1E0198108812396089515
:108386000E9412B6EF53FD4EA1E0A0830E9412B6E2
:10839600EE53FD4E00830E9412B6ED53FD4E108340
:1083A600E091D912EF5FE093D912E0E019810881DC
:1083B60023960895BA93AA93A2970E9404C24FEFF8
:1083C6005FEF3AA50E9418B6E8A5F9A50E943BAF53
:1083D600A32FBB270E94E71B00E0E02FF0E00E94DE
:1083E60056AFEC91E07F1E2FE02FF0E00E9456AFD3
:1083F600EC91EF702E2F103711F40C9407421038C1
:1084060011F40C94074201C0422F103711F00C945E
:108416001342E2E5F4E060E070E00E9422B60AC092
:10842600103811F00C941D42E1E6F4E060E070E0D3
:108436000E9422B6103911F40C942642103A11F417
:108446000C94264207C0522FAFE6B4E080E090E0DD
:108456000E94799A0F5F031710F00C943342BDCF38
:108466004A93A52F0E94B441E1E00E940BC2AB964D
:1084760008950A9300E00A3010F00C945342A3E0EA
:108486000A9FF001E250FD4E0E942AB5E150FD4ED2
:108496000E942AB5E050FD4EA0E0A0830F5FEBCF0F
:1084A600E0E0E0931C13E0931E13E0931D13E093AA
:1084B6002013E0931F1309910895A8970E9405C2FF
:1084C600E0911D13E03011F00C9482420E94933922
:1084D600E03011F40C9477420E942AB610F40C9402
:1084E60076420E9433B606C0E0E0E0931E13A5E193
:1084F6000E94DD0FE0E00E940CC2AD960895A091A7
:108506001D13A13011F00C949342E1E0EA93A8E028
:108516000E946B3AA5E10E94DD0F0E9433B687C127
:10852600A0911D13A23011F00C94A6420E942AB607
:1085360010F40C94A5420E9439B60E9433B6A5E108
:108546000E94DD0F74C1A0911D13A33011F00C948D
:10855600E0420E9442B6013011F40C94B742043056
:1085660011F40C94B74205C0E0E0E0931E130E949C
:1085760033B6A5E10E94F40F3E2F4F2F3536E0E0CB
:108586004E0710F40C94D6420E9447B6A63010F45B
:108596000C94D3420E944FB6E9ECE093E91203C073
:1085A600E1E0E0931D130E949339E03011F00C9442
:1085B600DF42E0E0E0931D133AC1A0911D13A43001
:1085C60011F00C94EE42E1E0EA93A9E00E946B3AC6
:1085D6000E9433B62CC1A0911D13A53011F00C9446
:1085E60067430E9442B6043011F00C945D430E942A
:1085F60058B6153010F00C9413430E9447B6AB30B2
:1086060010F40C940F430E944FB6EAECE093E91283
:10861600E0E0E0931D1303C0E4E0E0931D134AC0BD
:108626000E94A7B50E94E03AACE5B0E0ED810E9459
:10863600C8C3EEE5F0E0FF93EF93EE81EA93A885D9
:108646000E94B521AF91BF910E94C0C3E885AAE5FB
:10865600B0E00E94C8C3ABE5B0E0E9850E94C8C39C
:10866600E0E6F0E0FF93EF93EA85EA93AC850E949B
:10867600B521AF91BF910E94C0C320E0203110F018
:108686000C945343A2E6B0E0E22F0E9478B1E22FA9
:10869600E95F0E9446B4D0010E94C8C32F5FEECFA7
:1086A600A2E7B0E0E1E00E94C8C30E9433B6E1E071
:1086B600E093E9120E949339E03011F00C9466437E
:1086C600E0E0E0931D13B3C0A0911D13A63011F096
:1086D6000C94A543E0911F13E03011F40C948043F1
:1086E600E0912013E03011F00C948043A0911C130C
:1086F600A33010F00C94804301C003C0E7E0E09380
:108706001D13E0911F13E03011F40C949743E09190
:108716002013E03011F40C949743A0911C13A3305E
:1087260010F00C94974301C003C0E8E0E0931D13DA
:108736000E949339E03011F00C94A443E0E0E093FA
:108746001D1375C0A0911D13A73011F00C94E043C2
:10875600E0911F13E03011F00C94B443E6E0E0938F
:108766001D13E0912013E03011F40C94BD43E8E0B2
:10877600E0931D130E949339E03011F00C94C64328
:10878600E0E0E0931D13A0911C13AA3010F40C94A2
:10879600CF43E6E0E0931D130E9442B6043011F089
:1087A6000C94DF430E9458B6113010F40C94DF434A
:1087B6000E94A7B50E945DB63AC0A0911D13A830CD
:1087C60011F00C941A44E0911F13E03011F00C9450
:1087D600EF43E6E0E0931D13E0912013E03011F043
:1087E6000C94F843E7E0E0931D130E949339E030C0
:1087F60011F00C940144E0E0E0931D13A0911C13CA
:10880600AA3010F40C940A44E6E0E0931D130E948B
:1088160042B6043011F00C941A440E9458B6113036
:1088260010F40C941A440E94A7B50E945DB6E1E0CC
:108836000E940CC2AD9608950E9404C2AD01A4E741
:10884600B0E0EF81F8850E94C0C3A6E7B0E0EE81F4
:108856000E94C8C300E010E00031E0E01E0710F0FF
:108866000C944C44A8E7B0E0F8010E949DB50F01B6
:10887600F801DA010E9464B6D0010E94C0C321E06B
:1088860030E0E02FD9010E9448C29F010F5F1F4FC1
:10889600E3CFA2E7B0E0E1E00E94C8C30E94A2B520
:1088A60008950A930A2FA0911D13A63010F00C9478
:1088B6005F44E0E009910895003011F00C9468449B
:1088C6000E944FB6E0E0099108950E9439B6E1E0B2
:1088D6000991089526971A930A93A0911D13A6301D
:1088E60010F00C947B44E1E01981088128960895E4
:1088F600E0911F13E03011F00C948644E2E01981F8
:10890600088128960895A4E7B0E00E94A8C38F01C5
:10891600002E012A11F00C949844E0E0E093201315
:10892600E3E01981088128960895E1E0E093201399
:108936000E94ACB50E9468B6DE0115960E947E3A8A
:10894600E0E019810881289608952697A0911D13C5
:10895600A63010F00C94B244E1E0269608950E94E9
:10896600CAB50E9468B6DE0113960E947E3AE0E020
:10897600E0932013269608950E94DEB10034E0E0CD
:108986001E0710F00C94CD44F8010E9489AE0F5FCB
:108996001F4FF4CFA2E7B0E00E94ACC3AE81BF8107
:1089A600EC93E0911D13AE81BF811196EC93ACE57B
:1089B600B0E00E94ACC3AE81BF811296EC93AEE5E7
:1089C600B0E00E94A8C38F010E94D3B5AAE5B0E02B
:1089D6000E94ACC3AE81BF811596EC93ABE5B0E0C7
:1089E6000E94ACC3AE81BF811696EC9300E010E006
:1089F6000031E0E01E0710F00C941045F8013796A0
:108A06000E94B3AF0F01E2E6F0E0E00FF11FDF01D5
:108A16000E946FB60F5F1F4FEBCFA4E7B0E00E9436
:108A2600A8C38F010E94E6B5A6E7B0E00E94ACC3DA
:108A3600AE81BF815996EC93E0911F13AE81BF8141
:108A46005A96EC93E09120130E94EDB50031E0E0D8
:108A56001E0710F00C944245A8E7B0E0F8010E940A
:108A6600E1B10E94A8C3AF010E94F6B54083452F2D
:108A760055270E94F6B540830F5F1F4FE7CFA0E64C
:108A8600B0E00E94A8C30E9474B6AE81BF81DC9696
:108A9600EC930E947AB6AE81BF81DD96EC93E0E45A
:108AA6000E940BC228960895E0911C1308950E9417
:108AB600C4AEE0911C13E03011F00C947545AF85FF
:108AC600B889E0E0EC93AD85BE85EFEF0E94FAB57C
:108AD600E0E0EC93AF81B885EC93E1E00E940BC235
:108AE60061960895E0911C13E150E0931C130E94D7
:108AF6007FB6E250FD4EE081AF85B889EC930E94C7
:108B06007FB6E150FD4EE081AB85BC85EC930E94BB
:108B16007FB6E050FD4EE081EE83AD85BE85EC93D9
:108B2600AE81A03110F00C94BD45A8E7B0E0F0E0AE
:108B36000E94E1B10E94A8C38F010024001601061D
:108B460010F00C94A845980115C0A2E6B0E0EE819D
:108B5600F0E0AE0FBF1F0E94ACC32E2F3327AAE54D
:108B6600B0E00E94ACC34E2F5527FA01D9010E94EE
:108B7600BEC29F01A985BA852C93E32FF070AF8101
:108B8600B885EC930E947FB6E250FD4EA0E0A0832C
:108B96000E947FB6E150FD4EA0E0A0830E947FB602
:108BA600E050FD4EA0E0A083E0E00E940BC261967B
:108BB60008950E9485B6A0911C13AA3010F40C9457
:108BC600E945E1E00E940EC2259608950E947FB60F
:108BD600E250FD4E20830E947FB6E150FD4E008399
:108BE6000E947FB6E050FD4E1083E0911C13EF5FAC
:108BF600E0931C13E0E00E940EC225960895BA93F6
:108C0600AA93A3970E9404C210E02FEF30E040E041
:108C16005BA50E948BB60E9490B6E9A5FAA5FA93C9
:108C2600EA930E9496B6A52FBB270E94E71B00E099
:108C3600E02FF0E0DE011796AE0FBF1FEC91EE833A
:108C4600E07811F40C943046EE81E0774E2F429591
:108C56004F70EE81EF702E2F2DC0EE81E07411F46F
:108C66000C945046EE81E07FE03711F00C943D46BF
:108C760013E00FC0EE81E07FE03511F00C9445461D
:108C860012E007C0EE81E07FE03411F00C944C4610
:108C960011E0EE81EF702E2F0DC0EE81E07211F41F
:108CA6000C94564607C0EE81E07111F40C945C46B4
:108CB60001C03E810F5F051710F00C946C46103012
:108CC60011F40C946B46303011F40C946B4601C0D1
:108CD60001C001C0ADCF1A932A93A32F0E94DC4591
:108CE600E1E00E940BC2AC9608950895E0E0089575
:108CF6000E949BB60E94D614A1E00E94FA27A0E02B
:108D06000E941A2808950E9496B20E94D14C0E9491
:108D160096B20E94F4460E9496B2A5E00E94194BB4
:108D26000E9496B2A5E00E942B4B0E9496B2EDE0FF
:108D3600EA93E4E0EA93A2E0B0E080E090E00E94EB
:108D4600A0B6EDE0EA93E9E00E94A3B6EEE0EA936E
:108D5600E3E00E94A3B6E2E1EA93E3E0EA93A6E940
:108D6600B0E080E090E00E944E4BE6E9F0E0E09350
:108D76003013F09331130E9496B2E2E1EA93E7E1F1
:108D8600EA93AEE1B0E080E090E00E94A0B6E2E1B6
:108D9600EA93E7E2EA93A8EEB3E080E090E00E946F
:108DA600A0B6E2E1EA93E8E2EA93A4E6B0E080E066
:108DB60090E00E94A0B6E8E0EA93AAE00E947A4713
:108DC6000E9496B2A0E00E94CD470E9496B2A0E013
:108DD6000E94B5470E9496B2A4E6B0E00E94674D95
:108DE60008950E94A9B60E94B4B60E94BAB6E1E4FC
:108DF600EC930E94BFB6E0E00E94C2B6A2E0B0E0EB
:108E06000E9465160881659608950E947B46A1E238
:108E16000E947515A1E00E942C2EA8ECB0E00E94DD
:108E2600650F0E945328E03011F40C941E470E94EF
:108E360086460E94F4460895A0E00E942C2E0895CE
:108E460026970A930A2F033011F00C943947ADE0A8
:108E56000E947515AAE00E947515AAE00E94751574
:108E6600AAE00E947515AAE00E947515EBE1E98358
:108E7600E3E4EA83013011F40C944647033011F41D
:108E86000C94464703C0E0E0EB8306C0023011F0C5
:108E96000C944F47E1E0EB83E0E0EC830E94C8B618
:108EA6000E94CDB608812796089564970E94C2B1A4
:108EB6000E94D1B60E94E4B6E6E40E94E9B6E0E07C
:108EC600EC930E943BB40E94FDB6089564970E94FD
:108ED600C2B10E94D1B60E94E4B6ECE50E94E9B6A2
:108EE600E0E0EC930E943BB40E94FDB608956497BF
:108EF6000E9407C21A2F2F8900E02F3110F40C941C
:108F0600854720E0163010F40C948E47153110F08A
:108F16000C948E4701C01AE00E9405B70E94B4B6B1
:108F26000E940DB7E0E5EC930E9405B7EFEF0E94B3
:108F360012B7DE0113960E9417B7DE011396EA0FE9
:108F4600FB1F10830E941EB70E9421B7A5E0B0E068
:108F56000E94651620932113109322130E940EC2BD
:108F6600689608950E9428B7153010F40C94BC47F3
:108F760010E00E942EB70E9436B7E7E50E9412B7AE
:108F86000E943BB70E9441B71093231319810881B1
:108F9600669608950E9428B7183010F40C94D447AA
:108FA60010E00E942EB70E9436B7E8E40E9412B77E
:108FB6000E943BB70E9441B7109324131981088180
:108FC600669608950E9428B70E942EB70E9436B76B
:108FD600E9E50E9412B70E943BB70E9441B7109381
:108FE600251319810881669608950E9428B71230C4
:108FF60010F40C94FF4710E00E942EB70E9436B77B
:10900600EAE40E9412B70E943BB70E9441B7109350
:10901600261319810881669608950E9428B7123092
:1090260010F40C94174810E00E942EB70E9436B731
:10903600ECE40E9412B70E943BB70E9441B710931E
:10904600271319810881669608950E9428B7123061
:1090560010F40C942F4810E00E942EB70E9436B7E9
:10906600E9E40E9412B70E943BB70E9441B71093F1
:10907600281319810881669608950E9428B71C3620
:1090860011F40C945B48133611F40C945B481237B8
:1090960011F40C945B481C3411F40C945B481334A3
:1090A60011F40C945B48123511F40C945B4801C022
:1090B60001C01CE60E942EB70E9436B7E9E60E9460
:1090C60012B70E943BB70E9441B71093291319812A
:1090D6000881669608950E9428B70E942EB70E94BE
:1090E60036B7E3E20E9412B70E943BB70E9441B72F
:1090F60019810881669608950E9428B70E942EB7A6
:109106000E9436B7EDE60E9412B70E943BB70E9456
:1091160041B71981088166960895AA93EF976997D2
:109126000E9404C224E630E040E0FE01E25AFF4F0E
:109136005081FE01B896FA93EA930E9490B60E9477
:1091460018B65F3110F40C94A9485EE100E00517EB
:1091560010F00C94BA480E944AB70E944FB7E02F0D
:10916600F0E0DE0116960E944FB70F5FF0CFDE01EA
:10917600AE59BF4FAC91A03011F00C94C9480E9473
:109186005FB7A13011F00C94C94801C001C012E4C8
:109196000E9464B7A03011F00C94D8480E945FB7C3
:1091A600A03011F00C94D84801C001C012E60E940C
:1091B60064B7A13011F00C94E7480E945FB7A13064
:1091C60011F00C94E74801C001C013E40E9464B793
:1091D600A13011F00C94F6480E945FB7A03011F050
:1091E6000C94F64801C001C013E60E9464B7A23091
:1091F60011F00C9405490E945FB7A13011F00C9450
:10920600054901C001C014E40E9464B7A23011F000
:109216000C9414490E945FB7A03011F00C941449C5
:1092260001C001C014E60E9464B7A33011F00C948B
:1092360023490E945FB7A13011F00C94234901C065
:1092460001C019E40E9464B7A33011F00C943249AE
:109256000E945FB7A03011F00C94324901C001C0E2
:1092660019E60E9464B7A43011F00C9441490E949B
:109276005FB7A13011F00C94414901C001C015E55A
:109286000E9464B7A43011F00C9450490E945FB755
:10929600A03011F00C94504901C001C015E70E949E
:1092A60064B7A53011F00C945F490E945FB7A130F6
:1092B60011F00C945F4901C001C016E50E9464B725
:1092C600A53011F00C946E490E945FB7A03011F0E2
:1092D6000C946E4901C001C016E7123411F40C94C7
:1092E6007949123611F40C9479491AC000E0051731
:1092F60010F00C9484490E9469B70E946FB70F5F03
:10930600F6CFEAE2EE830E9473B7EAE2EC93E52F2A
:10931600EE5FF0E00E9456AFE0E0EC935E5FAAC01D
:10932600133411F40C949C49133611F40C949C4993
:109336000CC0E52FF0E00E9456AFEFEFEC930E94D1
:1093460073B7E0E0EC935F5F95C0143411F40C94AE
:10935600B149143611F40C94B1491AC00E9418B6DA
:109366000E9478B70E947FB75CE000E0051710F016
:109376000C94CA490E944AB70E9483B711F40C9410
:10938600C8490E9469B70E946FB70F5FEFCF72C0DE
:10939600193411F40C94D449193611F40C94D449A7
:1093A60029C00E9478B70E9486B700E0051710F022
:1093B6000C94EA490E944AB70E9483B711F40C94B0
:1093C600E8490E9469B70E946FB70F5FEFCFE0E0F0
:1093D600EE835F5F50FF08C0E52FF0E00E9456AFB6
:1093E600EFEFEC935F5F05C00E9473B7EFEFEC936E
:1093F6005E5F40C0153511F40C94064A153711F41A
:109406000C94064A13C00E9418B60E9478B70E94B0
:109416007FB700E0051710F00C94174A0E9469B751
:109426000E946FB70F5FF6CF5CE024C0163511F4CB
:109436000C94224A163711F40C94224A1BC00E943F
:1094460018B60E9478B7A7E0B0E00E94D41C57E097
:1094560000E0051710F00C943D4A0E944AB70E949E
:1094660083B711F40C943B4A0E9469B70E946FB708
:109476000F5FEFCF0E948AB70E948FB70E94B4B6E3
:109486000E948FB7E3E60E9412B70E9495B7108339
:10949600E02F0F5FF0E0DE01A65BBF4F0E9417B71B
:1094A6000E9495B73083E02F0F5FF0E00E9495B7DA
:1094B6004083E02FF0E00E948FB7E0E0EC93FE01DE
:1094C600E65BFF4FFA93EA93A6E0B0E00E946516CA
:1094D6000E949BB7A52FBB270E9465160E940BC250
:1094E600EF96A496089564970E942EAD00E00E9420
:1094F60005B70E94B4B60E940DB7E3E6EC930E944E
:1095060005B7EDEFEC93012E022A11F00C94934A65
:10951600E02F0F5FF0E0DE0113960E9424AF04C037
:109526000E9405B7E1E3EC930E941EB70E9421B7A3
:10953600A4E0B0E00E9465160E940EC267960895E8
:1095460064970E942EAD00E00E9405B7ECE0EC9314
:109556000E941EB70E9421B7A1E0B0E00E946516E6
:109566000E940EC2679608951A930A931A2F00E076
:10957600011710F00C94C44AAAE00E9475150F5FFB
:10958600F7CF0991199108950E94A0B7AAE00E9409
:1095960075150E940DC2249608950E94A0B70E94D8
:1095A6000DC2249608950E949CC30E948DC30E94FA
:1095B600981624960895EF97EF9724970A9300E05C
:1095C600023810F00C94ED4A0E94BFB6E0E0EC932E
:1095D6000F5FF6CF00E0013610F00C94F94A0E94B6
:1095E600BFB6E02FE05EEC930F5FF5CF0E94C8B6E2
:1095F600A0E6B0E00E94651600E0003810F00C947A
:109606000B4B0E94BFB6E02FE058EC930F5FF5CFEF
:109616000E94C8B6A0E8B0E00E946516AAE00E94C3
:1096260075150881EF96EF9625960895AA930A93E5
:10963600E981EE0FEE0FEE0F0E2FE1E1EA93E4E083
:10964600EA930E94ABB70E944E4B0881229608957A
:10965600AA932497E0ECE883E1E0E9830E9422B52F
:109666000A93ED81EE0FEE0FEE0F0E2F0E94B0B7AC
:109676000E9425C2A983BA838B839C83E1E1EA9386
:10968600E5E0EA93AB81BC818D819E810E944E4BC1
:109696000881269608950E949CC3AF970E94B8B78A
:1096A6000E9422B50E9404C200E020E0EDA9FEA9B6
:1096B6006FA978AD0E94BCB7ADA9BEA98FA998AD18
:1096C600A935EEE3BE07EFE08E07E0E09E0710F453
:1096D6000C94724BE1E00E940BC2EB9608951AAD12
:1096E600A12FE4E60E94F6C23E2F0E94C1B74E2F7C
:1096F6000E949EB05E2F305D405D505D19ADA12F7A
:10970600E4E60E94F6C2EE8B0E94C1B7ED8B0E9482
:109716009EB0EC8BEE89E05DEE8BED89E05DED8B26
:10972600EC89E05DEC8B0E9412B10E9482AD0E9432
:109736001CC3EB8B0E9412B10E9482AD0E94C7B778
:10974600E0E1F7E260E070E00E941CC3EA8B0E9451
:10975600D0B7E0E1F7E260E070E00E94D5B7E8EE4E
:10976600F3E060E070E00E941CC3E98B0E9412B136
:10977600E8EEF3E060E070E00E94C7B7E4E6F0E0F0
:1097860060E070E00E941CC3E88B0E94D0B7E4E65C
:10979600F0E060E070E00E94D5B70E94DAB70E9460
:1097A6001CC3EF870E9412B10E94DFB7EE87EB89D8
:1097B600E05DEB8BEA89E05DEA8BE989E05DE98BA8
:1097C600E889E05DE88BEF85E05DEF87EE85E05D9B
:1097D600EE870E94E4B7AE0FBF1FEEE10E9412B7FC
:1097E6000E94EAB7EBE50E9412B70E94EAB7E2E3ED
:1097F6000E9412B70E94EAB7EAE3EC93313310F401
:109806000C940A4C0E94E4B7EA0FFB1F30834133E5
:1098160010F00C94134C313310F00C94134C05C01B
:109826000E94E4B7EA0FFB1F40830E94E4B7EA0FE9
:10983600FB1F50830E94E4B70E941FAFAE89A1337D
:1098460010F40C942C4C0E94E4B7EA0FFB1FAE896F
:10985600A083AD89A13310F00C94374CAE89A133A7
:1098660010F00C94374C06C00E94E4B7EA0FFB1FB9
:10987600AD89A0830E94E4B7EA0FFB1FAC89A083E1
:109886000E94E4B7AE0FBF1FEAE3EC93AB89A133A6
:1098960010F40C94544C0E94E4B7EA0FFB1FAB89FA
:1098A600A083AA89A13310F00C945F4CAB89A13335
:1098B60010F00C945F4C06C00E94E4B7EA0FFB1F41
:1098C600AA89A083A989A13310F00C94754CAA89A2
:1098D600A13310F00C94754CAB89A13310F00C94A5
:1098E600754C06C00E94E4B7EA0FFB1FA989A08346
:1098F600A889A13310F00C94904CA989A13310F0DB
:109906000C94904CAA89A13310F00C94904CAB891E
:10991600A13310F00C94904C06C00E94E4B7EA0FF5
:10992600FB1FA889A083AF85A13310F00C94B04C1F
:10993600A889A13310F00C94B04CA989A13310F07A
:109946000C94B04CAA89A13310F00C94B04CAB899E
:10995600A13310F00C94B04C06C00E94E4B7EA0F95
:10996600FB1FAF85A0830E94E4B7EA0FFB1FAE85FD
:10997600A0830E94E4B7AE0FBF1FEDE5EC93E02F86
:10998600F0E00E94EAB7E0E0EC93FE0177960E94D1
:10999600EFB7E0E00E940BC2EB9608950E94A9B6CD
:1099A600EEE10E9412B70E94BAB6EBE50E9412B72A
:1099B6000E94BAB6E6E30E9412B70E94BAB6EAE37C
:1099C6000E9412B70E94F5B70E94F9B7E02F0F5F09
:1099D600F0E00E94F5B70E9400B8EAE30E9412B7D1
:1099E6000E94F5B70E9400B8EDE50E94C2B6A02F0E
:1099F600BB270E9465160E948AB70E94BAB6EEE19E
:109A06000E9412B70E94BAB6EBE50E9412B70E94F6
:109A1600BAB6E9E30E9412B70E94BAB6EAE30E9418
:109A260012B70E94F5B70E94F9B7E02F0F5FF0E07A
:109A36000E94F5B70E9400B8EAE30E9412B70E949E
:109A4600F5B70E9400B8EDE50E94C2B6A02FBB276D
:109A56000E94651608816596089564970E9404C25F
:109A66002A2F3A8D4B8D5C8D00E015E0E02F0F5FBD
:109A7600F0E00E9456AF0E94B4B60E9404B850832C
:109A86000E9409B840830E9409B830830E9409B831
:109A96002083403011F00C94524D12E00BC0303050
:109AA60011F00C94584D13E005C0203011F00C94C1
:109AB6005D4D14E00E949BB7A12FBB270E9465163F
:109AC6000E940BC26D9608951A930A938D01053074
:109AD600E0E01E0710F40C94774D0B3FE0E01E0704
:109AE60010F00C94774D01C00DC0E2E1EA93E3E07B
:109AF600EA93D801882799270E944E4B009330138A
:109B0600109331130991199108956C970E9404C21C
:109B160000E030E010E00E948215E0E0E0932F13B1
:109B26000E948AB70E940DB80E94B4B60E940DB872
:109B3600EBE6EC93E02FF0E00E940DB8E0E0EC934A
:109B4600FE013E960E94EFB7ADE00E94DD0F00E0F9
:109B56000E9457160E2FADE00E94F40FAF010030A1
:109B660011F00C94BD4D4436E0E05E0710F00C9405
:109B7600BD4D01C001C0ECCF003011F00C94CA4DB0
:109B8600E0E4E0932F130E940BC2A29608950E9470
:109B96000316EE83FF83AE81BF81199714F40C94EC
:109BA600D64D0E9412B8AE81BF81119714F40C9461
:109BB600E34DAE81BF81199714F00C94E34D06C0B6
:109BC6001F5F1E3110F00C94E94D01C001C0A3CFF8
:109BD600AE81BF81119714F00C94FA4D0E94821544
:109BE600E0E8E0932F130E940BC2A2960895FE01AF
:109BF6003E960E9416B80E941BB8FE013E96FA9346
:109C0600EA93A4E1B0E00E94281600E0063010F0C6
:109C16000C94154EE02FF0E0DE0118960E941FB856
:109C26000F5FF4CFAE81BF81169714F40C941F4ECC
:109C3600E5E0F0E0EE83FF8300E0EE81FF81A02FF8
:109C4600B0E0AE17BF0714F00C945C4EE02FF0E0C6
:109C56000E940DB82C91E22FE07F1E2F17FF03C044
:109C660016FD01C001C004C0E22FEF73E8871FC0D4
:109C7600103C11F00C94434EE22FEF70E98717C0A9
:109C8600103D11F00C944B4EE22FEF70EA870FC097
:109C9600103E11F00C94534EE22FEF70EB8707C085
:109CA600103F11F00C945A4EE22FEF70EC870F5FC5
:109CB600C4CF00E0053010F00C946E4EAAE2B3E17A
:109CC600E02F0E9478B1E12FF0E0DE0118960E94A5
:109CD600A4AF0F5FEFCF388530FF02C03E7F01C0D3
:109CE6003160E32F0E940BC2A29608950E942EAD0A
:109CF60000E00E9424B8A0912A13A0830E9424B8F1
:109D0600A0912B13A0830E9424B8A0912C13A083AA
:109D16000E9424B8A0912D13A0830E9424B8A0917C
:109D26002E13A0830E9424B8A0912F13A0830E9413
:109D360033AD08950E9404C2AD0100E00E942AB826
:109D4600A0912113A0830E942AB8A0912213A08378
:109D56000E942AB8A0912413A0830E942AB8A09139
:109D66002313A0830E942AB8A0912613A0830E94E1
:109D76002AB8A0912813A0830E942AB8A09127137D
:109D8600A0830E942AB8A0912513A08320913013A6
:109D960030913113122F232F33270E942AB82083A4
:109DA6000E942AB810830E942AB8A0912913A08382
:109DB600E02F0E940BC226960895A1E00E9417513B
:109DC600E0E0E093351308950895BA93AA93A09717
:109DD6000E9404C2E0E0EE83AE81A73010F00C943E
:109DE600FE4EEE81AEA1BFA1F0E00E941FB8EE814B
:109DF600EF5FEE83F1CFE0E0EE83AE81AA3010F0A4
:109E06000C940F4FEE81F0E0DE0117960E941FB80A
:109E1600EE81EF5FEE83F1CF0E9430B8E8E00E945A
:109E260035B8DE0157960E94AB122E2F213010F462
:109E36000C94204F0E943BB80895EA89E07811F00F
:109E46000C94384FEA89EA8FE068EA8F0E9430B8AE
:109E5600E1E00E9435B80E9440B810F40C94364FE9
:109E66000E943BB808950E946DB3ED89E07211F02F
:109E76000C943F4FED89ED8FED89E07111F40C9450
:109E8600564FED89ED8FDE015D96EC91EF7E0E94D7
:109E960047B80E9440B810F40C94544F0E943BB847
:109EA60008950E946DB3ED89E87011F00C946D4F22
:109EB600ED89ED8FDE015D96EC91E8600E9447B872
:109EC6000E9440B810F40C946B4F0E943BB8089562
:109ED6000E946DB3EC89E07411F40C94844FEC8904
:109EE600EA8FEF7BEA8FE2E0F0E00E944EB80E9434
:109EF60040B810F40C94824F0E943BB808950E941B
:109F06006DB3EA89E0933213EB89E0933313EC895E
:109F1600E0933413ED89E0933513E7703E2F31302B
:109F260010F40C949B4F383010F00C949B4F01C0EA
:109F360001C03F83ED89E0933513EC89EF730E94EE
:109F460052B82E2F0B89A02F0E9469211E2F1C3379
:109F560010F00C94B14FFE0138961083EA89EF7722
:109F66000E9452B81E2F1C3310F00C94BD4FFE01F8
:109F760039961083283110F00C94C44FFE013A969E
:109F86002083EF89EF710E9452B85E2FEE89EF733E
:109F96000E9452B8E98BA88D0E9469214E2FFE01BE
:109FA6003B964083FE013C965083E989ED87AB855D
:109FB600A43610F40C94E44FE2E00E940BC2A8967B
:109FC6000895AC85AD3010F00C94EE4FA03011F42E
:109FD6000C94EE4F05C0E3E00E940BC2A8960895CC
:109FE600AD85A03210F00C94FD4FA03011F40C9406
:109FF600FD4F05C0E4E00E940BC2A8960895AA850D
:10A00600A83110F40C940C50E5E00E940BC2A896FF
:10A016000895A885AC3310F40C941650E6E00E941F
:10A026000BC2A8960895AF81A83010F40C94205066
:10A03600E7E00E940BC2A8960895E0E0EE83AE81A9
:10A04600A73010F00C943650EE81AEA1BFA10E944D
:10A0560078B1EE81F0E0DE0117960E94A4AFEE81A2
:10A06600EF5FEE83ECCFE0E00E940BC2A896089566
:10A0760029970E9404C22A2F3F8548895989583159
:10A0860011F00C94475050E0583110F40C944E5097
:10A096000E9456B808954C3311F00C94535040E08A
:10A0A6004C3310F40C945A500E9456B808953C3321
:10A0B60010F40C945F5030E0E0913513E862E093C1
:10A0C6003513EF7EE0933513E32FE068EE83E091DE
:10A0D6003313EF83E0913413E887E0913513E98772
:10A0E600E0E0EA87EB87EC87ED87503011F00C94BF
:10A0F6008150403011F00C94815009C0583110F055
:10A106000C948A504C3310F00C948A5001C00CC049
:10A11600A32F0E947A21EE83A42F0E947A21EF8337
:10A12600A52F0E947A21E887213010F40C94A050C4
:10A13600283010F00C94A05001C007C010913513C0
:10A14600187F122BFE0139961083EE81E068EE83AC
:10A15600DE011996EC91E862EC930E9430B8E4E0D7
:10A166000E9435B80E945BB80E9496B2003011F486
:10A176000C94C0500E9456B80895E0E00E940BC2AD
:10A186006296089524970E9406C21A2F288539855B
:10A19600203011F40C94D4502D3010F00C94D4507F
:10A1A60003C00E9461B80895103011F40C94E05079
:10A1B600103210F00C94E05003C00E9461B808956C
:10A1C600343110F40C94EC50333310F00C94EC5002
:10A1D60001C037E1A12F0E947A21EC83A22F0E94B1
:10A1E6007A21ED83A32F0E947A21EE83E0E0EF83AC
:10A1F6000E9466B8E4E0F0E0FA93EA93E3E00E9496
:10A2060035B8DE0119960E94DB110E2F0E9466B842
:10A21600003011F40C9412510E9461B80895E0E0E8
:10A226000E940DC22A96089522970E9407C22A2FDD
:10A23600022FE02FE03011F00C942451E0E0EB8384
:10A246000DC0E13011F00C942B51E0E4EB8306C015
:10A25600E23011F00C943151E4E4EB83E0E0EC835E
:10A26600E7E0F0E00E944EB8DE0118960E94DB118E
:10A276001E2F103011F40C944551E1E00E940EC2DD
:10A2860025960895E0E00E940EC22596089522972D
:10A296000A93E7E0F0E00E944EB8DE0116960E94AF
:10A2A600AB120E2F003011F00C945D51E98108813C
:10A2B60023960895EFEF0881239608950881239643
:10A2C60008952C970E9406C29D010E946AB8ACE0D0
:10A2D6000E9440B4E0E3EA930E946DB80E9471B810
:10A2E600DE0119960E947CB810F40C947F51E1E0CF
:10A2F6000E940DC26096089510E0183010F00C947C
:10A306008D510E9481B8F0E0DE0114960E94A4AF40
:10A316001F5FF3CFE0E00E940DC260960895689734
:10A326000E9404C29D014E8D5F8D05C0E2E00E9431
:10A336000BC2A0960895FE0172960E9416B80E945E
:10A346007FB75A934A93E0E3EA93A0E10E9440B4B0
:10A35600E0E3EA930E941BB80E9471B8DE015796AB
:10A366000E947CB810F40C94BD51E1E00E940BC22F
:10A37600A0960895E98D0E9488B8DA011F96EC939D
:10A38600EE85DA011E96EC93E88D0E9488B8DA0114
:10A396001D96EC93EE85DA011C96EC93EF890E94EC
:10A3A60088B8DA011B96EC93EE85DA011A96EC93DF
:10A3B600EE890E9488B8DA011996EC93EE85DA01E7
:10A3C6001896EC93ED890E9488B8DA011796EC93FB
:10A3D600EE85DA011696EC93EC890E9488B8DA01CC
:10A3E6001596EC93EE85DA011496EC93EB890E94B0
:10A3F60088B8DA011396EC93EE85DA011296EC939F
:10A40600EA890E9488B8DA011196EC93EE85DA01A2
:10A41600EC93EE89FF27662777270E9493B8EF898A
:10A426000E949BB8E88D0E949BB8E98DFF2766279E
:10A4360077270E9412B10E942AC20E94BCB7EA89FD
:10A44600FF27662777270E94A3B8EB890E94ACB83E
:10A45600EC890E94ACB8ED89FF27662777270E9412
:10A46600D0B70E942AC20E9443B00E9453B03A93CA
:10A476002A930E94B4B80E941CB10E9497C3FE01A1
:10A486007696FA93EA930E94B4B813E11A3010F460
:10A496000C9457520E9481B8EA50F0E0DE015296C1
:10A4A6000E94A4AF1150F2CF10E0143110F00C94BA
:10A4B60069520E9432AEEC91E03011F00C94675272
:10A4C6000E9432AEE0E3EC931F5FEFCFE0E00E9424
:10A4D6000BC2A09608952E970A93DE0115960E9448
:10A4E600E84E0E2F003011F40C947C5208812F9602
:10A4F6000895E885E093D011EE81E093D111EF81C4
:10A50600E093D211E985E093CC11EA85E093CD1171
:10A51600EB85E093CE11ED81E093CF11A3EDB1E190
:10A52600E091D011F0E0ED93FC93A091D311B0919E
:10A53600D411ECE30E94E6C2E093D311F093D41158
:10A54600A091D311B091D411E091D111F0E0EA0FAE
:10A55600FB1FE093D311F093D411E091D311F09146
:10A56600D411662777270E94BDB80E94A6B10E9423
:10A5760087ADE091D2110E94B0B70E9420C20E941E
:10A58600BDB8E093D511F093D6116093D7117093AF
:10A59600D811E0E008812F960895E0E0E0933613A5
:10A5A60008951A930A93E3E0EA93A3E0B0E00E94C9
:10A5B600A40CA1E00E947F27A8E0B0E00E9471C52C
:10A5C600E1E0E0933813E0E0E09337130E94C1B86E
:10A5D60000E0053010F00C94035310E0123010F038
:10A5E6000C940153AAE01A9FF001E359FC4EDF01D7
:10A5F6000E94C8B80E9487B41F5FF0CF0F5FE9CFF3
:10A60600EAE0F0E0E0933913F0933A13A09139139E
:10A61600B0913A13E2E00E94E6C2E0933913F09358
:10A626003A13E0E0E0933B13E0933C130991199150
:10A6360008950E94CBB811F40C9424530E94D0B80C
:10A6460008950E948B27E03011F00C943053A1E05E
:10A656000E947F27A3E00E94DD0FA3E00E94F40F73
:10A666008F010630E0E01E0710F40C9472530E942E
:10A67600090D9F0144E0413010F40C9455530E949B
:10A68600D5B8DF01E42F0E94F3B1BF010E94D5B80F
:10A69600DF01E42FE1500E9426B5DB01ED93FC9328
:10A6A6004150E9CF0E94D5B820833183E09137131A
:10A6B600EF5FE0933713A0913713A23010F40C9498
:10A6C6006753E0E0E09337130E94C1B80E94DDB8FB
:10A6D60010F40C947253ABE3B3E10E9450AD0E94A8
:10A6E60079530E94A8530E94D0B808950E9407C2C9
:10A6F6000E948B27E03011F00C9483530E94E8B837
:10A706000E94DDB810F40C948E53E0EEFEE20E9437
:10A716000EC22396089500E010E020E0253010F0E8
:10A726000C949D53A7E7B3E10E94EFB80E94D5B4FD
:10A736002F5FF4CF0E94F2B80E94F9B8009351132C
:10A74600109352130E94FAAC08950E9405C20E940B
:10A756008B27E03011F00C94B2530E94E8B80E94A7
:10A76600DDB810F40C94C153ECE8F0E0E093531319
:10A77600F09354130E940CC22596089500E010E051
:10A7860040E0453010F00C94D253E42FADE6B3E12F
:10A79600F0E00E94E1B10E94D5B44F5FF2CF0E9473
:10A7A600F2B8D8010E947F889F01209353133093FB
:10A7B60054130E940CC2259608950E9406C23A2F91
:10A7C600323010F40C94ED53E0E0F0E00E940DC23C
:10A7D6002496089500E010E020E0253010F00C9457
:10A7E6000054AAE03A9FF001E359FC4EDF010E94B3
:10A7F600EFB80E94D5B42F5FF0CF0E94F2B8F801EF
:10A806000E940DC2249608950E9406C2A1E00E94ED
:10A816007F27A0E00E9408B9D8010E947F889F0187
:10A826000E940DC2249608951A930A93A1E00E94ED
:10A836007F27A1E00E9408B90E94F9B8F8010991A2
:10A84600199108951A930A930E9412B9E1E0E093D0
:10A856004C13E0E0E093901400E010E00530E0E0F7
:10A866001E0714F00C943E54ABE8B4E10E9445AECA
:10A876000F5F1F4FF3CF0E94B665E0E0E0938A14A6
:10A88600A3E10E942310A1E20E94DD0FE0E0E09325
:10A896008914E0934813E0934713E0934B1309910F
:10A8A6001991089524970E9405C200E010E00E94C5
:10A8B600718DE03011F40C946754A1E8B4E10E9464
:10A8C6004E8D1E2F10934613A0919014AF5FA09348
:10A8D6009014A53010F40C947354E0E0E0939014B7
:10A8E600E0919014F0E0E557FB4EFF93EF930E9442
:10A8F6007165AF91BF91EC93EBE8F4E10E9418B952
:10A9060011F40C94A65400918B140093481300FF85
:10A9160004C0E1E0E0933D1303C0E0E0E0933D13A3
:10A9260001FF04C0E1E0E0933E1303C0E0E0E093E2
:10A936003E1302FF04C0E1E0E0933F1303C0E0E0F2
:10A94600E0933F1301C003E6E0919014F0E0EF5668
:10A95600FB4EFF93EF930E94EF64AF91BF91EC9390
:10A96600E1E9F4E10E9418B911F40C94CD54409138
:10A976009114E0919114E0934B13403011F40C9430
:10A98600CA54E1E0E093EE12E0934C1303C0E8EC06
:10A99600E093EE120E94B9652E2F203011F40C942C
:10A9A6000455E0E0E0938A14113011F40C94E0545D
:10A9B600123011F40C94E0540AC00E94B6650E944D
:10A9C600908D003011F40C94EA540E9412B90030B4
:10A9D60011F40C94F254A3E20E94DD0F0DC0A3E221
:10A9E6000E94F40F0E9420B9A83EE3E0BE0710F4CF
:10A9F6000C94FF540E94B665E1E00E940CC22996B1
:10AA06000895113011F00C940C55A1E00E9425B95F
:10AA160007C0123011F00C941355A0E00E9425B91E
:10AA2600033610F00C941C55013010F40C941C5590
:10AA360001C005C0E02FE853E093F3121CC00030BC
:10AA460011F00C943E55E1E0E093F312E0E0E09360
:10AA56004913E0934A13E0938A14AFE00E943F1033
:10AA6600ED83FE83AD81BE815F9710F40C943E5555
:10AA7600E0E0E0934713033610F00C944E55E02FB8
:10AA8600E57011F40C944E55A0914913A03011F0C5
:10AA96000C944E5501C01AC0E1E0E09349130E94A0
:10AAA6009865113011F40C945F55E0914713E0302E
:10AAB60011F00C945F5501C003C00E94A26502C04C
:10AAC6000E94B6650E94908D0E94BFA9033610F0C1
:10AAD6000C94765501FF07C0A0914A13A03011F0DF
:10AAE6000C94765501C01DC0E1E0E0934A130E9424
:10AAF6009865123011F40C948755E0914713E030B5
:10AB060011F00C94875501C003C00E94A26505C0D0
:10AB16000E94B665E1E0E0938A140E94908D0E943F
:10AB2600BFA9A0918A14A13011F00C94A755A09149
:10AB36004C13A13010F40C94A755A0914B13A030E0
:10AB460011F00C94A75501C007C0E0918A14EF5F7D
:10AB5600E0938A140E940BAAA0918A14A23011F0E5
:10AB66000C94B555013010F40C94BE55E1E00E94EA
:10AB76000CC229960895E0E00E940CC22996089519
:10AB8600E0918A140895EAE7F4E060E070E00E943C
:10AB960097C3A6E9B4E10E94041DE3E8F4E060E08F
:10ABA60070E00E9497C3AEE9B4E10E94041DECE890
:10ABB600F4E060E070E00E9497C3A6EAB4E10E9468
:10ABC600041DE5E9F4E060E070E00E9497C3AEEA98
:10ABD600B4E10E94041DEEE9F4E060E070E00E943A
:10ABE60097C3A6EBB4E10E94041DE7EAF4E060E037
:10ABF60070E00E9497C3AEEBB4E10E94041DE0EB47
:10AC0600F4E060E070E00E9497C3A6ECB4E10E9415
:10AC1600041DE9EBF4E060E070E00E9497C3AEEC3F
:10AC2600B4E10E94041D08951A930A93A091E514B5
:10AC3600A33010F40C942856A5E20E942FB910F404
:10AC46000C942856E0E0E093E514A091E514A230B8
:10AC560011F00C943356A5E20E94DD0F0E9436B91E
:10AC6600A091E514A13010F40C943D56E1E0099151
:10AC760019910895E0E00991199108950A93E1E088
:10AC8600E093E5140E9478460E9408470E9412B895
:10AC96000E94884D0E2F0E945328E03011F00C942C
:10ACA60055560062003011F00C945D56E1E0E093D9
:10ACB600E4121DC0E02FE07E11F40C946656E8EC19
:10ACC600E093E41214C0E02FEC7111F40C946F566B
:10ACD600E9ECE093E4120BC001FF04C0EAECE09358
:10ACE600E41205C000FF03C0E4E6E093E4120E940C
:10ACF60036B9E02F09910895EF97EF97A297E1E013
:10AD0600E093E5140E9469B30E9486460E9469B3E7
:10AD16000E943DB9A2ECB4E080E090E00E94D64AE1
:10AD2600A3EDB4E080E090E00E94D64AA4EEB4E041
:10AD360080E090E00E9446B90E9469B3A2E00E94BA
:10AD4600B547A3E00E94CD47A5EFB4E080E090E0D0
:10AD56000E94D64A0E943DB9A1E00E946E480E9418
:10AD660069B3A2E00E94B547A2E00E94CD47ABEFCF
:10AD7600B4E080E090E00E94D64A0E943DB90E946D
:10AD860069B3A1E00E94B74A0E944BB9A4E0B5E0BE
:10AD960080E090E00E94D64AE1E1F5E060E070E0F4
:10ADA6000E94A6B20E9451B9FE013296FA93EA9326
:10ADB600A4E10E9490480E9469B3A1E00E94B74AAC
:10ADC6000E9458B9A0E00E94B547A0E00E94CD4776
:10ADD600ADE3B5E080E090E00E94D64A0E944BB910
:10ADE600A6E5B5E080E090E00E94D64AA2E00E9487
:10ADF600CD47A2E6B5E080E090E00E94D64A0E94E8
:10AE06004BB9A1E00E94F847A6E7B5E080E090E0E4
:10AE16000E94D64AA0E00E94F847A1E00E9410488E
:10AE2600A3E8B5E080E090E00E94D64AA0E00E9448
:10AE36001048A1E00E942848A3E9B5E080E090E030
:10AE46000E94D64AA0E00E9428480E9458B90E9453
:10AE560069B3A3E00E94B74AA1E00E942347A8EE87
:10AE6600B3E00E94650F0E9436B9EF96EF96A29660
:10AE760008956A970E9405C2E1E0E093E5140E94F6
:10AE860041560E2F023010F40C945857E0EAF5E0C4
:10AE960060E070E00E9497C30E94ABB70E94269BB9
:10AEA600E1E00E940CC26F9608950E9469B3FE010C
:10AEB60071960E9416B8AEE0B0E00E94D41C0E94C3
:10AEC60086460E9469B330911E1640911F160E9455
:10AED6005EB9E2E00E94E6C2EF87F88BE0911E16AB
:10AEE600F0911F16F695E795ED87FE870E945EB9ED
:10AEF600E5E0F0E00E9404C3EB87FC870E945EB9A0
:10AF0600EAE0F0E00E9404C3E987FA87A0E00E9425
:10AF1600B547A1E00E94CD47A1E00E94B74AAFEA3B
:10AF2600B5E080E090E00E9446B9A0E00E94CD47DF
:10AF3600A5ECB5E080E090E00E94D64AE091EA14E4
:10AF4600F091EB140E94A3B10E9463B90E94C74A14
:10AF5600AAEDB5E080E090E00E9446B9AEEDB5E01E
:10AF660080E090E00E94D64AE091F6140E9467B90C
:10AF7600E091F7140E9467B9E091F8140E9478B93D
:10AF8600A1E00E94B74AA2EFB5E080E090E00E94FF
:10AF9600D64AE091F9140E9478B90E9483B9E091EB
:10AFA600FA140E9478B90E9483B9E091FB140E94BA
:10AFB60078B9A2E00E94B74AA4E0B6E080E090E04B
:10AFC6000E9446B900E0083010F00C941758A2EE23
:10AFD600B5E10E94C8B81D912C91012E022A11F0EC
:10AFE6000C94F65710C0E3E0F0E0E117F20711F019
:10AFF6000C940458ADE1B6E080E090E00E94D64A99
:10B0060002C00E9489B900240116020610F00C94B1
:10B0160015580E9493B91D912C910E9489B9A1E0FF
:10B026000E94B74A0F5FCFCFA1E00E94B74AA6E2BF
:10B03600B6E080E090E00E9446B908E0003110F0EA
:10B046000C94D358A2EEB5E10E94C8B81D912C917C
:10B05600012E022A11F00C94315891C0E3E0F0E081
:10B06600E117F20711F00C943F58A1E4B6E080E036
:10B0760090E00E94D64A83C0E32FF42FE456F040B6
:10B08600E117F20710F00C945258E32FF42FEC5905
:10B09600FF4F1E172F0710F00C94525801C007C01F
:10B0A600A7E4B6E080E090E00E94D64A68C0EF854B
:10B0B600F889E85CF040E117F20710F00C946D583F
:10B0C600EF85F889E853FF4F1E172F0710F00C94F1
:10B0D6006D5801C007C0AAE4B6E080E090E00E9487
:10B0E600D64A4DC0ED85FE85F297E117F20710F0BE
:10B0F6000C948658ED85FE85F2961E172F0710F0E4
:10B106000C94865801C007C0ADE4B6E080E090E03C
:10B116000E94D64A34C0EB85FC857497E117F20786
:10B1260010F00C949F58EB85FC8574961E172F071C
:10B1360010F00C949F5801C007C0A2E5B6E080E06D
:10B1460090E00E94D64A1BC0E985FA853A97E11736
:10B15600F20710F00C94B858E985FA853A961E174E
:10B166002F0710F00C94B85801C007C0A7E5B6E049
:10B1760080E090E00E94D64A02C00E9489B900246D
:10B186000116020610F00C94D1580E9493B91D9135
:10B196002C910E9489B9A1E00E94B74A0F5F4ECF59
:10B1A600A1E00E94B74AACE5B6E080E090E00E94DC
:10B1B600D64AE091EC14F091ED140E94A3B10E94DE
:10B1C60063B90E94C74AABE6B6E080E090E00E9411
:10B1D600D64AE091EE14F091EF140E94A3B10E94BA
:10B1E60063B90E94C74AA9E7B6E080E090E00E94F2
:10B1F600D64AE0910215F0910315609104157091FD
:10B2060005150E94ACAD0E9463B90E94C74AA6E824
:10B21600B6E080E090E00E94D64AE0910A15F091EF
:10B226000B1560910C1570910D150E94ACAD0E9426
:10B2360063B90E94C74AA7E9B6E080E090E00E94A1
:10B24600D64AE0911E16F0911F160E94A3B10E94E5
:10B2560063B90E94C74AA8EAB6E080E090E00E947F
:10B26600D64AA3E00E94B74A0E9469B3A3E00E94AF
:10B276002347E0E00E940CC26F9608950E949CB995
:10B286000E94A4B910F00C944B590E94AFB902C0A9
:10B296000E94B4B900E010E00030E2E01E0710F0B2
:10B2A6000C945C59DE0113960E9445AE0F5F1F4F4A
:10B2B600F3CF0E94BBB90E94C5860E940EC2239698
:10B2C600DE5F0895AA9323970E94C8B9E985EE83A5
:10B2D600F801E07CAF01405C5F4FFA01E01BF10B27
:10B2E600EF83F887EE810E94CFB910F00C947E5957
:10B2F6008A010E94AFB90E94D5B9AE85BF850E946A
:10B30600DCB92C960895AA932B97E8E0E8830E946F
:10B31600C8B9F801E07CAF01405C5F4FDA01A01BC1
:10B32600B10BEE81F0E0AE17BF0710F00C949E59FA
:10B336008A010E94AFB9EBE1EF83EC89E887EB89DC
:10B34600E987EA89EA87E989EB87E0E2EC87ED8716
:10B35600EE870E94D5B9DE011B960E94DCB9659680
:10B3660008950E949CB90E94A4B910F00C94BE598D
:10B376000E94AFB902C00E94B4B900E010E00030EC
:10B38600E2E01E0710F00C94CF59DE0113960E94DE
:10B3960045AE0F5F1F4FF3CF0E94BBB90E94EEB9B7
:10B3A6000E9422B60E944F9A0E94F5B90E94FAB9ED
:10B3B6000E940EC22396DE5F08950E9404C23A2FB1
:10B3C6004E815F81E1E0E093E514E32FE0530E2F19
:10B3D600023010F40C94F05900E04A93A32F0E9417
:10B3E60018251E2F523611F00C94FD59A02F0E94DD
:10B3F600F84742C0553711F00C94055AA02F0E9409
:10B4060010483AC05C3611F00C940D5AA02F0E94D9
:10B41600284832C0513611F00C94155AA42F0E94B8
:10B4260040482AC0543611F00C94225A133310F4B3
:10B436000C941E5A12E3A12F0E94E5471DC05636F2
:10B4460011F00C942B5A1A93ACE00E947A4714C060
:10B45600533711F00C943F5AA12FEAE00E94F6C22E
:10B466002E2FA22F0E94CD47A12FEAE00E9445C3AE
:10B476002E2FA22F0E94B5470E9436B90E940BC2FA
:10B48600289608950E94B4ADE1E0E093E514E22F1A
:10B49600E0530E2F3A93A22F0E9418251E2FE42F59
:10B4A600E33611F00C945B5AA1E00E9423475EC07C
:10B4B600E03711F00C94635AA2E00E94234756C06D
:10B4C600E53611F00C946B5AA3E00E9423474EC058
:10B4D600E23411F00C94745AA8EEB3E00E94A34A29
:10B4E60045C0EE3611F00C94865A003011F40C94D7
:10B4F600815A0A3010F00C94815A01C001E0A02F45
:10B506000E94B74A33C0EC3611F00C94925A000FE1
:10B51600000F000FA02FBB270E94584727C0E23616
:10B5260011F00C949E5A000F000F000FA02FBB279E
:10B536000E9469471BC0ED3611F00C94A65AA12F44
:10B546000E94194B13C0E23711F00C94AE5AA12F8A
:10B556000E942B4B0BC0E33711F00C94B95AAAE0AA
:10B566001A9F102DA12FBB270E94674D0E9436B946
:10B576000E940CC227960895A2970E9404C25A2FD1
:10B58600E1E0E093E5140E9418B6A9A5A43411F0F1
:10B596000C942A5BE52FE03311F00C94D95AE6E9B6
:10B5A600F4E10E943BAF0E940CBA4CC0E13311F0AB
:10B5B6000C94E45AEEE9F4E10E943BAF0E940CBA07
:10B5C60041C0E23311F00C94EF5AE6EAF4E10E942E
:10B5D6003BAF0E940CBA36C0E33311F00C94FA5A12
:10B5E600EEEAF4E10E943BAF0E940CBA2BC0E433B2
:10B5F60011F00C94055BE6EBF4E10E943BAF0E9470
:10B606000CBA20C0E53311F00C94105BEEEBF4E1BC
:10B616000E943BAF0E940CBA15C0E63311F00C94A1
:10B626001B5BE6ECF4E10E943BAF0E940CBA0AC039
:10B63600E73311F00C94255BEEECF4E10E943BAF8E
:10B646000E940CBA0E9410BA0E9415BA0895E9A584
:10B65600E33611F00C94345B0E941ABA0E941FBAAA
:10B666009CC0ED3611F00C943D5B0E9428BA0E94F6
:10B676001FBA93C0EC3611F00C944A5BE4EAF0E092
:10B686000E943BAFA0E2B0E00E940E1C86C0E736E7
:10B6960011F00C94535B0E942DBA0E941FBA7DC014
:10B6A600EA3711F00C945C5B0E9432BA0E941FBA12
:10B6B60074C0E13611F00C94655B0E9437BA0E94A3
:10B6C6001FBA6BC0E43711F00C94825BA8A5AC36A8
:10B6D60011F00C94705B41E001C040E0E091D011A4
:10B6E600EA93E091D111EA93E091D211EA93E0E076
:10B6F600EA934A93DE011B960E94821F4EC0E436EF
:10B7060011F00C949F5B20E030E0A8A5A53711F05E
:10B716000C948F5B22E031E0E091CE110E943CBA9E
:10B72600E0E2EA93E091CC11EA932A933A93DE01A0
:10B736001C960E942E2031C0E73711F00C94D05B86
:10B74600A091CF11A13010F40C94B05BA091CF1151
:10B75600A83010F00C94B05B0BC0E4EEF6E060E0AD
:10B7660070E00E9497C3DE011A960E94EC1C15C079
:10B7760041E0553611F00C94C15B42E0E091CF11E7
:10B78600EA934A93DE0118960E94D225A8A5A3370C
:10B7960011F00C94D05BE0E0E8870E9410BA0E949A
:10B7A60015BA0895EF97EF97A2970E9406C21A2F2F
:10B7B600FE01EC55FF4F2081FE01EB55FF4F308116
:10B7C600E1E0E093E5140E946AB8A0EAB0E00E94C6
:10B7D600D41CE32FE23611F00C94045CE0EFF6E0A3
:10B7E60060E070E00E9441BA0E9451B90E949BB786
:10B7F600A4E10E9490480E9469B3A1E00E94B74A62
:10B806001EC0EC3611F00C94195CE12FE0530E2F9C
:10B816000A3010F40C94105C01E0A02F0E946E48D0
:10B826000E9469B3A1E00E94B74A09C0E13711F04E
:10B836000C94225C0E9469B3A1E00E94B74A0E9460
:10B8460036B90E940DC2EF96EF96A89608951A9300
:10B856000A938D01E1E0E093E514F801E181E33715
:10B8660011F00C943B5C0E9446BA0E94E0591AC043
:10B87600E63611F00C94445C0E9446BA0E94455A82
:10B8860011C0E63711F00C944D5C0E9446BA0E9436
:10B89600BF5A08C0E73611F00C94555C0E9446BAB0
:10B8A6000E94D55B0E9436B9099119910895AA9311
:10B8B6002897D2500E9404C2E1E0E093E514A0E08C
:10B8C6000E9491270E9434B2FE01E25FFD4F008183
:10B8D6001127D801E9E00E9448C28F010030EEE34B
:10B8E6001E0710F00C947A5C0E94AFB902C00E9449
:10B8F600B4B900E010E00030E2E01E0710F00C944E
:10B906008B5CDE0116960E9445AE0F5F1F4FF3CF8C
:10B91600E0912616F09127160E944FBAE0E0F2E079
:10B92600FA93EA93DE011C960E94EEB90E9497C331
:10B93600DE01AE5EBD4FAC910E9456BA0E944F9A90
:10B946000E949BB70E94FAB90E9441564E2F423080
:10B9560010F40C94B65C0E9436B9E42F0E940BC218
:10B966002F96DE5F0895A3E00E94B74A20E030E0FC
:10B9760040E0F9012F5F3F4F0E9456AF5C915B316B
:10B9860011F00C94C85C41E009C0503011F00C94E1
:10B99600CE5C42E003C0A52F0E9475152034E0E07E
:10B9A6003E0710F00C94DC5C403011F00C94DC5C2B
:10B9B60001C001C0DECF0E9496B2413011F00C9456
:10B9C600FA5C21503040F9010E9404B8FA93EA93D8
:10B9D600FE01E85FFD4FFA93EA930E940CBADE017E
:10B9E600AA5FBD4F0E942A5C285F3F4F05C04230C8
:10B9F60011F00C94FF5C00C02030E2E03E0710F02E
:10BA06000C94065DB5CF0E9496B20E9436B9E0E06E
:10BA16000E940BC22F96DE5F08950A9300E00E94F3
:10BA2600652AE03011F40C94195D02600E94932A95
:10BA3600E03011F40C94205D04600E94C32AE030CB
:10BA460011F40C94275D08600E94EF2AE03011F48F
:10BA56000C942E5D00610E941D2BE03011F40C94B5
:10BA6600355D0062E02F099108950A9300E00E9477
:10BA7600AE2DE03011F40C94415D01600E94D42B90
:10BA8600E03011F40C94485D04600E943D2BE030D8
:10BA960011F40C944F5D08600E945D2BE03011F4A8
:10BAA6000C94565D00610E94B32BE03011F40C94A7
:10BAB6005D5D0062E02F099108950E9404C21A2F6D
:10BAC6002E813F8148855985183010F00C94705DA1
:10BAD600E1E00E940BC22A9608950E945BBA00E03C
:10BAE6000E946429E03011F40C947A5D01600E9492
:10BAF6001028E03011F40C94815D02600E94302819
:10BB0600E03011F40C94885D04600E949B28E030BC
:10BB160011F40C948F5D08600E94162AE03011F42F
:10BB26000C94965D0061E02FDA01EC930E94385D7B
:10BB3600DA011196EC9300E00E94022EE03011F437
:10BB46000C94A65D01600E94CE2DE03011F40C9499
:10BB5600AD5D02600E94E727E03011F40C94B45DFD
:10BB660004600E94C129E03011F40C94BB5D0860AA
:10BB76000E94AB29E03011F40C94C25D00610E9472
:10BB8600D729E03011F40C94C95D00620E94F729B0
:10BB9600E03011F40C94D05D00640E94422EE03037
:10BBA60011F40C94D75D0068FA0102830E94FE2B03
:10BBB600DA011396EC930E944A2CDA011496EC9360
:10BBC600D901E8E0EC930E940BC22A9608952A97C1
:10BBD6000E9404C21A2F288939894A895B8900E0A4
:10BBE600183010F00C94FC5DE1E00E940BC26496E4
:10BBF60008950E945BBA0E949BB70E94D3B100E0F1
:10BC06000E945A2DE03011F40C940A5E01600E94E5
:10BC1600742DE03011F40C94115E02600E94BC2E6B
:10BC2600E03011F40C94185E04600E94322DE0306E
:10BC360011F40C941F5E08600E94402DE03011F450
:10BC46000C94265E0061E02FDA01EC9300E00E947E
:10BC5600D02CE03011F40C94315E01600E94B42CBB
:10BC6600E03011F40C94385E02600E94F82CE0304B
:10BC760011F40C943F5E04600E94202DE03011F414
:10BC86000C94465E08600E94A22CE03011F40C94DD
:10BC96004D5E00610E948E2DE03011F40C94545ECE
:10BCA6000064FA0101830E94105DDA011296EC939A
:10BCB60000E00E94F127E03011F40C94635E01600D
:10BCC6000E941929E03011F40C946A5E02600E9409
:10BCD6005328E03011F40C94715E04600E9495299B
:10BCE600E03011F40C94785E08600E94012AE0307E
:10BCF60011F40C947F5E00610E94F528E03011F487
:10BD06000C94865E00620E94672BE03011F40C945E
:10BD16008D5E0064FA01038300E00E948029E03012
:10BD260011F40C94975E01600E941029E03011F422
:10BD36000C949E5E02600E942829E03011F40C9457
:10BD4600A55E04600E94162AE03011F40C94AC5EE5
:10BD560008600E948F2EE03011F40C94B35E0061EF
:10BD66000E94982EE03011F40C94BA5E00620E9494
:10BD7600A42EE03011F40C94C15E00640E94AD2E36
:10BD8600E03011F40C94C85E0068FA0104830E9446
:10BD9600E32EDA011596EC935A934A930E9463BAFE
:10BDA6000E940CBAD901E8E0EC93E0E00E940BC2D5
:10BDB600649608956697FE010E9416B8A6E1B0E063
:10BDC6000E94D41CE6E0F7E060E070E00E94A6B2B4
:10BDD6000E9468BA66960895A8970A930E94C8B604
:10BDE6000E9475BAE8A7E7E1F7E060E070E00E941C
:10BDF6007DBADE0111960E94F81A0E2F0E94BFB678
:10BE0600E0E2EC93E4E2F7E060E070E00E9497C3C2
:10BE16000E943BB4A4E1B0E00E94AB1CDE01119687
:10BE26000E94F81AEA93DE0112960E944176A0E07B
:10BE36000E9432760881A9960895A8970E949AB220
:10BE4600E1E3F7E060E070E00E94A6B20E9468BA03
:10BE5600A89608956E970E9405C20A2F1BA12CA1D1
:10BE66003DA14EA10E3110F00C943E5FE1E00E9420
:10BE76000CC2A79608954A933A93E0E0EA93A02F5E
:10BE8600BB270E94D41C0E943BB40E94D3B1E09110
:10BE9600DF12A32FB42FEC93E091E012A32FB42F5F
:10BEA6001196EC93E091E112A32FB42F1296EC9326
:10BEB600E091E212A32FB42F1396EC93E091E312D4
:10BEC600A32FB42F1496EC93E091E412A32FB42F72
:10BED6001596EC93E091E512A32FB42F1696EC93EA
:10BEE600E091E612A32FB42F1796EC93E091E71298
:10BEF600A32FB42F1896EC93E091E812A32FB42F3A
:10BF06001996EC93E091E912A32FB42F1A96EC93AD
:10BF1600E091EA12A32FB42F1B96EC93E091EB125B
:10BF2600A32FB42F1C96EC93E091EC12A32FB42F01
:10BF36001D96EC93E091ED12A32FB42F1E96EC9371
:10BF4600E091EE12A32FB42F1F96EC93E091EF121F
:10BF5600A32FB42F5096EC93E091F012A32FB42F99
:10BF66005196EC93E091F112A32FB42F5296EC93D5
:10BF7600E091F212A32FB42F5396EC93E091F312B3
:10BF8600A32FB42F5496EC93E091F412A32FB42F61
:10BF96005596EC93E091F512A32FB42F5696EC9399
:10BFA600E091F612A32FB42F5796EC93E091F71277
:10BFB600A32FB42F5896EC93E091F812A32FB42F29
:10BFC6005996EC93E091F912A32FB42F5A96EC935D
:10BFD600E091FA12A32FB42F5B96EC93E32FF42F84
:10BFE6007C96A0E0A083E32FF42F7D96A083E32F19
:10BFF600F42F7E96A0834A933A930E948BB6AEE1C5
:10C00600B0E00E94E71BA12FB22FEEE1EC93E0E037
:10C016000E940CC2A7960895E6971A930A93E09198
:10C02600D011EE83E091D111EF83E091D211E88730
:10C03600E091CC11E987E091CD11EA87E091CE112C
:10C04600EB87E091CF11EC87E0E2ED870091D31109
:10C056001091D4111A930A93A0E00E94A124EE87AE
:10C066000E947AB6EF87E0E2E88BE98BE091D51182
:10C07600F091D6116091D7117091D8110E9483BAB0
:10C08600EA8B0E948CBAA1E00E94BD24EB8B0E9431
:10C096008CBAA2E00E94BD24EC8B0E948CBAA3E06D
:10C0A6000E94BD24ED8BA091CC110E94DB23EE8B68
:10C0B600A091CC110E94E823EF8BA091CC110E9495
:10C0C6000324E88FE091CF11EA93A091D0110E944A
:10C0D6003224E98FE091CF110E9493BA0E94432443
:10C0E6000E9474B6EA8F0E947AB6EB8FE091CE1169
:10C0F600EA93A091D0110E9451240E9474B6EC8F4D
:10C106000E947AB6ED8FE091CE110E9493BA0E94FA
:10C116005F240E9474B6EE8F0E947AB6EF8F0E945B
:10C126009ABAA091CE110E94A4230E9474B6E8A3E5
:10C136000E947AB6E9A30E949ABAE091CE11EA93D8
:10C14600A091D0110E946C240E9474B6EAA30E94AA
:10C156007AB6EBA3E0E0ECA3EDA30E949ABAE091D5
:10C16600CE110E9493BA0E9480240E9483BAEEA345
:10C176000E948CBAA1E00E94BD24EFA30E948CBA53
:10C18600A2E00E94BD24E8A70E948CBAA3E00E9408
:10C19600BD24E9A70E944A51EAA7E0E0EBA7ECA775
:10C1A600EDA7EA83EB83EC83ED830E948CBAA0E0D3
:10C1B6000E94BD24EEA70E948CBAA1E00E94BD2475
:10C1C600EFA70E948CBAA2E00E94BD24E8AB0E94B1
:10C1D6008CBAA3E00E94BD24E9ABECE2EA93DE014F
:10C1E60017960E944176A0E00E943276E0E019811F
:10C1F6000881E8960895E0E0E0932816E093291672
:10C20600E0932A16EAE0E0932B16E0932C160E94A0
:10C216009DBAE0E0E0933D16E0933C16E0933F16AE
:10C2260008950E949DBAA0E00E94DE2BA0E00E9425
:10C236001F2CA0E00E94B5290E94A3BAA0E00E948C
:10C24600982D0E9495B30E94822C089521970E94F2
:10C25600ABB2A0912816A13011F00C943261A091D6
:10C266002816A23011F00C943861A0912916A1303D
:10C2760011F00C943E61A0912916A23011F00C9495
:10C286004461A0913B16A33011F00C9455610E94B5
:10C296009529E03011F40C9452610E94ADBAEE81FA
:10C2A600E260EE83A0913B16A23011F40C9460611B
:10C2B600A33011F40C94606120C020913A16332704
:10C2C600AAE0A29FF001A39FF00D9F012436E0E0B3
:10C2D6003E0710F00C94716124E630E0A3E10E9461
:10C2E600F40F8F010217130710F40C947D61A0E080
:10C2F6000E94B529EE81E260EE830E94B3BA5E2FFA
:10C30600513011F40C948C61523011F40C948C6100
:10C3160077C0A4E10E94F40F8F010E94012A4E2FDC
:10C32600A0913C16A23011F00C94A0610536E0E015
:10C336001E0710F40C94A06101C002C00E94A3BAAB
:10C346000333E0E01E0710F40C94B4610436E0E019
:10C356001E0710F00C94B461403011F00C94B461D7
:10C366000CC0093CE0E01E0710F40C94BF6140309D
:10C3760011F40C94BF6101C009C0A0913C16A23013
:10C3860011F00C94C961E9ECE093EA120333E0E0A2
:10C396001E0710F40C94DA610436E0E01E0710F074
:10C3A6000C94DA61403011F40C94DA6101C003C0D8
:10C3B600E1E0E0933D16093CE0E01E0710F40C9422
:10C3C600F5610A3FE0E01E0710F00C94F56140307D
:10C3D60011F00C94F561E0913D16E03011F40C94E7
:10C3E600F56101C006C0E1E0E093EA12E0E0E09307
:10C3F6003D16403011F40C940362EE81E260EE8348
:10C40600AAE10E942FB910F40C940D62A0E00E94DC
:10C41600C62E03C0EE81E260EE830E94B8BA5E2F9C
:10C42600513010F40C946B62A0913E16A53010F4B6
:10C436000C941E624DC0A0913E16A03011F40C94CF
:10C446002962A23011F40C94296207C00E94672B5E
:10C45600E03011F00C94306201C002C00E94BDBAF7
:10C46600A0913E16A13011F40C943E62A33011F453
:10C476000C943E6207C00E94672BE03011F40C94C6
:10C48600456201C002C00E94BDBAABE10E94F40F32
:10C496008F01A0913E16A43011F00C945A62A0E0D0
:10C4A6000E946D2B0E94BDBAE1E0E093ED120D32C1
:10C4B600E1E01E0710F40C946862A0E00E946D2B68
:10C4C6000E94BDBAE8ECE093ED12EE81E260EE83E5
:10C4D600A0912A16A23011F00C949062A7E10E9456
:10C4E600F40F8F01E0912D160E94C3BA10F00C9440
:10C4F6008362A0E00E94982DA7E10E94DD0F0DC087
:10C50600E0912C160E94C3BA10F00C949062A1E040
:10C516000E94982DEE81E460EE83A0912E16A23043
:10C5260011F00C94B162A8E10E94F40F8F01E09122
:10C5360031160E94C3BA10F00C94A862A0E00E94C3
:10C54600BE2BA8E10E94DD0F09C0E09130160E94C3
:10C55600C3BA10F00C94B1620E94C8BAA091351605
:10C56600A23011F00C94D262A9E10E94F40F8F015F
:10C57600E09138160E94C3BA10F00C94C962A0E08C
:10C586000E94BE2BA9E10E94DD0F09C0E09137167B
:10C596000E94C3BA10F00C94D2620E94C8BAE0910D
:10C5A600DC14E03011F40C94E762AAE00E94CFBAE2
:10C5B60010F40C94E462A0E00E94D827E0E0E09337
:10C5C600DC14EE81E860EE83A091FA12A23011F03D
:10C5D6000C94FD62A9E00E94D6BA10F40C94F9629C
:10C5E600A0E00E94D82DE1E0E093FA12EE81E0612E
:10C5F600EE831FC0A091FA12A33011F00C941363BE
:10C60600A9E00E943F108F010A30E0E01E0710F4F7
:10C616000C940F630E94DDBAEE81E061EE8309C0DF
:10C62600E091FA12E03011F00C941C63A0E00E9435
:10C63600D82DA0913F16A23011F00C942C63ADE0DA
:10C646000E94CFBA10F40C942B63E0E0E0933F16FF
:10C656001CC0A0913F16A13011F00C944863ADE0C8
:10C666000E943F108F010430E0E01E0710F40C9486
:10C676004563A0E00E94F42BE2E0E0933F16ADE0B4
:10C686000E942310EE81E160EE83EE810E940BC2D0
:10C69600279608950A930A2F00932816A1E00E9470
:10C6A600822CA0912816A13011F00C945C630E9494
:10C6B600E4BAA0912816A23011F00C9464630E948B
:10C6C600E4BAE0912816E03011F00C946D63A0E016
:10C6D6000E94DE2B099108950A930A2F00932916CA
:10C6E600A0912916A13010F40C947C63E1E0E0934C
:10C6F6002916A1E00E94822CA0912916A13011F0E2
:10C706000C9492630E94F82CE03011F00C94926322
:10C71600A2E10E94DD0FA09129160E941F2CA09174
:10C726002916A23011F00C949863E0912916E03096
:10C7360011F00C94A163A0E00E941F2C09910895AA
:10C746000E94B4AD40932A16313010F40C94AD63B8
:10C7560030932B16213010F40C94B36320932C16CF
:10C76600E0912B16A0912C16EA0FE0932D1641307E
:10C7760011F00C94C563A1E00E94982DA4E20E94DA
:10C78600DD0F0DC0A4E20E94F40F8F010D32E1E02F
:10C796001E0710F40C94D263A0E00E94982D0E940C
:10C7A6000CC2279608950E9485B620932E16113046
:10C7B60010F40C94E06310932F16013010F40C94CF
:10C7C600E66300933016E0913016A0912F16EA0F1B
:10C7D600E0933116213011F00C94F563A1E00E942C
:10C7E600BE2B03C0A0E00E94BE2B0E940EC225965F
:10C7F60008950E9485B620933216113010F40C94D9
:10C80600066410933316013010F40C940C640093F4
:10C816003416213011F00C941464A1E00E94272BE9
:10C8260003C0A0E00E94272B0E940EC22596089501
:10C836000E9485B620933516113010F40C942564A9
:10C8460010933616013010F40C942B6400933716AF
:10C85600E0913616A0913716EA0FE093381621308C
:10C8660011F00C943A64A1E00E94472B03C0A0E0AB
:10C876000E94472B0E940EC2259608950A930A2FFE
:10C8860000933916013011F00C944D64A1E00E941A
:10C896009D2B03C0A0E00E949D2B099108950A9349
:10C8A6000A2F003011F40C945F64A1E00E94B529B0
:10C8B600E1E0E0933B1606C0A0E00E94B529E1E066
:10C8C600E0933B16099108950E94ADBAE2E0E09329
:10C8D6003B160895E3E0E0933B1608950A930A2F6A
:10C8E60000933A16099108951A930A931A2F0E94F3
:10C8F600B3BA0E2F013011F40C948664023011F491
:10C906000C94866420C0113011F00C949464A0E05D
:10C916000E94C729A1E00E94DD29E1E0E0933C16D0
:10C926000FC0123011F00C949E640E94EBBAE1E045
:10C93600E0933C1605C00E94F1BAE0E0E0933C1695
:10C94600A4E10E94DD0F0991199108950A930E94AE
:10C95600B3BA0E2F013011F40C94B664023011F400
:10C966000C94B66408C0A1E00E94DD29A0E00E94F4
:10C97600C7290E94F7BA099108950A930E94B3BA8B
:10C986000E2F013011F40C94CD64023011F40C9486
:10C99600CD6404C00E94EBBA0E94F7BA09910895CB
:10C9A600A1E00E94C62EAAE10E94DD0F08950A9317
:10C9B6000E94B8BA0E2F013010F40C94ED640E9458
:10C9C600DF2EA1E00E946D2BABE10E94DD0FE0E0BF
:10C9D600E0933E16099108950A930E94B3BA0E2F6A
:10C9E600013010F40C940E650E94A22CE03011F474
:10C9F6000C940265A1E00E94822C0E9428B40E9439
:10CA0600322DE03011F40C940B65E1E009910895A4
:10CA1600E0E009910895E1E0099108950A930E94E2
:10CA260000BB0E2F013010F40C9430650E94A22C2E
:10CA3600E03011F40C942465A1E00E94822C0E943F
:10CA460028B40E94402DE03011F40C942D65E1E0ED
:10CA560009910895E0E009910895E1E009910895AA
:10CA66000A930E94A22CE03011F40C943C650E94BB
:10CA760005BB0E94C22C0E2F013011F00C944665A6
:10CA8600E1E009910895E0E0099108950A930E9472
:10CA9600A22CE03011F40C9452650E9405BB0E9452
:10CAA600BC2E0E2F003011F00C945C65E0E009916D
:10CAB6000895E1E0099108950E94A22CE03011F456
:10CAC6000C9467650E9405BB0E94742DE03011F43A
:10CAD6000C946F65E1E00895E0E008951A930A93D7
:10CAE60010E00E94A22CE03011F40C947C650E94A8
:10CAF60005BB0E94C22C0E2F013011F00C948465E8
:10CB060011600E94BC2E0E2F013011F00C948C6522
:10CB160012600E94742D0E2F003011F00C94946553
:10CB26001460E12F099119910895E1E0E093DC1476
:10CB3600A1E00E94D827AAE00E94231008950A9334
:10CB4600E1E0E093FA120E940CBB0E2F013010F4C4
:10CB56000C94B065E2E00E9411BB09910895E3E0F0
:10CB66000E9411BB08950E94DDBA0895E091FA1261
:10CB760008950A930A2FE0913F16E03011F00C94C5
:10CB8600D565013010F40C94CC65A1E00E94F42B1D
:10CB960003C0A2E00E94F42BE1E0E0933F16ADE073
:10CBA6000E942310099108950895E0E00895BA932C
:10CBB600AA93EF97AD970E9404C2FE01EC58FF4F6F
:10CBC6000190F081E02DDE01A059BF4FED93FC935B
:10CBD600FE01EE58FF4F0190F081E02DDE01A259D3
:10CBE600BF4FED93FC930E94B3BA5E2FDE01A059AE
:10CBF600BF4FAC910E947376FE01E059FF4F019042
:10CC0600F081E02DEA30A0E0FA0711F00C940E66F0
:10CC16000E94DD5EE6C2E436A0E0FA0711F00C944D
:10CC260020660E9419BB2E2FE1E0EA93ADB7BEB78E
:10CC36002F930E9441762F91D4C2E936A0E0FA07DD
:10CC460011F00C9436660E941EBBEA8FE8E0EB8F6B
:10CC56000E9423BBEC8FE2E0ED8FE0E0EE8FE4E094
:10CC66000E9428BBBEC2EB30A0E0FA0711F00C947C
:10CC76003F660E94EF5EB5C2EC30A0E0FA0711F005
:10CC86000C9448660E94205FACC2E536A0E0FA0725
:10CC960011F00C945C660E942DBBEDB7FEB7FA93BB
:10CCA600EA932F93A2E40E942D5F2F910E9432BB3C
:10CCB60098C2E636A0E0FA0711F00C9470660E945E
:10CCC6002DBBEDB7FEB7FA93EA932F93A2E40E9429
:10CCD600EA5D2F910E9432BB84C2E736A0E0FA07D4
:10CCE60011F00C9484660E942DBBEDB7FEB7FA9343
:10CCF600EA932F93A2E40E94605D2F910E9432BBBB
:10CD060070C2E836A0E0FA0711F00C94A166DE01C5
:10CD1600A45ABF4F0E94E84E3E2FE0E0DE01AD5917
:10CD2600BF4FEC93303011F00C94A066E8E0EA9324
:10CD3600DE01A35ABF4F0E94417653C2E331A0E001
:10CD4600FA0711F00C94AA660E940F604AC2EA36EE
:10CD5600A0E0FA0711F00C94D6660E94A8530E9430
:10CD660074B6EA8F0E947AB6EB8F0E9479530E94BE
:10CD760074B6EC8F0E947AB6ED8FA0E00E94E05365
:10CD86000E9474B6EE8F0E947AB6EF8FA1E00E94E1
:10CD9600E0530E9474B6E8A30E947AB6E9A3E8E0DD
:10CDA6000E9428BB1EC2EE30A0E0FA0711F00C94D8
:10CDB6002867A4ECB0E00E94ACC3EA8F0E94B3BA25
:10CDC600EB8FA6ECB0E00E94ACC3EC8FA7ECB0E012
:10CDD6000E94ACC3ED8FA8ECB0E00E94ACC3EE8F0E
:10CDE600A9ECB0E00E94ACC3EF8FAAECB0E00E94C1
:10CDF600ACC3E8A30E94B8BAE9A3ACECB0E00E94C9
:10CE0600ACC3EAA30E9400BBEBA3AEECB0E00E9469
:10CE1600ACC3ECA30E940CBBEDA3A0EDB0E00E9456
:10CE2600ACC3EEA3A1EDB0E00E94ACC3EFA3A2EDAC
:10CE3600B0E00E94ACC3E8A7A3EDB0E00E94ACC38B
:10CE4600E9A7E0E10E9428BBCCC1E131A0E0FA07E6
:10CE560011F00C9477670E941ABA0E9437BBEA8FCA
:10CE66000E941ABA0E943CBBEB8F0E9428BA0E940D
:10CE760037BBEC8F0E9428BA0E943CBBED8F0E9404
:10CE86002DBA0E9437BBEE8F0E942DBA0E943CBB82
:10CE9600EF8F0E9432BA0E9437BBE8A30E9432BAD3
:10CEA6000E943CBBE9A30E9437BA0E9437BBEAA3A3
:10CEB6000E9437BA0E943CBBEBA340E0403210F020
:10CEC6000C947367E42FE65F0E9441BB0F01A4EA4E
:10CED600B0E0EE27A40FBE1F0E946FB64F5FEECFE5
:10CEE600EAE20E9428BB7DC1E231A0E0FA0711F018
:10CEF6000C949267DE0116960E9464513E2F3030E4
:10CF060011F00C948D67E8E0EA93DE0117960E9413
:10CF1600417604C0E2E00E9447BB089562C1EF3645
:10CF2600A0E0FA0711F00C949F670E944A51EA8F1D
:10CF3600E1E00E9428BB55C1E431A0E0FA0711F0F8
:10CF46000C94B3670E944CBBFA93EA930E9453BBBE
:10CF5600DE015E960E94160EE0E40E9428BB41C1E7
:10CF6600E531A0E0FA0711F00C94D1670E944CBBA2
:10CF76000E944FBA0E9453BBDE0190960E94B38571
:10CF86003E2F303011F00C94CC67E0E40E9428BBB1
:10CF960004C0E2E00E9447BB089523C1EB36A0E03F
:10CFA600FA0711F00C94EA670E9458BB0E945BBB1B
:10CFB6000E949339EA8F0E94AD2EEB8F0E9428299A
:10CFC600EC8FE1E0EC8FE3E00E9428BB0AC1E6317A
:10CFD600A0E0FA0711F00C940F680E9458BB0E945B
:10CFE6005BBBE0914016EA8FE0914116EB8FA09172
:10CFF60040160E94C73AEC8FA09140160E94D63A7E
:10D00600ED8FE0914016EA93DE015F960E94E03ACA
:10D01600E8E20E9428BBE5C0E731A0E0FA0711F07C
:10D026000C942F68533011F00C941E68DE015A964A
:10D036000E94BF440DC0513011F40C942768523041
:10D0460011F40C94276804C0DE015A960E94D84059
:10D05600E0E40E9428BBC5C0EC36A0E0FA0711F058
:10D066000C9467680E9458BB0E945BBB533011F05A
:10D076000C944C680E945745EA8F41E0E42F0E94C9
:10D0860041BB0E945FBB0E946FBB0E945A454B5F2B
:10D0960017C0513011F40C945568523011F40C94A9
:10D0A60055680EC00E943C41EA8F41E0E42F0E9481
:10D0B60041BB0E945FBB0E946FBB0E943F414B5F1A
:10D0C600E8E00E9428BB8DC0ED36A0E0FA0711F01B
:10D0D6000C9472680E9458BB0E945BBB82C0E83108
:10D0E600A0E0FA0711F00C948268203011F00C943D
:10D0F6007D6804C0E4E00E9447BB089572C0E93130
:10D10600A0E0FA0711F00C94A2680E9458BB0E9496
:10D116005BBBE8E4F7E060E070E00E9497C3FE01C5
:10D126007E960E9482BBE0E0DE01A55ABF4FEC93DB
:10D13600DE015A960E94F81A0E9428BB52C0EE36AB
:10D14600A0E0FA0711F00C94B3680E9458BB0E9445
:10D156005BBB0E9488BB2F5FE8E00E9428BB41C0F2
:10D16600EA31A0E0FA0711F00C94C5680E9458BB9A
:10D176000E945BBBDE015A960E949D4E2E2F0E9496
:10D1860032BB2FC0EB31A0E0FA0711F00C94F06827
:10D196000E9458BB0E945BBB0E949BB7E0E0EA93EB
:10D1A6000E941BB80E9488BBDE0116960E949D4E07
:10D1B6002E2F0E949BB70E9430B8FE017E96FA93EE
:10D1C600EA93EAE0F0E0FA93EA93AAE0B0E00E947C
:10D1D600811CE6E10E9428BB04C0E1E00E9447BB37
:10D1E6000895E0E00E9447BB08950895E0E00895A1
:10D1F600BA93AA932D97D1500E9404C2FE01E85E0D
:10D20600FE4F0190F081E02DDE01AF5EBE4FED9343
:10D21600FC93FE01EA5EFE4F0190F081E02DDE01F7
:10D22600A15FBE4FED93FC93FE01EB5EFE4F508176
:10D23600FE01E153FF4F0E9416B8A0E4B0E00E9441
:10D24600D41C0E9453BBDE01A95EBE4FAC91BB2726
:10D256000E9456235E2F20E0251710F00C94476994
:10D26600E22F0E9491BBEA0FFB1FBF01DE01AD5EFC
:10D27600BE4F0D90BC91A02DEE27A20FBE1FEC91C4
:10D28600DB01EC932F5FE8CF0E94B3BAEAA7DE0179
:10D29600AF5EBE4F0D90BC91A02DA130E0E1BE0760
:10D2A60010F40C945969E0E0E887E987FE01EF5E27
:10D2B600FE4F0190F081E02DEA30A0E0FA0711F070
:10D2C6000C947D69E4E6F7E060E070E00E9497C3A5
:10D2D600DE01AD52BF4F0E94FD204E2F403011F4AB
:10D2E6000C9478690E94070E04C0E2E00E9496BB87
:10D2F6000895A7C5E436A0E0FA0711F00C948869F2
:10D306000E949BBB0E94A3639CC5E536A0E0FA077A
:10D3160011F00C948F6995C5E636A0E0FA0711F076
:10D326000C949A690E949BBB0E94D6638AC5E73615
:10D33600A0E0FA0711F00C94A5690E949BBB0E941D
:10D34600FC637FC5E836A0E0FA0711F00C94B069DB
:10D356000E949BBB0E941B6474C5E936A0E0FA07D5
:10D3660011F00C94BB690E94A8BB0E94416469C578
:10D37600EA36A0E0FA0711F00C94C26962C5EB36F2
:10D38600A0E0FA0711F00C94CD690E94A8BB0E9498
:10D39600D82D57C5EC36A0E0FA0711F00C94D869E1
:10D3A6000E94A8BB0E94B82D4CC5ED36A0E0FA0736
:10D3B60011F00C94E3690E94A8BB0E94CC2741C5DA
:10D3C600EE36A0E0FA0711F00C94EE690E94A8BBB5
:10D3D6000E940A2A36C5E231A0E0FA0711F00C9441
:10D3E600096A0E9460AF0E94412A0E94ADBB0E945A
:10D3F6006F2A0E94B2BB0E949D2A0E94B7BB0E9460
:10D40600CB2A0E94BCBB0E94F92A1BC5E331A0E0CF
:10D41600FA0711F00C94246A0E9460AF0E94592A00
:10D426000E94ADBB0E94872A0E94B2BB0E94B52A09
:10D436000E94B7BB0E94E32A0E94BCBB0E94112B2C
:10D4460000C5EF36A0E0FA0711F00C942F6A0E948F
:10D45600A8BB0E94822CF5C4E431A0E0FA0711F0C3
:10D466000C94656A0E94C1BBDE01A752BF4FAC9106
:10D476000E943B504E2F0E94CFBB0E94B7BB0E941A
:10D48600D5BB8F010A93FE01EB52FF4FE081EA9371
:10D49600DE01A952BF4FAC910E94C5503E2F4030CD
:10D4A60011F00C945B6A303011F00C945B6A01C089
:10D4B60004C0E0E00E9496BB0895E1E00E9496BB9E
:10D4C6000895BFC4E531A0E0FA0711F00C94786A1C
:10D4D6000E94C1BBDE01AB52BF4FAC910E943B50D4
:10D4E6004E2F0E9496BB0895ACC4E631A0E0FA0721
:10D4F60011F00C94926A0E94DBBB0E94D5BB8F018F
:10D506000A93FE01EE52FF4FE081EA930E94BCBBF4
:10D516000E94C5504E2F0E9496BB089592C4E037D4
:10D52600A0E0FA0711F00C94A86A0E94E2BB41E061
:10D53600323010F00C94A36AA32F0E9417514E2F7D
:10D54600E42F0E9496BB08957CC4E137A0E0FA0759
:10D5560011F00C94AF6A75C4E237A0E0FA0711F037
:10D566000C94B66A6EC4E337A0E0FA0711F00C9487
:10D57600C16A0E94A8BB0E944D6363C4E437A0E061
:10D58600FA0711F00C94CC6A0E94A8BB0E946F6344
:10D5960058C4E537A0E0FA0711F00C94D56A0E944A
:10D5A600D3644FC4E637A0E0FA0711F00C94E06AA2
:10D5B6000E94A8BB0E946D2B44C4E737A0E0FA077F
:10D5C60011F00C94E96A0E94DA643BC4E731A0E0EA
:10D5D600FA0711F00C94CE6B0E94E2BB323010F4C5
:10D5E6000C94F66A31E0E32FA4ECB0E00E94C8C3C5
:10D5F600FE01E053FF4F3081343010F40C94046B7D
:10D6060031E0A5ECB0E0E32F0E94C8C3FE01EF5263
:10D61600FF4F3081323010F40C94126B31E0A6ECDF
:10D62600B0E0E32F0E94C8C3FE01EE52FF4F3081E7
:10D63600323010F40C94206B30E0A7ECB0E0E32F0E
:10D646000E94C8C3FE01ED52FF4F3081313010F405
:10D656000C942E6B30E0A8ECB0E0E32F0E94C8C318
:10D66600FE01EC52FF4F3081313010F40C943C6BCC
:10D6760030E0A9ECB0E0E32F0E94C8C3FE01EB52F4
:10D68600FF4F3081313010F40C944A6B30E0AAEC35
:10D69600B0E0E32F0E94C8C3FE01EA52FF4F30817B
:10D6A600313010F40C94586B30E0ABECB0E0E32F63
:10D6B6000E94C8C3FE01E952FF4F3081313010F499
:10D6C6000C94666B30E0ACECB0E0E32F0E94C8C36C
:10D6D600FE01E852FF4F3081313010F40C94746B28
:10D6E60030E0ADECB0E0E32F0E94C8C3FE01E75284
:10D6F600FF4F3081313010F40C94826B30E0AEEC89
:10D70600B0E0E32F0E94C8C3FE01E652FF4F30810E
:10D71600313010F40C94906B30E0AFECB0E0E32FB6
:10D726000E94C8C3FE01E552FF4F3081313010F42C
:10D736000C949E6B30E0A0EDB0E0E32F0E94C8C3CE
:10D74600FE01E452FF4F3081313010F40C94AC6B83
:10D7560030E0A1EDB0E0E32F0E94C8C3FE01E35222
:10D76600FF4F3081313010F40C94BA6B30E0A2EDEB
:10D77600B0E0E32F0E94C8C3FE01E252FF4F3081A2
:10D78600313010F40C94C86B30E0A3EDB0E0E32F19
:10D796000E94C8C356C3EB30A0E0FA0711F00C9400
:10D7A600306C0E94DBBB0E94B5218F01A8E9B0E076
:10D7B6000E94C0C3FE01EE52FF4FE081EA930E9431
:10D7C600B2BB0E94B5218F01AAE9B0E00E94C0C396
:10D7D600FE01EC52FF4FE081EA930E94BCBB0E941F
:10D7E600B5218F01ACE9B0E00E94C0C3FE01EA5248
:10D7F600FF4FE081EA93DE01AA52BF4FAC910E942F
:10D80600B5218F01AEE9B0E00E94C0C3FE01E85227
:10D81600FF4FE081EA93DE01A852BF4FAC910E9410
:10D82600B5218F01A0EAB0E00E94C0C320E02032FB
:10D8360010F00C942F6CA4EAB0E0E22F0E9478B1AD
:10D84600E22FE65F0E9491BBAE0FBF1FEC91D001A5
:10D856000E94C8C32F5FEBCFF4C2E837A0E0FA07F7
:10D8660011F00C94426C0E94A8BBA13010F40C94E9
:10D876003F6C0E94BB3902C00E94A939E2C2E93757
:10D88600A0E0FA0711F00C944B6C0E948839D9C2BB
:10D89600EA37A0E0FA0711F00C94566C0E94A8BB78
:10D8A6000E94D939CEC2EB37A0E0FA0711F00C94EA
:10D8B600666C0E94E7BB0E945BAFEA930E94ADBB19
:10D8C6000E946B3ABEC2EC30A0E0FA0711F00C944D
:10D8D600766C0E94E7BB0E94C1BBDE01AB52BF4F14
:10D8E6000E947E3AAEC2E831A0E0FA0711F00C942D
:10D8F600D76C0E94DBBB0E94B5218F01E3E0F0E00C
:10D90600E887F987E0E0EE83EF83AE81BF81509729
:10D9160010F00C94B66CEE81FF81DE011A960E941F
:10D926009DB5FF93EF93E885F9853196DE01A15306
:10D93600BF4FAE0FBF1FEC91EA93E985FA85DE0172
:10D94600A053BF4FAE0FBF1FAC910E94B521AF9140
:10D95600BF91ED93FC93E885F9853296E887F987C0
:10D966000E940EAED2CFAAA5A33011F00C94C46CBF
:10D976001A930A930E94CFBBDE011D960E941F4494
:10D9860012C0AAA5A13011F40C94CE6CA23011F4E9
:10D996000C94CE6C08C01A930A930E94CFBBDE018A
:10D9A6001D960E94DA3F4DC2EC37A0E0FA0711F04F
:10D9B6000C94F66CAAA5A33011F00C94E76C0E94A7
:10D9C600A8BB0E9454440EC0AAA5A13011F40C9421
:10D9D600F16CA23011F40C94F16C04C00E94A8BB47
:10D9E6000E944D402EC2ED37A0E0FA0711F00C94CC
:10D9F600116DAAA5A33011F00C94046D0E946D441C
:10DA06000CC0AAA5A13011F40C940E6DA23011F42D
:10DA16000C940E6D02C00E94714013C2EE37A0E056
:10DA2600FA0711F00C942C6DAAA5A33011F00C94F2
:10DA36001F6D0E94A8440CC0AAA5A13011F40C9435
:10DA4600296DA23011F40C94296D02C00E94BA40CF
:10DA5600F8C1EF37A0E0FA0711F00C94336DF1C16D
:10DA6600E038A0E0FA0711F00C943A6DEAC1E1380B
:10DA7600A0E0FA0711F00C94456D0E94A8BB0E9425
:10DA86005264DFC1E238A0E0FA0711F00C94526D3F
:10DA96000E94A8BB0E9471640E946764D2C1E338E9
:10DAA600A0E0FA0711F00C945F6D0E9460AF0E942F
:10DAB60071640E946D64C5C1E438A0E0FA0711F0F4
:10DAC6000C947D6D0E945BAFE17011F40C946F6D48
:10DAD600A1E00E9477640DC00E945BAFE27011F472
:10DAE6000C94796DA2E00E94776403C0A0E00E94C6
:10DAF6007764A7C1E538A0E0FA0711F00C94866DAB
:10DB06000E94A9649EC1E638A0E0FA0711F00C94C1
:10DB16008F6D0E94C06495C1E738A0E0FA0711F046
:10DB26000C94A16D0E94E2BBA32F0E94732EA1E06C
:10DB36000E94FA27A1E00E941A2883C1E838A0E0D3
:10DB4600FA0711F00C94AC6D0E94A8BB0E946D28D8
:10DB560078C1E938A0E0FA0711F00C94B96D0E947B
:10DB6600A8BB0E949B2E0E94F5BB6BC1EA38A0E0C1
:10DB7600FA0711F00C94C46D0E94A8BB0E94D0282D
:10DB860060C1EB38A0E0FA0711F00C94D96D0E9441
:10DB9600A8BBA13011F00C94D36D0E94084702C0B7
:10DBA6000E941F47E0E0E09342164BC1E931A0E036
:10DBB600FA0711F00C94056EFE01EA52FF4FE08160
:10DBC6000E94FBBBFE01EB52FF4FE0810E94FBBBB4
:10DBD600FE01EC52FF4FE0810E94FBBBFE01ED52BD
:10DBE600FF4FE081FF2766277727EBA7FCA76DA7E6
:10DBF6007EA70E940EBCADA5BEA58FA598A90E94C2
:10DC06004E4B1FC1EA31A0E0FA0711F00C94146ED6
:10DC16000E94C1BBDE01AB52BF4FAC910E94304D9A
:10DC260010C1EB31A0E0FA0711F00C942F6E0E94A0
:10DC3600DBBB0E94B521DF010E94674D0E94ADBB90
:10DC46000E94E5470E94B2BB0E9440480E94B7BBB3
:10DC5600BB270E94764AF5C0EC38A0E0FA0711F01F
:10DC66000C944D6E0E9460AFA13011F00C94416E81
:10DC76000E94A8BBBB270E9458470BC00E9460AFFA
:10DC8600A23011F00C944C6E0E94A8BBBB270E94D8
:10DC96006947D7C0ED38A0E0FA0711F00C94636E1F
:10DCA6000E945BAFEA930E94ADBB0E947A470E9436
:10DCB600ADBB0E94B5470E94B2BB0E94CD47C1C012
:10DCC600EE38A0E0FA0711F00C94766E0E94A8BB1D
:10DCD6000E94F8470E9460AF0E9428480E94ADBB90
:10DCE6000E941048AEC0EF38A0E0FA0711F00C947D
:10DCF600816E0E94A8BB0E942347A3C0ED30A0E01E
:10DD0600FA0711F00C94916EFE01E153FF4FFA935E
:10DD1600EA93A52FBB270E94651693C0E039A0E0C1
:10DD2600FA0711F00C949C6E0E94A8BB0E94B74A99
:10DD360088C0E139A0E0FA0711F00C94A56E0E94A4
:10DD4600DE4A7FC0EE30A0E0FA0711F00C94CD6EEB
:10DD5600FE01ED52FF4F308120E0231710F00C94A6
:10DD6600C36EE22FF0E0DE019F96EA0FFB1F0F0164
:10DD7600E22FEB5F0E9491BB0E94A4AF2F5FEDCF15
:10DD86000E940EBCFE01F196FA93EA93A32F0E941D
:10DD9600904857C0EF30A0E0FA0711F00C94DF6E00
:10DDA600A0914216A33010F00C94DE6EE09142165C
:10DDB600EF5FE093421645C0E239A0E0FA0711F0A2
:10DDC6000C94E66E3EC0E339A0E0FA0711F00C941D
:10DDD600F56E0E9460AF0E947F480E94A8BB0E9419
:10DDE6006E482FC0E031A0E0FA0711F00C94006FE6
:10DDF600E42F0E9496BB089524C0E131A0E0FA0703
:10DE060011F00C940B6FE42F0E9496BB089519C075
:10DE1600E439A0E0FA0711F00C94126F12C0E23157
:10DE2600A6E3FA0711F00C94196F0BC0EC31A0E0D1
:10DE3600FA0711F00C94206F04C0E1E00E9496BB33
:10DE46000895FE01E15FFE4F0190F081E02DDE01B5
:10DE5600A15FBE4FED93FC93E0E00E9496BB089550
:10DE66001A930A938D01E2E0EC93099119910895B2
:10DE7600EA97E0E0EFAB20E030E040E050E0E4B7C6
:10DE8600EEABFE01F596EBABFCABABA9BCA90E94D1
:10DE9600336FABA9BCA90C9111279924E0E0F2E0FD
:10DEA6003E2E4F2EE4E3F2E17E2E8F2EE72DF82D47
:10DEB600A32DB42DED93FC93E2E0F0E03E0E4F1E51
:10DEC600E72DF82DEF5FFE4F7E2E8F2EEEEFF1E25F
:10DED6003E164F0610F00C94716FE8CFE0E0F2E0CA
:10DEE6003E2E4F2EE4E3F2E17E2E8F2EA32DB42D8F
:10DEF6005D906C907514860411F40C94846FE1E0C7
:10DF06009E2EE2E0F0E03E0E4F1EE72DF82DEF5F6D
:10DF1600FE4F7E2E8F2EEEEFF1E23E164F0610F0EC
:10DF26000C94966FE3CFE0E0F2E03E2E4F2EA32D49
:10DF3600B42DE0E0F0E0ED93FC93E2E0F0E03E0E7D
:10DF46004F1EEEEFF1E23E164F0610F00C94AC6F4A
:10DF5600EECF0E94A179E4B7E093F812992011F070
:10DF66000C94B96FE1E0E093DF1203C0E8ECE093B4
:10DF7600DF12E0E0E5BFE5BFE0E8E0936100E0E046
:10DF8600E0936100E3BF0E94310D0E94EE0D78948C
:10DF9600E1E0E093DD14A2EAB0E00E94A8C39F018D
:10DFA600EAE3FCE5E217F30711F40C940C71A8E917
:10DFB600B0E0E9E1F1E00E94C0C3AAE9B0E0E8EE12
:10DFC600F3E00E94C0C3ACE9B0E0E1E0F0E00E94FB
:10DFD600C0C3AEE9B0E00E94C0C3A0EAB0E0E8EE7C
:10DFE600F3E00E94C0C3E0E7F7E060E070E00E9463
:10DFF60097C3DE0115960E94EC1CE0E0EA83FE0161
:10E006003196FA93EA93E4EAF0E0FA93EA93A0E20F
:10E01600B0E00E94371CA8EDB0E0E1E00E94C8C362
:10E02600A9EDB0E0E5E00E94C8C3AAEDB0E0E0E0EB
:10E036000E94C8C3ABEDB0E0E3E00E94C8C3ACEDFC
:10E04600B0E0E0E00E94C8C3A4ECB0E0E1E00E94CA
:10E05600C8C3A5ECB0E00E94C8C3A6ECB0E00E941D
:10E06600C8C3A7ECB0E0E0E00E94C8C3A8ECB0E0EB
:10E07600E1E00E94C8C3A9ECB0E0E0E00E94C8C39A
:10E08600AAECB0E0E1E00E94C8C3ABECB0E0E0E08F
:10E096000E94C8C3ACECB0E0E1E00E94C8C3ADEC9E
:10E0A600B0E0E0E00E94C8C3AEECB0E00E94C8C396
:10E0B600AFECB0E0E1E00E94C8C3A0EDB0E00E9482
:10E0C600C8C3A1EDB0E00E94C8C3A2EDB0E00E94B3
:10E0D600C8C3A3EDB0E00E94C8C3A0E4B0E0EFEF70
:10E0E600FFEF0E94C0C3E0E0EFABAFA9AF3010F086
:10E0F6000C949770FA01A0E0B0E0EE0FFF1FAE0F90
:10E10600BF1FE0E0F0E00E94C0C3A0E2B0E0FA0169
:10E11600EE0FFF1FAE0FBF1FE0E0F0E00E94C0C38E
:10E12600EFA9EF5FEFABE1CFAEE0B0E0E8ECF0E0F7
:10E136000E94C0C3ACE0B0E0E4E6F0E00E94C0C3D9
:10E14600AAE0B0E0E2E3F0E00E94C0C3A8E0B0E0DD
:10E15600E4E1F0E00E94C0C3A6E0B0E0EAE0F0E04F
:10E166000E94C0C3AEE1B0E0E8ECF0E00E94C0C39C
:10E17600ACE1B0E0E4E6F0E00E94C0C3AAE1B0E0A2
:10E18600E2E3F0E00E94C0C3AEE2B0E0E8ECF0E00B
:10E196000E94C0C3ACE2B0E0E4E6F0E00E94C0C377
:10E1A600AAE2B0E0E2E3F0E00E94C0C3A8E2B0E079
:10E1B600E4E1F0E00E94C0C3A6E2B0E0EAE0F0E0ED
:10E1C6000E94C0C3AEE3B0E0E8EFF2E00E94C0C335
:10E1D600ACE3B0E0ECE7F1E00E94C0C3AAE3B0E034
:10E1E600EEEBF0E00E94C0C3A2E4B0E0ECE7F1E0A1
:10E1F60060E070E00E94B8C3A6E4B0E0E0E00E94F0
:10E20600C8C30E944DA9A2EAB0E0EAE3FCE50E9479
:10E21600C0C3AFECB0E0E0E00E94C8C3A7ECB0E03A
:10E226000E94C8C30E9437270E948B0FA1E00E945C
:10E236006B27A1E00E944C2E0E941B7FEEABAEA97D
:10E24600A13010F40C942B71E953E093E31203C050
:10E25600E1E0E093E3120E94762FEFABE03011F499
:10E266000C944271E2E0E093DD140E94992FA92DEF
:10E276000E94ED2FEEABAEA90E94AD31FCCFE3E0DC
:10E28600E093DD140E9423380E94BB39A5ECB0E070
:10E296000E94ACC3E883A881A33011F00C94567198
:10E2A6000E943C420CC0A881A13011F40C9460710C
:10E2B600A23011F40C94607102C00E94393D0E9494
:10E2C600FE600E9478460E94C3750E94D68A0E940C
:10E2D600D4520E9492100E94E04E0E942681E4E0F1
:10E2E600E093DD140E9478950E94BB790E94227B00
:10E2F6000E94CE79E5E0E093DD140E9425750E9428
:10E30600D0520E94C6550E94C4A60E942554A4E07D
:10E316000E942310A3E00E942310E1E0E093D914A9
:10E32600E0E0E093D614E093D714E093D814E1E04C
:10E33600E093DA14E0E0E093DC14E093DB14E0937E
:10E34600E414ACE00E94DD0FE2E0EA93E5E0EA9334
:10E35600E3E0EA93E0E0EA93A0E00E94D614E1E06D
:10E36600E0936916E0E0E0936A160E946E52789494
:10E37600A1E00E94DD0FA8E00E9423100E94CB0FAF
:10E38600E03011F00C94CA710E948B0F7894E0E093
:10E39600E093DE14E093DF14E093E014E093E114DD
:10E3A600E093E214E093E314A3E00E943F108F0190
:10E3B600A7ECB0E00E94ACC3EFABE03011F40C94D4
:10E3C600ED71E0E0E093D714E091DE14E260E093B3
:10E3D600DE1403C0E1E0E093D7140A30E0E01E0744
:10E3E60010F00C94FE71E0E0E093D714E091DE1497
:10E3F600E460E093DE14A4980E944727EFABE03078
:10E4060011F40C940E72E0E0E093D714E091DE1460
:10E41600E860E093DE140E942961EFABAFA9A1305A
:10E4260010F40C941C72E0E0E093D714EFA9E0938B
:10E43600E114A0916A160E941C53EFABE03011F470
:10E446000C942D72E0E0E093D714E091DE14E062C4
:10E45600E093DE140E94EF75EFABE03011F40C94FC
:10E466003C72E0E0E093D714E091DE14E064E093C0
:10E47600DE140E94F968EFABE03011F40C944B7295
:10E48600E0E0E093D714E091DE14E068E093DE1458
:10E496000E94D865EFABE03011F40C945A72E0E0BC
:10E4A600E093D714AFEDB4E1EC91E160EC930E94F8
:10E4B6007946EFABE03011F40C946972E0E0E0933A
:10E4C600D714AFEDB4E1EC91E260EC930E942B8B94
:10E4D600EFABE03011F40C947C72E0E0E093D714DB
:10E4E600AFEDB4E1EC91E460EC93E1E0E093E41489
:10E4F60003C0E0E0E093E414A0916A160E94DC7980
:10E50600EFABE03011F40C949072E0E0E093D71496
:10E51600AFEDB4E1EC91E860EC930E947638EFAB96
:10E52600E03011F40C949F72E0E0E093D714AFED65
:10E53600B4E1EC91E061EC93A5ECB0E00E94ACC3D1
:10E54600E883A881A33011F00C94B9720E9460424E
:10E55600EFABE03011F40C94B872E0E0E093D7141E
:10E56600AFEDB4E1EC91E062EC9319C0A881A13063
:10E5760011F40C94C372A23011F40C94C3720FC040
:10E586000E946B3DEFABE03011F40C94D272E0E0E8
:10E59600E093D714AFEDB4E1EC91E064EC930E9404
:10E5A600E74EA0916A160E943F81EFABE03011F46E
:10E5B6000C94E572E0E0E093D714AFEDB4E1EC9192
:10E5C600E068EC930E949F7EA091E4140E947C95E3
:10E5D600EFABE03011F40C94F872E0E0E093D7145E
:10E5E600A0EEB4E1EC91E068EC930E94B027EFABAB
:10E5F600E07111F40C941773E0E0E093D714A0EEE9
:10E60600B4E1EC91E160EC930E94C679E23010F03F
:10E616000C941473A0914D13A03011F00C94147344
:10E6260001C002C00E941B8BEFA9E07211F40C948A
:10E636003473E0E0E093D714A0EEB4E1EC91E2602D
:10E64600EC930E94C679E23010F00C943173A091DD
:10E656004D13A03011F00C94317301C002C00E941A
:10E666001B8BEFA9E07411F40C944173E0E0E09386
:10E67600D714A0EEB4E1EC91E460EC93EFA9E07856
:10E6860011F40C944E73E0E0E093D714A0EEB4E1DD
:10E69600EC91E860EC930E945554EFABE03011F436
:10E6A6000C945D73E0E0E093D714A0EEB4E1EC9136
:10E6B600E061EC930E94DFA6EFABE03011F40C941E
:10E6C6006C73E0E0E093D714A2EEB4E1EC91E16064
:10E6D600EC930E941756EFABE03011F40C947B7369
:10E6E600E0E0E093D714A2EEB4E1EC91E260EC93A3
:10E6F6000E947165EFABAFA9A13010F40C9487733B
:10E70600E853E093F31203C0E1E0E093F312EFA9BC
:10E71600E17011F40C949773E0E0E093D714A0EE47
:10E72600B4E1EC91E061EC93EFA9E27011F40C9482
:10E73600A473E0E0E093D714A0EEB4E1EC91E062BC
:10E74600EC93EFA9E47011F40C94B173E0E0E0935C
:10E75600D714A0EEB4E1EC91E064EC93E091D71409
:10E76600E03011F00C94BA73A4E00E942310A0913B
:10E77600D814A43011F00C94C573E1E0F0E0E8AFD2
:10E78600F9AF0FC0A091D814A13011F00C94D0733A
:10E79600EEE1F0E0E8AFF9AF04C0E3E0F0E0E8AFA7
:10E7A600F9AFA4E00E943F108F01E8ADF9AD0E1756
:10E7B6001F0710F40C94E673A0E00E94D8270E946D
:10E7C600927400E010E00E946E520E94FC80A1E06C
:10E7D6000E944C2EACE00E94F40F8F010536E0E05B
:10E7E6001E0710F40C94FA73ACE00E94DD0FC6CD40
:10E7F6009901AA01EA96FFCFE0E0E3BF0E945B0D14
:10E806000E94F574E1E0E093DA14E093D814A2E7ED
:10E81600B7E080E090E00E94799A0E9498650E9495
:10E82600D68A0895E0E0E3BF0E94890D0E94F57440
:10E83600E1E0E093DA14E2E0E093D814AFE7B7E062
:10E8460080E090E00E94799A0E9498650895E0E041
:10E85600E3BF0E94B70D0E94F574E2E0E093DA147C
:10E86600E3E0E093D814ADE8B7E080E090E00E94E2
:10E87600799A08950A93E0E0E3BF0E94E50DE3E08C
:10E88600E093DA14E4E0E093D8140E94DD74E0919A
:10E896006B16EF5FE0936B16E0916C16EF5FE093FB
:10E8A6006C16A0916B16A93310F40C946C74AAE93B
:10E8B600B7E080E090E00E94799AE7E0E093D81410
:10E8C600A1E00E947527E0E0E0936B160E94986530
:10E8D6000CC0A0916B16A83310F40C947874A1E0C8
:10E8E6000E947527E6E0E093D8140E9471650E2F0A
:10E8F600013010F40C9484740E949865E5E0E0936E
:10E90600D8140991089508950E94D912089508957A
:10E9160008950E9417BC08950E9417BC0895F894A4
:10E92600A2EBB7E080E090E00E94799AA1E00E9415
:10E936009127A0E00E946B27A0E00E947527E0E0E7
:10E94600E093D814E093D9140E9414610E94A93967
:10E956000E94E1100E94D60E0E94D5130E947115E6
:10E966000E945E170E94C118E0E9E0BF0E94D60C23
:10E976000E94D90E0E944927A0E00E940C2EE0E8D2
:10E98600E0936100E8E0E0936100A2E00E94360DAA
:10E99600A2E00E94640DA2E00E94920DA2E00E94F5
:10E9A600C00DE0E0EBB9EAB978940E94EDAC0E94A4
:10E9B600F1AC08950E9424BC0E942575A4E00E9433
:10E9C6002310E0E0E093D914E093DB140E948B0F50
:10E9D60078940E945995ADEBB7E080E090E00E94F4
:10E9E600799A08950E9424BCA1E00E946B270E9498
:10E9F60025750E9426810E9423380E94BB39A1E01A
:10EA06000E94DD0FA4E00E942310A1E00E944C2E7C
:10EA16000E94D4520E948B0E0E949210E1E0E09375
:10EA2600D914E0E0E093DB140E94D90E0E948B0F0C
:10EA360078940E945995A8ECB7E080E090E00E9497
:10EA4600799A08950E9405C20E9419BB0E2F0230C2
:10EA560010F40C943375A8EDB0E0E1E00E94C8C351
:10EA66000E941EBB1E2F113010F40C943F751930F6
:10EA760010F00C943F7506C0A9EDB0E0E2E00E94EC
:10EA8600C8C312E00E9423BB2E2F2F3411F40C941E
:10EA960055752E3411F40C945575253411F40C94D7
:10EAA600557501C006C0AAEDB0E0EEE40E94C8C3E9
:10EAB6002EE40E941EBBE53011F40C946775A9ED97
:10EAC600B0E0E5E00E94C8C30E9423BBEE3411F417
:10EAD6000C947275AAEDB0E0EEE40E94C8C3E12F73
:10EAE600E03011F00C94797540E025C0E13011F06A
:10EAF6000C947F7541E01FC0E23011F00C948575CF
:10EB060042E019C0E33011F00C948B7543E013C05A
:10EB1600E43011F00C94917544E00DC0E53011F02D
:10EB26000C94977545E007C0E63011F00C949D757E
:10EB360046E001C040E0E22FE53411F00C94A575E3
:10EB460031E00DC0EF3411F00C94AB7532E007C024
:10EB5600EE3411F00C94B17530E001C030E00E9443
:10EB66009BB60E944E13A1E00E94FA270E94D76529
:10EB76000E94F8680E9496B20E940CC225960895DB
:10EB86000A930E942575E1E0E093C4160E94E613FD
:10EB960000E0043510F00C94D875E02FF0E0E3594E
:10EBA600F94EA0E0A0830F5FF4CFE0E0E093C1163A
:10EBB600E093C216E093C3160E945A2DE093C51641
:10EBC6000E94742DE093C616E0E0E0936117A6E07C
:10EBD6000E942310099108950E9407C200E00E9436
:10EBE60082760E2FA2E0B0E00E94650F013011F090
:10EBF6000C941676E1E0E093C2160E9402771E2F6F
:10EC0600A12F0E940979103011F00C940D760E9404
:10EC1600127801C020E00E943E78E0E0E093C21640
:10EC26000E9404B308950E9437790E2F003011F424
:10EC36000C9420760E9404B308950E9423B408958C
:10EC46000A930A2F000F000F000F08710093181780
:10EC5600E0911717E260E0931717099108950A9358
:10EC66000A2F0295007F000F007600931817E09197
:10EC76001717E460E0931717099108950E9405C2DB
:10EC86009D014D8140932017E091CF16F091D0164B
:10EC9600E0931C17F0931D17E091D116F091D21650
:10ECA600E0931E17F0931F17E42FF0E0FA93EA9310
:10ECB600A0E4B0E00E9456231E2F00E0011710F0DA
:10ECC6000C946F76A1E2B7E1E02F0E9478B1D901EA
:10ECD6000E9430BC0F5FF2CF0E940CC226960895A8
:10ECE6000A930A2F043610F00C947D76E1E0E09347
:10ECF600611703C0E0E0E0936117099108950E944F
:10ED060007C20E9470148F01112312F00C948E76A4
:10ED16000E9437BC08950635E0E01E0714F40C94F3
:10ED260097760E9437BC089500240016010614F059
:10ED36000C94E57620E0243510F00C94AA76E22FA8
:10ED4600F0E0E359F94EA0E0A0832F5FF4CFEDE6A3
:10ED5600F6E1FA93EA93A4E5B0E00E9473140093F7
:10ED6600C116E091C116A0916217EA1711F40C942E
:10ED7600C376ACE10E94DD0FE091C116E093621705
:10ED8600A091C116AA3010F40C94D076A0916D16FD
:10ED9600AF3311F00C94D07601C003C00E943EBC84
:10EDA6000895A091C116A63410F40C94E176A091B2
:10EDB6006D16AD3311F00C94E17601C003C00E94CC
:10EDC6003EBC0895ACE10E94F40F8F010530E0E0EF
:10EDD6001E0714F40C94F676A0916217A13010F475
:10EDE6000C94F67601C008C00E94E613E0E0E093BA
:10EDF60062170E9409B308950E9423B408952297CA
:10EE06000E9489B1E0E0E093C716E0E0F0E0E0930D
:10EE1600C816F093C916E093CA16F093CB16E09382
:10EE2600CC16F093CD16EFEFE093CE16E0E0F0E0CF
:10EE3600E093CF16F093D016E093D116F093D21646
:10EE4600EFEF0E9445BCE0E0E093D61640E050E0CC
:10EE56004034E0E05E0710F00C943A77E7EDF6E117
:10EE6600E40FF51FA0E0A0834F5F5F4FF1CFA091A5
:10EE76006D16AD3311F40C944577AF3311F40C9441
:10EE8600457701C005C0E1E00E940BC228960895AF
:10EE9600A0916D16AD3311F00C945877A091C11660
:10EEA600A63410F00C9458770EC0A0916D16AF33AF
:10EEB60011F00C946577A091C116AA3010F00C944D
:10EEC600657701C005C0E2E00E940BC2289608954E
:10EED600E0E0EF83A0916D16AD3311F00C947677D8
:10EEE600E0E4EF8308C0A0916D16AF3311F00C94E7
:10EEF6007E77E4E0EF83EF81EA5FEE83E150F0E0B6
:10EF0600E359F94EE081EA93EF81E250F0E0E359EC
:10EF1600F94EA0810E94B5219F01EE81E250EE8359
:10EF260040E050E0EE810E9400B510F00C94A67708
:10EF3600ADE6B6E1A40FB51FEC91F0E00E0F1F1F72
:10EF46004F5F5F4FEFCF2017310711F40C94B27764
:10EF560040E050E0E4E00E940BC228960895A0919C
:10EF66006D16AD3311F00C94BB77E2E0E093C71653
:10EF7600A0916D16AF3311F40C94C477E1E0E093E1
:10EF8600C716E1E0F0E0E093C816F093C916AAECC4
:10EF9600B6E1E0916E16F0E0ED93FC93ACECB6E1D1
:10EFA600E0917016F0E0ED93FC93E0E0E093CE166E
:10EFB600AFECB6E1E0916F16F0E0ED93FC93E091D3
:10EFC600CC16F091CD16E093D116F093D216E0E070
:10EFD6000E9445BCEF81E093D616A091D616A134C7
:10EFE60010F40C94F977E0E4E093D61640E050E094
:10EFF600E091D6160E9400B510F00C940F78E7ED5C
:10F00600F6E1E40FF51FDF01FA01EF58F94EE08152
:10F01600EC934F5F5F4FECCF0E94DAB408950A93EA
:10F0260000E0E091CA16F091CB16FA93EA93E091CC
:10F03600CC16F091CD16FA93EA93E091D616EA93A0
:10F04600A7EDB6E10E94FB680E2FA02F0E94237643
:10F0560000E0E091CF16F091D016FA93EA93A091D2
:10F06600D116B091D2160E94DA650E2FA02F0E94FB
:10F07600327609910895EF9765970E9405C2E0914F
:10F086001717E03011F00C944E78E0E00E940CC2A5
:10F09600EF966A960895E0E0EF83E887AF81B8853A
:10F0A600A035E0E0BE0710F00C945E780E944EBCDE
:10F0B6000E9453BCF3CFE0916117E03011F00C943D
:10F0C6006878EFE5E98708E003C0EDE5E98700E445
:10F0D600A09120170A1710F00C947378009320174C
:10F0E600E0911817EA87E0E0EF83E887E0912017C0
:10F0F6000E94CFB910F00C949278EF81F885329681
:10F10600ED83FE830E9459BC0F01E1E2F7E10E9404
:10F11600D9AEEC91D001EC930E9453BCE7CF0E948C
:10F126005EBCED81FE81EF83F887E02FEE5F0E94E3
:10F13600CFB910F00C94A4780E944EBC0E9453BC28
:10F14600F4CFE02FF0E032961E2F2F2F30E040E074
:10F15600E0E0EF83E887AF81B885A117B20710F02A
:10F166000C94C278EF81F885DE011996AE0FBF1FA9
:10F17600EC91F0E03E0F4F1F0E9453BCECCFE12F05
:10F18600F22F0E9459BC3083342F4427E12FF22FEF
:10F1960031960E9459BC30831E5F2F4FA985AD352D
:10F1A60011F00C94DC78AA85A03211F00C94DC786E
:10F1B60001C004C0E1E0F0E0EF83F887E4E4F0E0AA
:10F1C600E117F20711F40C94F078ECE0F0E0E117A7
:10F1D600F20711F40C94F07807C00E9496B6A12F9E
:10F1E600B22F0E94C01403C0E0E0EF83E8870E94BC
:10F1F60028B4E0E0E0931717EF81F885EF83F887EE
:10F20600E1E00E940CC2EF966A9608951A930A935B
:10F216001A2F10931817E3E6E0931917E0931A17BD
:10F22600E0E0E093201700E0003410F00C9423791E
:10F23600A1E2B7E1EE27A00FBE1FEC930F5FF4CF5C
:10F24600E0911817E03011F00C942F79E091171720
:10F25600E160E093171705C0E0911717E161E093AD
:10F266001717099119910895A091C116AE3010F49F
:10F276000C949F79A0916D16A23011F00C9492799E
:10F28600A0916E16A13511F00C949279A0916F168B
:10F29600A33411F00C949279A0917016A23211F059
:10F2A6000C949279A0917116A53511F00C9492796F
:10F2B600A0917216AB3511F00C949279A091731649
:10F2C600AD3211F00C949279A0917416A43311F01A
:10F2D6000C949279A0917516A23411F00C9492793F
:10F2E600A0917616AD3411F00C949279A091771610
:10F2F600A83511F00C949279A0917816A23D11F0E0
:10F306000C949279A0917916A33D11F00C94927900
:10F31600A0917A16A33011F00C94927901C00CC01A
:10F32600A2EDB7E080E090E00E94799A0E9469B36E
:10F336000E94070EE1E00895E0E008950E9404C2ED
:10F3460000E210E04EED52E120E030E0DA01E0E0CC
:10F35600EC934F5F5F4FF90131969F01E017F1077C
:10F3660010F00C94B779F2CF0E940BC2269608953E
:10F37600E0E0E0936317E09364170E945995E3E693
:10F38600E09365170895E09164170895E2E0E0932D
:10F396006417E0E008950E9464BCA0E00E946E2914
:10F3A600A0E00E949F29A0E00E9489290E94218B4B
:10F3B6000895AA9325970E9404C2EB85E03011F4C4
:10F3C6000C94E8790E9468BC0895E0916317E030D8
:10F3D60011F00C94F1790E946DBC17C0E13011F068
:10F3E6000C94F8790E9473BC10C0E23011F00C94B2
:10F3F600FF790E94B6AC09C0E33011F00C94047A90
:10F4060004C0E43011F00C94087AA0916317AF5F42
:10F41600A0936317A53010F40C94147AE0E0E093FF
:10F4260063170E94718DE03011F40C94577AA6E6AA
:10F43600B7E10E944E8D5E2FE0916417E03011F423
:10F446000C942E7A513010F40C942E7A5A3010F017
:10F456000C942E7A01C015C0E0E0E0936417A0E09A
:10F466000E9452640E94F1BA0E9459950E9464BC9F
:10F47600AAEEB7E080E090E00E94799A0E94908D13
:10F4860013C0533011F00C944E7AE1E0E093641708
:10F496000E94908D09C0543011F00C94577AE2E026
:10F4A600E09364170E94908DA0916417A13011F02B
:10F4B6000C94657A0E9459950E94BE80E0E0E09324
:10F4C6006417BAC0A0916417A23011F00C94937A15
:10F4D6000E945995A9EFB7E080E090E00E94799AE2
:10F4E600A6E1B8E080E090E00E94799AADE3B8E04A
:10F4F60080E090E00E94799AAEE00E942310E091AD
:10F506006417EF5FE09364170E94BB390E940640C0
:10F51600A1E00E944D400E946D640E94EBBA8CC02F
:10F52600A0916417A33011F00C94097BAEE00E9401
:10F536003F109F012531E0E03E0710F40C94A87AB5
:10F54600E0916417EF5FE09364170E944A404E2FE4
:10F55600483011F00C94B17A0E947140E091651721
:10F56600E41711F40C94D97A409365170E945995C3
:10F57600483011F00C94C57AA2E5B8E080E090E03E
:10F586000E94799A493011F00C94CF7AA4E6B8E03B
:10F5960080E090E00E94799A4A3011F00C94D97A72
:10F5A600ADE6B8E080E090E00E94799AFE013A96D6
:10F5B600FA93EA93FE013B960E944CB1FE013D96FA
:10F5C600FA93EA93DE011E960E943F414E2F403089
:10F5D60011F00C94087B0E811127AFEFA09FF0016C
:10F5E600A19FF00D8F01EF81F0E00E0F1F1FE3E8E2
:10F5F600F8E060E070E00E9497C3D8010E9491B5E0
:10F606000E944F9AAEE00E94231016C0A091641784
:10F61600A43011F00C941F7BA0E00E9452640E945B
:10F62600F1BA0E9464BCAEE8B8E080E090E00E94C7
:10F63600799AE0E0E09364170E9468BC0895E69723
:10F646000E9405C200E00E9479BC0E944F9A0E9467
:10F6560079BCACE9B8E080E090E00E94799AA0918C
:10F66600DF12A13011F00C943F7BA5EBB8E080E0EF
:10F6760090E00E94799A06C0ACEBB8E080E090E09A
:10F686000E94799A1091E312113011F00C94527B7A
:10F69600ACECB8E080E090E00E94799A06C0E8ED14
:10F6A600F8E060E070E00E947DBC0E94567E1E2F4E
:10F6B600113010F40C94677B01E0E8EEF8E060E0AE
:10F6C60070E00E947DBC06C0A3EFB8E080E090E049
:10F6D6000E94799A0E948A7E1E2F103011F40C9493
:10F6E6007C7B01E0EAEFF8E060E070E00E947DBC20
:10F6F60006C0A5E0B9E080E090E00E94799A0E94F9
:10F7060033652E2F203011F40C948F7BACE0B9E0DA
:10F7160080E090E00E94799A0E9449653E2F303041
:10F7260011F40C949C7BAFE1B9E080E090E00E947C
:10F73600799A0E945F654E2F403011F40C94A97B94
:10F74600A2E3B9E080E090E00E94799A203011F0BF
:10F756000C94B67B303011F00C94B67B403011F02F
:10F766000C94B67B01C006C0A7E4B9E080E090E047
:10F776000E94799A0E9407540E9420B90E94ED7E49
:10F786001E2F103011F40C94D07B01E0E0E5F9E077
:10F7960060E070E00E947DBC06C0A3E6B9E080E0B0
:10F7A60090E00E94799A0E9417540E9420B90E9404
:10F7B600BC7E1E2F103011F40C94E97B01E0E2E7C9
:10F7C600F9E060E070E00E947DBC06C0A1E8B9E007
:10F7D60080E090E00E94799A0E94ED7D1E2F103005
:10F7E60011F40C94FE7B01E0ECE8F9E060E070E0D7
:10F7F6000E947DBC06C0A9E9B9E080E090E00E94C5
:10F80600799A0E94167E1E2F103011F40C94137CE8
:10F8160001E0E2EAF9E060E070E00E947DBC06C02B
:10F82600AFEAB9E080E090E00E94799A0E94A17D5B
:10F836001E2F103011F40C94287C01E0E8EBF9E05F
:10F8460060E070E00E947DBC06C0ABECB9E080E0F1
:10F8560090E00E94799A0E9441561E2F123010F4B1
:10F866000C94587C01E0EAEDF9E060E070E00E945B
:10F876007DBC11FF02C00E9481BC15FF02C00E9420
:10F8860087BC17FD03C016FD01C003C00E948DBCD6
:10F896000BC012FD03C014FD01C002C00E9493BC40
:10F8A60013FF02C00E9499BC06C00E949FBC10FFB5
:10F8B60002C00E94A5BC0E94EF641E2F103011F0FA
:10F8C6000C94707CE8ECE093EE1201E0A8E4BAE058
:10F8D60080E090E00E94799A09C0E1E0E093EE12A0
:10F8E600A5E5BAE080E090E00E94799A0E94116551
:10F8F6001E2F103011F40C948A7CE8ECE093EF1282
:10F90600A2E6BAE080E090E00E94799A09C0E1E0C0
:10F91600E093EF12AEE6BAE080E090E00E94799ABA
:10F926000E94BB390E943D401E2F113010F40C94EA
:10F93600A77CE8ECE093E81201E0AAE7BAE080E0F1
:10F9460090E00E94799A09C0E1E0E093E812A4E809
:10F95600BAE080E090E00E94799AE1E0E093F71245
:10F96600E0E0E093EB120E941B8BADE10E94DD0FFD
:10F97600ADE10E94F40FED83FE831091EB120E941D
:10F986002B8BAD81BE81A039E1E0BE0710F00C944F
:10F99600D17C103011F00C94D17C01C001C0E8CFAD
:10F9A6000E945995113011F00C94E07CABE8BAE056
:10F9B60080E090E00E94799A07C001E0E8E9FAE069
:10F9C60060E070E00E947DBCA9EABAE080E090E0C9
:10F9D6000E94799AA0E00E9461841E2F0E94768080
:10F9E600A091E812A83C10F40C94FD7CE8ECE0939E
:10F9F600E91239C0E0E0E093E9120E940640A1E076
:10FA06000E944D400E947140ADE10E94DD0FADE1C4
:10FA16000E94F40FED83FE831091E9120E9476385E
:10FA26000E946B3DAD81BE81A83EE3E0BE0710F0AB
:10FA36000C94227D103011F00C94227D01C001C07F
:10FA4600E6CF113011F00C942F7DA5ECBAE080E0E2
:10FA560090E00E94799A07C001E0E5EDFAE060E0E7
:10FA660070E00E947DBC003011F40C94447DA5EE3C
:10FA7600BAE080E090E00E94799AA1E00E947527A2
:10FA860009C0A4EFBAE080E090E00E94799AA1E074
:10FA96000E946B27E1E0E093F9120E944F9A0E94C0
:10FAA60096B60E9475BAE8ABEEEFFAE060E070E059
:10FAB6000E94ABBC0E94EC1CE4E1FBE060E070E05D
:10FAC6000E94ABBC0E94D79A0E9496B60E9475BA55
:10FAD600E8ABE0E2FBE060E070E00E94ABBC0E94B5
:10FAE600EC1CEDE2FBE060E070E00E94ABBC0E9423
:10FAF600D79A0E9496B60E9475BAE8ABE9E3FBE096
:10FB060060E070E00E94ABBC0E94EC1CE6E4FBE007
:10FB160060E070E00E94ABBC0E94B0BCE1E0E09304
:10FB2600EC12E0E0E093F2120E945995A7E00E94E1
:10FB36002310E02F0E940CC2EB9608951A930A93A5
:10FB460000E0E0E0E093EA120E94B3BA1E2F113003
:10FB560010F40C94DE7D0E94012AE03011F40C941E
:10FB6600B57D01E0A1E00E94C7290E9412B80E945B
:10FB7600012AE03011F00C94C17D02E0A0E00E9461
:10FB8600C7290E94B4BCA1E00E94DD290E9412B8D8
:10FB96000E94012AE03011F00C94D27D03E0A0E02F
:10FBA6000E94DD290E94B4BC0E94012AE03011F4B3
:10FBB6000C94DE7D04E0013010F40C94E67DE8EC54
:10FBC600E093EA1203C0E1E0E093EA12E02F099124
:10FBD600199108950A93EFEFFFE0FA93EA93A9E7E4
:10FBE6000E94B8BC093711F40C94FF7DE8ECE09351
:10FBF600E012E1E009910895EFEFFFE0FA93EA934E
:10FC0600A6E80E94B8BC063811F40C94107EE8EC05
:10FC1600E093E012E1E009910895E1E0E093E0125B
:10FC2600E0E0099108950A93A0E00E9491270E94BE
:10FC360034B2EEEFFFEF0E944FBAA2E10E94258692
:10FC46000E2F0E946DB30E94C0BC023111F40C94B9
:10FC5600327EE8ECE093E112E1E009910895EEEFDF
:10FC6600FFEF0E944FBAA7E30E9425860E2F0E943F
:10FC76006DB30E94C0BC073311F40C94487EE8ECC7
:10FC8600E093E112E1E009910895E1E0E093E112E9
:10FC9600E0E0099108950E9466B80895AEE1B0E0EB
:10FCA6000E94650F089562970A93DE0111960E94DD
:10FCB600E84E0E2F023010F40C946F7E0E9496B21E
:10FCC6000E94C1B2AFE10E94C5500E9496B2DE0109
:10FCD60011960E94E84E0E2F003011F00C94777E9C
:10FCE600E1E0E093E2120FC0013011F00C947F7E48
:10FCF600E8ECE093E21207C0023011F00C94867E25
:10FD0600E9ECE093E212E02F088163960895A89744
:10FD16000A93FE0177960E94CBBC0E9492510E2F49
:10FD2600003011F40C94987E04C0E02F0881A99647
:10FD360008950881A99608950E9406C220E0A1E0D0
:10FD46000E947F270E94517E0E946DBC3E2F31305B
:10FD560010F40C94AF7E21E00E9473BC3E2F31302C
:10FD660010F40C94B77E21E0E22F0E940DC2249677
:10FD760008950E94D0BC0832E3E21E0710F40C94EA
:10FD8600CB7E0939EAE31E0710F00C94CB7E05C042
:10FD960021E0E8ECE093F01218C00033EAE21E0717
:10FDA60010F00C94DB7EE9ECE093F01222E00DC03B
:10FDB600003CEBE21E0710F00C94E57EE4E6E093CF
:10FDC600F01203C0E1E0E093F012E22F0E940EC2AF
:10FDD600259608950E94D0BC0832E0E01E0710F474
:10FDE6000C94FC7E0530E1E01E0710F00C94FC7EBE
:10FDF60005C021E0E8ECE093F11215C00135E0E022
:10FE06001E0710F40C940E7F0C3DE0E01E0710F068
:10FE16000C940E7F05C022E0E9ECE093F11203C0DA
:10FE2600E1E0E093F112E22F0E940EC225960895BA
:10FE36001A930A9300E00E940A29E03011F40C9408
:10FE4600297FA0E00E94FE280E94517EA1E00E9428
:10FE5600FE280E944E7E0E941029E03011F00C947C
:10FE6600357F01E0013010F40C943D7FE02F0991BD
:10FE7600199108950E94222EE03011F40C94487FC7
:10FE8600A0E00E940C2E0E94517EA0E00E940C2E43
:10FE96000E944E7EA1E00E940C2E0E944E7E0E9481
:10FEA600AD2EE03011F00C94597F02E0013010F4D1
:10FEB6000C94617FE02F099119910895A0E00E94AA
:10FEC600D8BC11F40C94687F03E0A1E00E94D8BC72
:10FED60011F00C946F7F03E0A0E00E94E5BC11F4E2
:10FEE6000C94767F03E0A1E00E94E5BC11F40C942B
:10FEF6007D7F03E0013010F40C94857FE02F09919B
:10FF060019910895A0E00E94F2BC11F00C948C7F28
:10FF160004E0A1E00E940C2EA1E00E9489290E9423
:10FF26004E7EA1E00E94F2BC11F40C949B7F04E08B
:10FF3600013010F40C94A37FE02F099119910895D4
:10FF46000E947A29E03011F40C94AE7FA0E00E9462
:10FF56006E290E94517EA0E00E94FABC11F40C9416
:10FF6600B57F05E0A1E00E94FABC11F00C94BC7FBD
:10FF760005E0013010F40C94C47FE02F099119912B
:10FF860008950E94AB29E03011F40C94CF7FA0E0D5
:10FF96000E949F290E94517EA0E00E9402BD11F49A
:10FFA6000C94D67F06E0A1E00E940C2EA1E00E94F0
:10FFB60002BD11F00C94E07F06E0013010F40C94C1
:10FFC600E87FE02F0991199108950E94982CE0305E
:10FFD60011F40C94F37FA0E00E94822C0E94517EC3
:10FFE600A0E00E94822C0E944E7E013010F40C94F8
:0AFFF6000080E02F09911991089591
:020000021000EC
:060000000E947F2EE0309B
:1000060011F40C940B80A0E00E94732E0E94517E86
:10001600A0E00E94732E0E944E7EA1E00E94732EE5
:100026000E944E7E0E948F2EE03011F00C941C80B0
:1000360009E0013010F40C942480E02F0991199105
:1000460008950E94422EE03011F40C942F80A0E017
:100056000E942C2E0E94517EA0E00E942C2E0E940F
:100066004E7EA1E00E942C2E0E944E7E0E94A42E5F
:10007600E03011F00C9440800AE0013010F40C944A
:100086004880E02F099119910895A1E00E944C2E15
:100096000E944E7E0E94622EE03011F00C94548035
:1000A6000BE0013010F40C945C80E02F099119915B
:1000B6000895A0E00E940BBD11F40C9463800CE03F
:1000C600A1E00E940BBD11F00C946A800CE0013097
:1000D60010F40C947280E02F099119910895E02F85
:1000E600099119910895A091E512A13011F00C948F
:1000F6009580A2E5BBE080E090E00E94799AA0910D
:10010600E712A13011F00C948E80ABE5BBE080E0E5
:1001160090E00E94799AE6E6FBE060E070E00E94DB
:1001260014BD28C0AEE6BBE080E090E00E94799A5C
:10013600E091E512E83C11F00C94A880A5E0BAE045
:1001460080E090E00E94799A15C0E93C11F00C9489
:10015600B380ABE7BBE080E090E00E94799A0AC0EA
:10016600E43611F00C94BD80A6E8BBE080E090E098
:100176000E94799A08950A93A4E9BBE080E090E092
:100186000E94799A0E9441560E2F023010F40C9468
:10019600F280EAEDF9E060E070E00E9497C30E9409
:1001A600ABB70E94269B01FF02C00E9481BC05FFDF
:1001B60002C00E9487BC07FD03C006FD01C003C044
:1001C6000E948DBC0BC002FD03C004FD01C002C02D
:1001D6000E9493BC03FF02C00E9499BC08C00E9403
:1001E6009FBC00FF02C00E94A5BC0E947F560991D9
:1001F60008951A930A93A1E00E942FB910F40C9463
:100206000B81A0E00E946B27A1E00E94DD0F09C0D0
:100216000B35E0E01E0710F40C941481A1E00E9457
:100226006B27099119910895E091E514E03011F0DA
:100236000C9425810E9419BD0E949BB60E94D6147B
:100246000E9482150895E091E514E03011F00C94B7
:100256003D810E943E810E941781A1E00E94732E7B
:100266000E9434B2E0E0E0936E17E0936F17EFEF71
:10027600E0937017089508950E94CBB811F40C947A
:1002860047810E94D0B80895E091E514E03011F45A
:100296000C9450810E94D0B80895E0916E17A091F9
:1002A6007017EA1711F40C945D81E0937017E1E082
:1002B600E0936F17E0916E17E03011F00C947B819C
:1002C600E0916F17E03011F40C946E810E941FBD0F
:1002D60040E00E9417810E9425BD10F00C947881A1
:1002E600403011F00C94788102C00E942DBD87C069
:1002F600A0916E17A13011F00C94A281E0916F17B6
:10030600E03011F40C948E810E941FBD0E949C82E5
:1003160040E00E9419BD0E9457828F01D8010E94B9
:10032600CF824E2F0E9425BD10F00C949F81403045
:1003360011F00C949F8102C00E942DBD60C0A09157
:100346006E17A23011F00C94C681E0916F17E03061
:1003560011F40C94B2810E941FBD0E94AD820E94CE
:1003660057828F01D8010E9411834E2F0E9425BD0E
:1003760010F00C94C381403011F00C94C38102C07C
:100386000E942DBD3CC0A0916E17A33011F00C94B5
:10039600E281E0916F17E03011F40C94D5810E9450
:1003A6001FBD40E00E9436BD10F00C94DF81403046
:1003B60011F00C94DF8102C00E942DBD20C0A091D7
:1003C6006E17A43011F00C940282E0916F17E030A2
:1003D60011F40C94F1810E941FBD40E00E9436BDCD
:1003E60010F00C94FB81403011F00C94FB8106C098
:1003F600E0E0E0936E17E1E0E0936F1700C00E9423
:10040600D0B80895A0970E9405C200E010E020E051
:10041600E091E514E03011F40C9415820E947DAD54
:10042600A59608950E9496B20E945716E03011F4E0
:100436000C9443820E9403161E2F2F2FA12FB22F3A
:100446000E943EBD11F40C942B82E12FF22F02C0C4
:10045600E0E2F0E03E2F4F2F00240116020614F0D2
:100466000C9441820E943BB4A32FB42F0E942816FD
:100476000E943BB4A32FB42F0E94E2880E948215EB
:100486000F5F043610F00C944F820024011602060A
:1004960011F00C944F8201C001C0C4CFE12FF22F9E
:1004A6000E940CC2A5960895EF9721970E9406C256
:1004B60000E010E0E091E514E03011F40C946A825B
:1004C600E0E0F0E00E940DC2EF96259608950E94A6
:1004D6005716E03011F40C9496820E9403168F0191
:1004E600D801E0E4F0E00E94B2C2F0E0E03011F49E
:1004F6000C947F82F80102C0E0E4F0E09F01002442
:100506000016010614F00C949482FE013496FA93B8
:10051600EA93D9010E9428160E9445BDD9010E947E
:10052600E2880E948215F8010E940DC2EF96259678
:100536000895E091E514E03011F00C94AC820E942D
:1005460019BD0E948215A8EABBE080E090E00E94F7
:100556004ABD0895E091E514E03011F00C94BD8297
:100566000E9419BD0E948215AFEABBE080E090E0D0
:100576000E944ABD0895E091E514E03011F00C9414
:10058600CE820E9419BD0E948215A8EBBBE080E0D6
:1005960090E00E944ABD089526970E942EAD0E94C3
:1005A6004FBD11F40C94DA820E9454BD08951B309D
:1005B600E0E02E0710F40C940E83E2ECFBE060E022
:1005C60070E00E9497C32A931A930E9459BD11F4B2
:1005D6000C940E830E94F5B9A3E00E94588AAD815F
:1005E600AC3211F00C940583EB81E053AAE0EA9F4C
:1005F600F001AC81AE0FE0E30E94A4C3EA1BE093D6
:10060600E61204C0EB81E053E093E612E1E00E94BB
:100616000EC2299608950E9454BD089526970E94F9
:100626002EAD0E944FBD11F40C941C830E9454BD44
:1006360008951B30E0E02E0710F40C945783E9EC84
:10064600FBE060E070E00E9497C32A931A93A0E053
:100656000E9428890E2F003011F40C9457830E94B3
:10066600F5B9A3E00E94588AAB81A03311F00C942F
:100676004C83AC81AC3211F00C944C83AD81A13328
:1006860011F40C944B83A53311F40C944B8301C0E5
:1006960001C007C0E1E0E093E7120E940EC229966E
:1006A6000895E4E6E093E7120E9454BD0895AA93E4
:1006B600A2970E9404C238A5E091E514E03011F437
:1006C6000C946A83E0E00E940BC2A99608950E94EA
:1006D60019BD313011F00C9475830E949BB60E94AF
:1006E600D6143DC0323011F00C948183E2E0EA93D7
:1006F600EA930E9490B20E94D61431C0333011F0B2
:100706000C948E83E2E0EA93E3E0EA930E94B8B4A5
:100716000E94D61424C0343011F00C9499830E94A0
:100726008BB20E9490B20E94D61419C0353011F0D7
:100736000C94A683E2E0EA93E1E0EA930E9490B289
:100746000E94D6140CC0363011F00C94B283E2E04D
:10075600EA93E4E0EA930E9490B20E94D6140E94C3
:1007660082150E94B4BC00E00E94B4BCFE0138961B
:100776000E9416B80E9486B70E948215A1EDBBE0C2
:1007860080E090E00E944ABD10E0A8E0B0E00E9440
:10079600650F0E945716E03011F40C9408840E94ED
:1007A6000316AF01DA010E943EBD11F40C94DD83FD
:1007B600FA0102C0E0E2F0E0EE83FF8300240416B3
:1007C600050614F00C9406840E9463BAA885B985C0
:1007D6000E9428160E9463BAA885B9850E94E288FD
:1007E6000E945FBDEA85FB85FA93EA93A0E00E942A
:1007F60028892E2F203011F40C940684E32F0E94B2
:100806000BC2A99608950E9482151F5F143610F038
:100816000C941284203011F00C94128401C001C093
:10082600B4CF0F5F063010F00C941E84203011F008
:100836000C941E8401C001C097CFE0E00E940BC259
:10084600A99608951A930A930E944FBD11F40C9429
:100856003084E0E009911991089511E0A12F0E94DA
:100866005A830E2F1F5F163010F00C943F84003011
:1008760011F00C943F8401C001C0F0CFE02F099124
:10088600199108950A93E091E514E03011F40C945F
:100896005F840E9419BD0E94821501E0A7EDBBE0AE
:1008A60080E090E00E944ABD0E94B4BC0F5F033016
:1008B60010F00C945F84F2CF09910895A0970E94DE
:1008C60004C25A2F20E0E091E514E03011F40C94B4
:1008D6007184E0E00E940BC2A69608950E942681CC
:1008E6000E9419BDA8EEB3E00E94650F0E94258400
:1008F6002E2F0E9434B2203011F00C948684E8EC3E
:100906000E9466BD0895E1E0E093E5120E944584E9
:1009160000E00E9417810E94B4BC0E949BB70E940F
:100926006DBD0E948215A5EEBBE080E090E00E94BE
:100936004ABD0E9470BD0E946DBD0E948215AAEE3E
:10094600BBE080E090E00E944ABD0E9470BD0E941C
:100956006DBD0E948215A4EFBBE080E090E00E948E
:100966004ABD0E9475BD3B30E0E04E0710F40C9482
:10097600C984E8EFFBE060E070E00E947ABD11F008
:100986000C94C984E9EC0E9466BD08950E949BB749
:100996000E946DBD0E948215A1E0BCE080E090E05F
:1009A6000E944ABD0E9475BD3530E0E04E0710F446
:1009B6000C94EC840E945FBD4A933A93A0E00E9497
:1009C60028891E2F103011F00C94EC84E4E6E09395
:1009D600E5120E949BB70E946DBD00E0503011F4F5
:1009E6000C94F68403E6ACE2B1E00E94650F0E9427
:1009F6009C820E9475BDA32FB42F0E94CF820F5FE9
:100A0600043110F00C941585A091E612AC3010F468
:100A16000C941485A091E612A03210F00C94148563
:100A260001C001C001C0DFCF0E949BB70E946DBD0F
:100A36000E94AD820E9475BDA32FB42F0E94118320
:100A46000E949BB70E946DBD0E94BE820E9475BD2A
:100A56003B30E0E04E0710F40C943A85EEEAFBE0FA
:100A660060E070E00E947ABD11F00C943A85E0E0F7
:100A76000E940BC2A696089522970E9405C21A2FBD
:100A86002F81388549854A933A93E1E0EA932A9380
:100A96001A93DE011A960E947CB810F40C945885BD
:100AA600E0E00E940CC22A9608950D81E02F0E9474
:100AB6000CC22A96089522970E9405C23A2F4F81AA
:100AC600E885F985FA93EA93E2E0EA934A933A9342
:100AD600DE011A960E947CB810F40C9476850E946A
:100AE6007DAD2A9608951E812227212F1127ED819B
:100AF600F0E01E2B2F2BE12FF22F0E940CC22A961C
:100B0600089528970E9405C21A2F2D853E854F8588
:100B16004A933A93E4E0EA932A931A93DE011E96E7
:100B26000E947CB810F40C949C850E94CCB160960F
:100B36000895EC85FF27662777270E9484BDEB85FD
:100B46000E948DBDEA850E948DBDE9850E949FADFC
:100B56000E9495BD0E94ACAD0E940CC2609608959D
:100B6600BA93AA93EF9727970E9404C2FE01E05B0F
:100B7600FF4F5081FE01EE5AFF4F11912081FE0179
:100B8600E25BFF4F0190F081E02DE887F987E0E016
:100B9600EE83EF832A931A93E0E4EA930E94B0B2BD
:100BA600EA935A93DE011F960E947CB810F40C94C7
:100BB600E285E1E00E940BC2EF9665960895A8854E
:100BC600B985A134E0E0BE0710F40C94FE8530E050
:100BD60040E03034E0E04E0710F00C94F7850E94B8
:100BE6009BBD3F5F4F4FF5CFE885F985E054F04058
:100BF600E887F98711C030E040E0E885F9853E17BF
:100C06004F0710F00C940C860E949BBD3F5F4F4F20
:100C1600F4CFE0E0E887E987EE81FF81E05CFF4FF3
:100C2600EE83FF83105C2F4FA885B9850E94E1C330
:100C360010F00C941F86AECFE0E00E940BC2EF9638
:100C46006596089522970E9404C21A2F2885398531
:100C56004A855B85A5E0B0E00E94430F1E835A9348
:100C66004A93E1E0EA933A932A930E945BB80130F3
:100C760010F40C944386E1E00E940BC22C96089572
:100C86000E9468BC089522970E9404C23A2F4B2FF7
:100C96005885E985E987132F242F1E83122F2227D3
:100CA600FE0137961083EA85FB85FA93EA93E2E024
:100CB600EA93EC85EA935A930E945BB8013010F4EC
:100CC6000C946A86E1E00E940BC22C9608950E945D
:100CD60068BC08950E949CC328970E9405C2398962
:100CE6004A891B892C89ED85FE856F8578890E9446
:100CF60095ADED81E9870E94B0BDEA870E94B0BD3F
:100D0600EB870E94B0BDEC872A931A93E4E0EA933E
:100D16004A933A93DE011E960E94DB110E2F013094
:100D260010F40C949B86E1E00E940CC2659608952F
:100D3600E0E00E940CC2659608950E9404C29D01DF
:100D46004E815F81042F013410F40C94AB8600E4CD
:100D5600E885F985FA93EA930A935A93E1E0EA93D0
:100D6600D9010E94DB111E2F0E946DB3103011F4C1
:100D76000C94C0860E9430AF0895E02F0E940BC2EB
:100D86002A960895BA93AA93EF972F970E9404C2C2
:100D9600FE01E65AFF4F01911081FE01E65AFF4F10
:100DA6000190F081E02D662777270E9443B00E94CC
:100DB600B9BD662777270E94D0B70E9420C20E943D
:100DC600BCB70E94B9BD0E94C0BD40E050E00E9481
:100DD600C6BDA034E0E0BE0710F00C944B8720E0BF
:100DE60030E00E94CDBD2E173F0710F00C9400870F
:100DF6000E94D4BD2F5F3F4FF4CFFE01EE5AFF4F46
:100E0600E081E770EF87E03011F40C940E87AF8530
:100E1600E8E0EA1B01C0E0E0EE8720E030E0EE8586
:100E2600D901F0E0AE17BF0710F00C9425870E9499
:100E3600CDBDE20FF31FDE0150960E941FB82F5F53
:100E46003F4FEDCFEE850E94C6BDF0E0EA0FFB1FD7
:100E56000E94C0BD1A930A930E94B0B20E94E5BDDB
:100E66000E94E5BD0E94EBBDAF85A13010F40C9445
:100E760041870E945CADEF966D9608950E94CDBDA8
:100E8600E40FF51F9F010E940BC2EF966D96089521
:100E960020E030E02034E0E03E0710F00C94588764
:100EA6000E94D4BD2F5F3F4FF5CF1A930A93E0E41B
:100EB6000E94E5BD0E94E5BD0E94EBBDAF85A13055
:100EC60010F40C946B870E945CADEF966D960895B6
:100ED6000E94CDBDE054F0400E94C0BD0E94CDBD31
:100EE600309711F00C947D87FA010E940BC2EF96A1
:100EF6006D960895005C1F4F0E94F3BDE05CFF4FA6
:100F06006F4F7F4F0E9443B0405C5F4F0E941CB101
:100F16000E94D0B70E94F0C310F00C94938757CF6D
:100F26000E945CADEF966D9608950A930A2FE4E150
:100F3600E09FF00109910895BA93AA93AC978CE2C9
:100F4600002470E0ECE0FCE060E00E9412C20E9427
:100F560005C209A91AA9ED81FE81E017F10710F46F
:100F66000C94BA87E0E00E940CC2E396089541E033
:100F7600E42FF0E0DE0115960E94E1B12D913C913F
:100F86000217130710F00C94CE87E42FE1500E944D
:100F96000CC2E39608954F5F453110F00C94D48748
:100FA600E7CFE4E10E940CC2E3960895BA93AA93B0
:100FB600EF9721978CE2002470E0E8E3FCE060E024
:100FC6000E9412C20E9404C2FE01EA5BFF4F019119
:100FD6001081EEA5FFA50E94F8BD0E171F0710F49D
:100FE6000C94FC87E0E9F1E00E940BC2EF9629968B
:100FF60008954E815F814017510710F40C940888BC
:101006000E945CADEF9629960895D8010E949F87AD
:10101600EBAFF0E0DE0116960E94E1B14D915C91D6
:10102600EBADEF5FF0E0DE0116960E9464B60E941B
:10103600F8BDE41BF50BEEAFFFAFABAD0E94988792
:10104600DE01AE5BBF4FED93FC93EBADEF5FEAAF16
:10105600AAAD0E949887DE01A05CBF4FED93FC937A
:10106600DE01AE5BBF4F0D90BC91A02DEA1BFB0BC2
:10107600ECAFFDAFEEADFFAD309711F00C944788A5
:10108600E4E1F0E0EEAFFFAFECADFDAD0E94FEBDDA
:10109600DF01CB01EEADFFAD0E94FEBD0E942DC566
:1010A600EEABFFAB68AF79AFF801E41BF50B0E941E
:1010B600FEBDEAABFBAB6CAB7DABEEA9FFA968ADA1
:1010C60079ADAAA9BBA98CA99DA90E94DFC4EAABE8
:1010D600FBAB6CAB7DAB0E9422C49F01FE01EE5BB5
:1010E600FF4F0190F081E02D2E0F3F1FF9010E9466
:1010F6000BC2EF9629960895BA93AA9366970E9413
:1011060004C2E0E0F0E46CE975E40E94BCB744EE8A
:101116005CE0E0E0F0E46CE17AE40E9443B00E9417
:10112600D0B7E0E0F0E060E874E40E942DC50E94CC
:1011360043B00E94D0B7E0E0F0E06AE774E40E94B2
:101146002DC50E9443B0EC8DFD8D0E94FEBD0E9410
:1011560003BE0E94F3BD0E9408BEEE8BFF8B688F14
:10116600798FAE89BF89888D998D0E941CB10E94A6
:101176008EC4EE87FF87688B798BAE89BF89888D91
:10118600998D0E942DC50E9403BEFA010E94FEBDE4
:101196000E9408BE0E9403BEEA89FB896C897D898C
:1011A6000E9422C4EA8FFB8FAA8DBB8D0E94D9872D
:1011B6008F0130969F010E940BC26E9608950E9481
:1011C60004C29D014E815F812A32E3E03E0710F49E
:1011D6000C94EF882AE233E000E010E00A32E3E004
:1011E6001E0710F00C94FE88A1E7B7E10E9445AEF9
:1011F6000F5F1F4FF3CF20939B1A30939C1A5A937D
:101206004A93E1E7F7E1FA93EA93A0919B1AB0912A
:101216009C1A0E94E71B0E940FBEEF58F84EA0E0F2
:10122600A083E0E0E0939F1AE093A01AE0939D1A52
:10123600E0939E1AE093A11AE093A21AE093A31AF0
:10124600E093A41A0E94DAB40895AA932697D1507F
:101256000E9404C2FE01E35FFE4F0190F081E02D83
:10126600EA87FB87FE01E45FFE4F10810E9414BEF1
:1012760010F00C944289E0E00E941DBE08950E9481
:1012860022BE0E9429BE0E9432BE0E9439BE10F0C4
:101296000C946189FA01DE011C96EA0FFB1FFF938D
:1012A600EF93FA010E9429BE0E94CAAE6BBFE69177
:1012B600AF91BF91EC934F5F5F4FE7CF0E943EBE69
:1012C60001E040E050E0FA010E94B3AF0E944ABE3E
:1012D60011F40C946F8900E04F5F5F4F0E9439BE96
:1012E60010F00C947B89013011F00C947B8901C0BD
:1012F60001C0E9CF0E940EAEAE81BF812A173B071F
:1013060010F40C948B89003011F00C948B8901C079
:1013160001C0D6CF0E9454BE11F40C9495890E9448
:1013260069BE02C00E9476BE003011F40C94A089FA
:10133600103011F40C94A08901C005C00E947FBE34
:101346000E941DBE0895003011F40C94AE89E1E0B0
:101356000E941DBE0895E0E00E941DBE08950E94F1
:101366001DBE0895AA932697D1500E9404C2FE017D
:10137600E25FFE4F0190F081E02DEA87FB87FE01D8
:10138600E35FFE4F10810E9414BE10F00C94CE89CC
:101396000E9489BE08950E9422BE0E948FBE0E94AE
:1013A60032BE0E9439BE10F00C94ED89FA01DE01BE
:1013B6001C96EA0FFB1FFF93EF93FA010E948FBE64
:1013C6000E94CAAE6BBFE691AF91BF91EC934F5F9F
:1013D6005F4FE7CF0E943EBE01E040E050E0FA01D9
:1013E6000E94B3AF0E944ABE11F40C94FB8900E040
:1013F6004F5F5F4F0E9439BE10F00C94078A013090
:1014060011F00C94078A01C001C0E9CF0E940EAE0C
:10141600EE81FF81EF58F84EA081FE01E45FFE4F9A
:10142600E081EA1711F00C94238A103011F40C9421
:10143600208AEE81FF810E9498BE0E9489BE08958F
:10144600AE81BF812A173B0710F40C942F8A003017
:1014560011F00C942F8A01C001C0BECF0E9454BE69
:1014660011F40C94398A0E9469BE02C00E9476BEAD
:10147600003011F40C94448A103011F40C94448A10
:1014860001C005C00E947FBE0E949DBE0895003027
:1014960011F40C94528AE1E00E949DBE08950E94C8
:1014A60089BE08950E949DBE08950E9404C25A2FC7
:1014B60040E0E52F0E94A2BE8F012091A31A309131
:1014C600A41A2017310710F00C94798AE42F4F5F85
:1014D600AE81BF810E9478B1A1E7B7E1A20FB31F29
:1014E600EC91D001EC932F5F3F4FEBCFAE81BF81E4
:1014F6000E94AABE0E940BC228960895E091A31AE4
:10150600F091A41A0E9498BE08950A930A2FE02F1C
:10151600A0919F1AB091A01AF0E0EA0FFB1F0E945B
:1015260098BEE02F0E94A2BEE093A31AF093A41ADD
:1015360009910895AA9321970E94ABB240E0EF81EA
:101546000E94A2BE8F012091A31A3091A41A2017DF
:10155600310710F00C94CF8AA1E7B7E1A20FB31FB1
:101566005C91523211F00C94C18AA885B9850E940B
:10157600AABEEE810E940BC22A960895E42F4F5F01
:10158600A885B985F0E0EA0FFB1F5083EE81EF5F77
:10159600EE832F5F3F4FDBCF2093A31A3093A41A1D
:1015A6000E9430AF08950A93E0E0E093D71AE093E3
:1015B600D81A0E942AB30E9464B311F00C94E68AEA
:1015C600A0E10E94DD0FA1E00E94FE280E949BB6CA
:1015D6000E94D7160E946F170E9434B2E1E0E09392
:1015E600D71AE0E0E093D91AE093D81AE8ECE09332
:1015F600D61AEAEDFAE10E9416B80E94B3BEEAEEE8
:10160600FAE10E9416B80E946DB8E2EFFAE10E9474
:1016160016B80E946DB8E0E0E093FA1AE093FB1A60
:10162600E093FC1AE093FD1AE093FE1A09910895DF
:101636000E94D68AE1E0E093D71A0895A0E00E94BE
:10164600FE28E3E6E093D71AA0E10E94DD0F089595
:101656006D970E9404C2E091D71AE03011F00C9405
:10166600398BE0E00E940BC2A3960895A091D71A89
:10167600A33611F00C94498BE0E00E94B8B40E94A6
:10168600A363E0E00E940BC2A3960895A091D71A27
:10169600A13011F00C94628BA0E10E94F40F8F012F
:1016A600093CE0E01E0710F40C945E8BE0E0E0934A
:1016B600EB120E94B7BEE0E0E093D81AE9C1A09110
:1016C600D71AA23011F00C946E8BE0EF0E94BDBECB
:1016D6000E94B7BEDDC1A091D71AA33011F00C94B9
:1016E600B18BEDB7FEB7FA93EA935F930E94C7BE3C
:1016F6005F914E2F403011F00C94988B513010F4BE
:101706000C948C8BE1E00E94CFBEEAEC0E94D5BE21
:101716000895E1E0E093EB12AFE00E94DD0FACE04C
:101726000E9423100E94B7BE0BC0423010F40C94E6
:10173600A38BE2E00E94CFBEE9EC0E94D5BE0895DD
:10174600AFE00E942FB910F40C94B08BE3E00E9436
:10175600CFBEE8EC0E94D5BE08959AC1A091D71AD3
:10176600A43011F00C94FE8B0E94F5284E2F4030C9
:1017760011F40C94CE8B0E946F17E1E00E94BDBE5F
:10178600ACE00E942310E2E0EA93EA93A2E00E9412
:10179600A3630E94B7BEE1E00E94B8B40E94A363AF
:1017A600ACE00E943F108F010630E0E01E0710F407
:1017B6000C94E48BA091FA12A03011F00C94E48BF7
:1017C6000EC00F31E0E01E0710F40C94F18BA091CF
:1017D600FA12A13010F40C94F18B01C00BC0E0E0BA
:1017E6000E94B8B40E94A363E0E00E94CFBE0E94AC
:1017F600DCBE08954DC1A091D71AA53011F00C9406
:10180600408CEDB7FEB7FA93EA935F930E94C7BE8A
:101816005F914E2F403011F00C94298C513010F40A
:101826000C941B8CE4E00E94CFBE0E94DCBE08959F
:10183600AFE00E94DD0FE8A1EA93DE0117960E9451
:10184600B1940E9482910E94B7BE0AC0423010F441
:101856000C94338CE5E00E94CFBE0E94DCBE089556
:10186600AFE00E942FB910F40C943F8CE6E00E9482
:10187600CFBE0E94DCBE08950BC1A091D71AA63038
:1018860011F00C946E8C0E948C8F4E2F413010F408
:101896000C94538CE7E00E94CFBE0E94DCBE0895F4
:1018A600AFE00E94DD0F0E94B7BEE0E00E94B8B430
:1018B6000E94A363AFE00E94F40F8F01053FE1E0B1
:1018C6001E0710F40C946D8CE8E00E94CFBE0E94B7
:1018D600DCBE0895DDC0A091D71AA73011F00C9494
:1018E6008D8CAAEDBAE10E949B90AAEEBAE10E9405
:1018F600AE90A2EFBAE10E94C1900E94D790E09309
:10190600FA1AF093FB1A6093FC1A7093FD1A0E9460
:10191600B7BEBEC0A091D71AA83011F00C941F8D87
:10192600E0E0E093FE1A0E949BB70E94E1BEE4EB62
:10193600FCE060E070E00E94E4BEEAEDFAE10E949D
:101946003BAFA0E1B0E00E94D21A2E2F0E949BB7B7
:101956000E94E1BEE5ECFCE060E070E00E94E4BEBF
:10196600EAEEFAE10E943BAFA8E0B0E00E94D21A8C
:101976003E2F203011F40C94C58C303011F40C94A9
:10198600C58C01C047C0A091EF1AA43411F00C9485
:10199600D38CA091F01AA53511F00C94D38C01C00C
:1019A60004C0E1E0E093FE1A35C0A091EF1AA4341A
:1019B60011F00C94E58CA091F01AA63511F00C9458
:1019C600E58C01C004C0E2E0E093FE1A23C0A091BA
:1019D600EF1AA43511F00C94F78CA091F01AA035EB
:1019E60011F00C94F78C01C004C0E3E0E093FE1AFA
:1019F60011C0A091EF1AA43511F00C94098DA09195
:101A0600F01AA33411F00C94098D01C003C0E4E070
:101A1600E093FE1AA091FE1AA13010F40C94188DD2
:101A2600A43610F00C94188D01C003C0ABE00E94E0
:101A360023100E94B7BE2CC0A091D71AA93011F06E
:101A46000C94428DA091FA1AB091FB1A8091FC1A5F
:101A56009091FD1A0E945F932E2F203011F40C9462
:101A66003B8DA091FE1AA13010F40C943B8D01C061
:101A760003C0E4E6E093FE1A0E94B7BE09C0A09137
:101A8600D71AAA3011F00C944B8DE3E6E093D71ADF
:101A96000E94DCBE08951A930A938D01A091FE1A46
:101AA600A13010F40C945C8DA43610F00C945C8D6F
:101AB60001C009C0E2EFFAE1FA93EA931A930A9396
:101AC6000E940CBA06C01A930A93E0E0EA930E94B9
:101AD6006DB8E091FE1A0991199108951A930A9327
:101AE600ABE00E94D6BA10F40C947C8DE0E0E09353
:101AF600FE1AA091FE1AA13010F40C94878DA4361C
:101B060010F00C94878D01C004C0E1E00991199191
:101B16000895E0E0099119910895E0E0E093FE1A36
:101B260008950E9404C21A2F2E813F814885598547
:101B36000C85043010F00C94C88DA7E00A9FF001C4
:101B4600EB55F54EAB85A083A7E00A9FF001EA5559
:101B5600F54EAA85A083A7E00A9FF001E955F54E48
:101B660050830A9FF001E855F54E40830A9FF00125
:101B7600E755F54E30830A9FF001E655F54E208372
:101B86000A9FF001E555F54E10830E940BC22D9673
:101B960008950E9406C29D010C91043010F00C9429
:101BA600018EA7E00A9FF001EB55F54EA081AB3BF5
:101BB60011F00C94E38DF9013196ABEBA08304C0D0
:101BC600F9013196AAEAA08310E0163010F00C94C1
:101BD600008EE12FF0E03296E20FF31FBF01A7E07F
:101BE6000A9FF001EA55F54EDF01EE27A10FBE1F51
